:020000040800F2
:203000001822002001310008970C0108D9C30008950B0108AD4900087D4C01080000000053
:2030200000000000000000000000000007280108F56A000800000000F90F01086D37010833
:203040001B3100081B3100081B3100081B3100081B3100081B3100081B3100081B310008D0
:20306000D57000081B3100081B310008B95900081B3100081B3100081B3100081B310008F1
:203080001B3100081B310008854200081B310008D14801081B3100081B3100081B31000847
:2030A0001B310008993801081B3100081B3100081B3100081B3100081B3100081B310008EA
:2030C0001B3100081B3100081B3100081B3100081B3100081B3100081B310008E54701086F
:2030E000C97000081B3100081B310008DFF80CD001F078F80048004761420008182200203F
:203100000648804706480047FEE7FEE7FEE7FEE7FEE7FEE7FEE7FEE7FEE7FEE74138010891
:20312000ED3000082DE9FF1F002000210022002300240025002600275FF000085FF000096B
:203140005FF0000A5FF0000B5FF0000C002001210222032304240525062607275FF00808CA
:203160005FF009095FF00A0A5FF00B0B5FF00C0C00281DD101291BD1022A19D1032B17D167
:20318000042C15D1052D13D1062E11D1072F0FD1B8F1080F0CD1B9F1090F09D1BAF10A0FDA
:2031A00006D1BBF10B0F03D1BCF10C0F00D101E004F028BCBDE8FF1F7047000073B400208B
:2031C00000210124002501262046A04226D1A94224D12846A84221D1A9421FD14FEA440498
:2031E00006F10106202EEFDD5FF0FF305FF0FF317FF000445FF0FF3501262046A0420DD137
:20320000A9420BD12846A84208D1A94206D14FEA740406F10106202EEFDD01E004F0F2BBA9
:2032200073BC7047E7B40021002000220125002601272946A94230D1B0422ED1B2422CD1F9
:203240003146B14229D1B04227D1B24225D14FEA450507F10107202FEBDD5FF0FF315FF0CE
:20326000FF305FF0FF327FF000455FF0FF3601272946A94211D1B0420FD1B2420DD13146E8
:20328000B1420AD1B04208D1B24206D14FEA750507F10107202FEBDD01E004F0B3BBE7BC1A
:2032A00070472DE9CE01002200210023012600275FF001083246B24233D1B94231D1BB42FC
:2032C0002FD13A46BA422CD1B9422AD1BB4228D14FEA460608F10108B8F1200FEADD5FF014
:2032E000FF325FF0FF315FF0FF337FF000465FF0FF375FF001083246B24212D1B94210D1E0
:20330000BB420ED13A46BA420BD1B94209D1BB4207D14FEA760608F10108B8F1200FEADD79
:2033200001E004F06FBBBDE8CE0170472DE99C0300230022002401275FF000085FF001096D
:203340003B46BB4233D1424531D144452FD1434643452CD142452AD1444528D14FEA470740
:2033600009F10109B9F1200FEADD5FF0FF335FF0FF325FF0FF347FF000475FF0FF385FF09B
:2033800001093B46BB4212D1424510D144450ED1434643450BD1424509D1444507D14FEA0A
:2033A000770709F10109B9F1200FEADD01E004F029BBBDE89C0370472DE9381C0024002386
:2033C00000255FF0010A5FF0000B5FF0010C5446544533D15B4531D15D452FD15C465C45FA
:2033E0002CD15B452AD15D4528D14FEA4A0A0CF1010CBCF1200FEADD5FF0FF345FF0FF335D
:203400005FF0FF357FF0004A5FF0FF3B5FF0010C5446544512D15B4510D15D450ED15C46D1
:203420005C450BD15B4509D15D4507D14FEA7A0A0CF1010CBCF1200FEADD01E004F0E2BA40
:20344000BDE8381C70472DE9701C0025002400265FF0010A5FF0000B5FF0010C5546554566
:2034600033D15C4531D15E452FD15D465D452CD15C452AD15E4528D14FEA4A0A0CF1010CF1
:20348000BCF1200FEADD5FF0FF355FF0FF345FF0FF367FF0004A5FF0FF3B5FF0010C5546C7
:2034A000554512D15C4510D15E450ED15D465D450BD15C4509D15E4507D14FEA7A0A0CF1BA
:2034C000010CBCF1200FEADD01E004F09BBABDE8701C70472DE9E01C0026002500275FF057
:2034E000010A5FF0000B5FF0010C5646564533D15D4531D15F452FD15E465E452CD15D45A2
:203500002AD15F4528D14FEA4A0A0CF1010CBCF1200FEADD5FF0FF365FF0FF355FF0FF374D
:203520007FF0004A5FF0FF3B5FF0010C5646564512D15D4510D15F450ED15E465E450BD1AA
:203540005D4509D15F4507D14FEA7A0A0CF1010CBCF1200FEADD01E004F054BABDE8E01C85
:2035600070472DE9C01D002700265FF000085FF0010A5FF0000B5FF0010C5746574533D1B0
:203580005E4531D1D8452FD15F465F452CD15E452AD1D84528D14FEA4A0A0CF1010CBCF12B
:2035A000200FEADD5FF0FF375FF0FF365FF0FF387FF0004A5FF0FF3B5FF0010C57465745AF
:2035C00012D15E4510D1D8450ED15F465F450BD15E4509D1D84507D14FEA7A0A0CF1010C2A
:2035E000BCF1200FEADD01E004F00CBABDE8C01D70472DE9801F5FF0000800275FF00009C9
:203600005FF0010A5FF0000B5FF0010CD046D04533D15F4531D1D9452FD1D846D8452CD16F
:203620005F452AD1D94528D14FEA4A0A0CF1010CBCF1200FEADD5FF0FF385FF0FF375FF040
:20364000FF397FF0004A5FF0FF3B5FF0010CD046D04512D15F4510D1D9450ED1D846D845C9
:203660000BD15F4509D1D94507D14FEA7A0A0CF1010CBCF1200FEADD01E004F0C3B9BDE89A
:20368000801F70472DE970075FF000095FF000085FF0000A012400250126A146A14530D100
:2036A000A8452ED1AA452CD1A946A94529D1A84527D1AA4525D14FEA440406F10106202EC4
:2036C000EBDD5FF0FF395FF0FF385FF0FF3A7FF000445FF0FF350126A146A14511D1A84594
:2036E0000FD1AA450DD1A946A9450AD1A84508D1AA4506D14FEA740406F10106202EEBDD14
:2037000001E004F07FB9BDE8700770472DE9700E5FF0000A5FF000095FF0000B01240025E0
:203720000126A246A24530D1A9452ED1AB452CD1AA46AA4529D1A94527D1AB4525D14FEADA
:20374000440406F10106202EEBDD5FF0FF3A5FF0FF395FF0FF3B7FF000445FF0FF35012618
:20376000A246A24511D1A9450FD1AB450DD1AA46AA450AD1A94508D1AB4506D14FEA740403
:2037800006F10106202EEBDD01E004F03BB9BDE8700E70472DE9701C5FF0000B5FF0000A1D
:2037A0005FF0000C012400250126A346A34530D1AA452ED1AC452CD1AB46AB4529D1AA45C5
:2037C00027D1AC4525D14FEA440406F10106202EEBDD5FF0FF3B5FF0FF3A5FF0FF3C7FF06B
:2037E00000445FF0FF350126A346A34511D1AA450FD1AC450DD1AB46AB450AD1AA4508D106
:20380000AC4506D14FEA740406F10106202EEBDD01E004F0F7B8BDE8701C70472DE9701811
:203820005FF0000C5FF0000B012400250126A446A44526D1AB4524D1AC46AC4521D1AB45EE
:203840001FD14FEA440406F10106202EEFDD5FF0FF3C5FF0FF3B7FF000445FF0FF3501266F
:20386000A446A4450DD1AB450BD1AC46AC4508D1AB4506D14FEA740406F10106202EEFDD7F
:2038800001E004F0BFB8BDE8701870472DE9F0030024002546594E51445105F10405182D8F
:2038A000F8DB04255FF0000801245FF0010944514659B4425FD105F10407C659B0455AD19D
:2038C0002F1FC659B04556D140F805804659B04551D105F10407C659B0454CD12F1FC6594D
:2038E000B04548D14FEA440409F10109B9F1200FDDDD05F10405142DD6DB5FF0FF3400250A
:20390000445105F10405182DFADB04255FF0FF387FF000445FF0010944514659B4422AD119
:2039200005F10407C659B04525D12F1FC659B04521D140F805804659B0451CD105F10407E9
:20394000C659B04517D12F1FC659B04513D14FEA740409F10109B9F1200FDDDD05F10405DE
:20396000142DD5DB00254E59465105F10405182DF9DB012000E00020BDE8F00370472DE955
:20398000F00300240025445105F104058D42FADB00255FF0000801245FF001094451465985
:2039A000B44268D1002D03D02F1FC659B04562D105F104078F4202DAC659B0455BD140F81D
:2039C00005804659B04556D1002D03D02F1FC659B04550D105F104078F4202DAC659B04562
:2039E00049D14FEA440409F10109B9F1200FD5DD05F104058D42CEDB5FF0FF3400254451EA
:203A000005F104058D42FADB00255FF0FF387FF000445FF0010944514659B4422BD1002DF9
:203A200003D02F1FC659B04525D105F104078F4202DAC659B0451ED140F805804659B04559
:203A400019D1002D03D02F1FC659B04513D105F104078F4202DAC659B0450CD14FEA7404E6
:203A600009F10109B9F1200FD5DD05F104058D42CDDB012000E00020BDE8F0037047202A87
:203A800004DB203A21FA02F00021704721FA02F3D040C2F12002914008431946704740EAB7
:203AA00001039B0703D009E008C9121F08C0042AFAD203E011F8013B00F8013B521EF9D249
:203AC0007047D2B201E000F8012B491EFBD270470022F6E710B513460A4604461946FFF7AF
:203AE000F0FF204610BD10B5044604E00B7800F8013B03B1491C521EF8D2204610BD421C16
:203B000010F8011B0029FBD1801A704730B505460020034600E05B1C934205D2EC5CC85C33
:203B2000201A01D1002CF6D130BDF0B480EA0102D40F4200B2EB410F02D2024608461146B5
:203B40004A0042D0C30DDDB2C1F3C752AD1A202D35DAC1F3160141F4000204B15242C5F1B9
:203B6000200602FA06F12A411044B3EBD05F23D0C4B1012DA0EBC35009DCF0BC4FF000425A
:203B800002EAC352DBB200F5000000F04FBA400000F1807000EBC350A0F1807040EAD1709E
:203BA000490009E0490841EAC071A0EBC35000F50000400800EBC350F0BC00F02EBA614226
:203BC000012202EB4101001BF6E7F0BC704781F00041AAE780F00040A7E780EA010210B585
:203BE00002F00043400022D04A001FD0010E01EB1261C0F35600C2F3560240F4000042F437
:203C00000002A0FB022000047F39140400D0401C50EA124001D44000491EC2B20C0604EB68
:203C2000D010401C4008802A02D003E0002010BD20F00100002900DA0020184310BD2DE942
:203C4000FE4F804681EA0300C00F0C46009021F0004123F00045B8EB0200A94105D240469C
:203C6000214690461C460B46024623F00040104347D0270DC7F30A00C3F30A510290401A5A
:203C8000019040286BDAC3F3130040F4801B0098924620B10023D2EB030A63EB0B0B019823
:203CA0005946C0F14002504600F096F906460D4650465946019A00F09EF910EB08006141C2
:203CC000002487EA115284EAE7731A4340D0009A62B3019A012A4FEA075215DC001B61EB58
:203CE00002014FF0004202EA0752CDE90042001C41F5801132462B4600F0D5F903B0BDE821
:203D0000F08F40462146F9E7001B61EB0201001C41F5801300185B412018A2F5001747EB3C
:203D2000030140EAD570B6196D4111E06D084FEA360645EAC0754FEA0752001B61EB020158
:203D4000001C41F5801149084FEA30000019514132462B4603B0BDE8F04F00F095B90098C5
:203D6000012240000023D0EB020263EBE073009821464FEAE074B8EB000061EB0401E9E70D
:203D800083F000435BE781F0004158E72DE9F04D81EA030404F0004B21F0004514464FF047
:203DA000000A23F0004150EA050220D054EA01021DD0C5F30A570246C5F31303C1F3130050
:203DC000C1F30A5640F4801543F48013A7EB0608101BD64608F2FD3873EB050002D308F1F5
:203DE000010801E092185B41B8F1000F03DA00200146BDE8F08D00204FF48011064684466B
:203E00000EE0171B73EB050705D3121B63EB050306434CEA010C49084FEA300092185B4131
:203E200050EA0107EDD152EA030012D082EA040083EA0501084305D0101BAB4106D201224C
:203E4000002306E000224FF0004302E06FF0010253101AEB06004CEB085110EB0A0041EB42
:203E60000B01BDE8F04D00F00FB996230022114600F0DCB80EB5C10F80EAE0700844CA077C
:203E8000002140F233438DE80E000A460B4600F00AF903B000BD0EB540F2334102910021B5
:203EA000CDE900110A460B4600F0FDF803B000BD00F0004220F00040C10DC0F3160040F4F8
:203EC00000007F2901DA00207047962903DCC1F19601C84001E096398840002AF4D04042B1
:203EE000704720F00040C10DC0F3160040F400007F2901DA00207047962903DCC1F19601AF
:203F0000C840704796398840704770B5C1F30A5201F000450024C1F3130140F2FF3341F4A4
:203F200080119A4201DA002070BD40F233439A42A2F2334203DC5242FFF7A1FD00E09040A8
:203F40002C43F1D0404270BDC1F30A5210B5C1F3130140F2FF3341F480119A4201DA0020E4
:203F600010BD40F233439A42A2F2334203DC5242FFF785FD10BD904010BD00F0004230F040
:203F800000400AD0C10D01F56071C0F3160042EA0151C208400711437047002001467047F1
:203FA00001F0004330B421F0004150EA010206D00A0DA2F56072C1F31301002A02DC30BC48
:203FC00000207047440F44EAC104C100E01830BC00EBC25000F021B8202A04DB203A00FADC
:203FE00002F1002070479140C2F1200320FA03F3194390407047202A06DBCB17203A41FABB
:2040000002F043EAE07306E041FA02F3D040C2F1200291400843194670470029A8BF7047BA
:20402000401C490008BF20F00100704710B4B0FA80FC00FA0CF050EA010404BF10BC7047E7
:2040400049B1CCF1200421FA04F411FA0CF118BF012121430843A3EB0C01CB1D4FEA0061A5
:204060004FEA102042BF002010BC704700EBC35010440029A4BF10BC7047401C490008BF66
:2040800020F0010010BC704710B5141E73F1000408DA401C41F1000192185B411A4301D147
:2040A00020F0010010BD2DE9F04D92469B4611B1B1FA81F202E0B0FA80F220329046FFF71A
:2040C0008BFF04460F4640EA0A0041EA0B0153465A46084313D0114653EA010019D0C8F1AE
:2040E00040025046FFF7CBFC05460E46504659464246FFF771FF084305D0012004E02046DE
:204100003946BDE8F08D0020054346EAE0762C4337430A986305E40AA0EB08000022FD0A73
:2041200044EA47540A3002D500200146E9E7010510196941DDE9084500196941BDE8F04DDD
:20414000A2E72DE9F04D00231A461B1A8A4103DB00200146BDE8F08DC1F30A52C1F31301C1
:2041600041F480154FF0000BD10702D100186D41521E0027044640F2FF11384601EB620AC1
:204180003E468046024600204FF48011FFF777FCC2197141BB1846EB0100B4EB030C75EB90
:2041A000000C04D3E41A65EB000517460E46241908F101006D4180463428E3DDF91946EB0E
:2041C0000600091BA84103D24FF0FF32134601E0002213461BEB070046EB0A51BDE8F04D57
:2041E000FFF752BF064C074D06E0E06840F0010394E8070098471034AC42F6D3FEF77AFFE5
:20420000E07D0108007E010870B58C1810F8015B15F0070301D110F8013B2A1106D110F845
:20422000012B03E010F8016B01F8016B5B1EF9D12B0705D40023521E0DD401F8013BFAE7BE
:2042400010F8013BCB1A921C03E013F8015B01F8015B521EF9D5A142D8D3002070BD0000CF
:2042600010B572B606480079AA2801D00EF0CCF900200349087162B611F0EAF810BD000077
:204280000030024010B5024804F0F4FC10BD00006416002070B5044600252068806800F05E
:2042A0000100F0B12068806820F001002168886006F0FCF905460EE006F0F8F9401B0228DA
:2042C00009D9A06A40F01000A062E06A40F00100E062012070BD2068806800F0010000281C
:2042E000EAD10020F6E770B505466C6AA06A00F05000E0B9A06A40F40070A06220688068BD
:2043000000F46020B0F5602F0DD1E06858B9A06A20F48070A062A06A00F4805018B9A06A05
:2043200040F00100A062204604F054F903E0206A016B2846884770BD70B505466C6AA06A10
:2043400040F04000A062E06A40F00400E062204604F08FFC70BD70B50446656A284604F079
:2043600087FC70BD38B504460025002000902068806800F0010080BB2068806840F0010044
:2043800021688860164800681649B0FBF1F0009002E00098401E009000980028F9D106F083
:2043A00085F9054613E006F081F9401B02280ED9A06A40F01000A062E06A40F00100E0625C
:2043C00000BF002084F8240000BF012038BD2068806800F001000028E5D00020F6E700004E
:2043E0000000002040420F0070B505460E4606F05DF922490968401A02283DD3002418E070
:204400001F4850F824001F4931F81410C0EB81201B4951F8241001EBE010194941F824004C
:20442000084650F82400C0F38F2025F81400601CC4B20B2CE4DB002418E0134850F8240064
:20444000124931F81410C0EB81200F4951F8241001EBE0100C4941F82400084650F824004B
:20446000C0F38F2026F81400601CC4B2032CE4DB06F01CF90149086070BD00006C0400204E
:20448000D816002008160020041700201404002010B5154803F062FD144803F05FFD1248E4
:2044A00004F09EFD114804F09BFD104803F066FF0B220F490C4804F02BFE0B48006A0068BD
:2044C000006820F004000849096A09680860094807F02DF90C21074807F0A0FB0C210548CD
:2044E00007F046F810BD000034160020641600200816002048150020014600226648814221
:204500000DD1664848604A68824201D000207047634848604A68824201D00020F7E7614808
:2045200081420DD1604848604A68824201D00020EDE75E4848604A68824201D00020E6E7CD
:2045400040F2555048614A69824201D00020DEE740F6AA2048614A69824201D00020D6E7E0
:2045600040F2555088618A69824201D00020CEE740F6AA2088618A69824201D00020C6E7E0
:2045800040F25550C861CA69824201D00020BEE740F6AA20C861CA69824201D00020B6E7E0
:2045A00040F2555008620A6A824201D00020AEE740F6AA2008620A6A824201D00020A6E7DC
:2045C00040F2555048624A6A824201D000209EE740F6AA2048624A6A824201D0002096E7DC
:2045E00040F2555088628A6A824201D000208EE740F6AA2088628A6A824201D0002086E7DC
:204600002B48C862CA6A824201D000207FE72948C862CA6A824201D0002078E726480863F2
:204620000A6B824201D0002071E7244808630A6B824201D000206AE71F4848634A6B82421B
:2046400001D0002063E71D4848634A6B824201D000205CE71A4888638A6B824201D000206B
:2046600055E7184888638A6B824201D000204EE700204860C860086148618861C861086256
:2046800040F6FF70486200208862C86208634863886301203BE700000024014055554500FF
:2046A000AAAA8A000028014055554000AAAA800055555500AAAAAA0055555515AAAAAA2ABC
:2046C00055551500AAAA2A0088B001460022086800904868019088680290CB6803930B69FC
:2046E00004934B690593552008600A68552A02D0002008B07047AA2008600A68AA2A01D05F
:204700000020F6E745F2555048604A68824201D00020EEE74AF6AA20486048684AF6AA236D
:2047200000EA03021846824201D00020E1E745F2555088608A68824201D00020D9E742F64C
:20474000AA2088608A68824201D00020D1E745F25553CB60CA681846824201D00020C8E74A
:2047600042F6AA23CB60CA681846824201D00020BFE745F255530B610A691846824201D06D
:204780000020B6E742F6AA230B610A691846824201D00020ADE745F255534B614A69184635
:2047A000824201D00020A4E742F6AA234B614A691846824201D000209BE700980860019827
:2047C000486002988860039BCB60049B0B61059B4B6101208DE70246002004E0002322F871
:2047E0001030431C98B28842F8DB7047F0B50346002640F2FE34601E534F07EB80004288A8
:20480000154652480088401C504F3880384600880A2801DC0020F0BD4C4800880F2801DC56
:204820000A20F8E749480088142801DC1920F2E746480088192801DC2D20ECE743480088C4
:204840001E2801DC4120E6E740480088232801DC5520E0E73E48007801281FD100203C4FD1
:204860003870002110E00A2093FBF0F0364F37F82170B84205DB344800EB81004088151AE9
:2048800004E00025481C81B2A142ECDB00BF64206843B0FBF2F02F4F387051E02E48C07B4B
:2048A0002E4F3870384600782A4F38702C48006818442B4F38602B480078401C294F38700B
:2048C0003846007819283BDB254800681927B0FBF7F086B20020224F3860224F3870002149
:2048E00010E00A2096FBF0F0174F37F82170B84205DB154800EB81004088151A04E0002564
:20490000481C81B2A142ECDB00BF64206843B0FBF2F0104F387038460078104F3F78B842CE
:204920000EDD0C4807780D4800781E30874207DA084800785A2803DA08480078054F387009
:204940000448007867E70000906A0108F2020020FB020020F9020020B4070020FA020020FF
:20496000F4020020F802002038B504460B48012300220A2100900A4807F01AFF09480123A5
:2049800000220A210090084807F012FF03480078044909780840207038BD0000C60300209B
:2049A000A8140020C7030020BC14002000BFFEE700B58BB0002006900790012008904CF269
:2049C00020000190002002904CF2E01003904FF6FF700490002005900120099001A91548F5
:2049E00004F056FC20B140F2271113A010F0C6FA0120069000200790012008904FF46040B9
:204A00000190002002904CF2E01003904FF6FF700490002005900120099001A9054804F0F0
:204A200037FC20B14FF49E7103A010F0A7FA0BB000BD00004C1B00202E2E5C436F72655C40
:204A40005372635C63616E2E630000002DE9F04104460D46002700260DB9666B00E0A66B56
:204A6000206800F5D87000EB0510006800F00400B060B06858B9206800F5D87000EB051017
:204A8000006840F2FF7101EA505030600AE0206800F5D87000EB051000686FF0604101EAEF
:204AA000D0007060206800F5D87000EB0510006800F00200F060206800F5D87000EB051022
:204AC000406800F00F0030613562206800F5D87000EB05104068C0F30720F061206800F5F2
:204AE000D87000EB051080683075206800F5D87000EB05108068010A7175206800F5D8707E
:204B000000EB05108068010CB175206800F5D87000EB05108068000EF075206800F5D87095
:204B200000EB0510C0683076206800F5D87000EB0510C068010A7176206800F5D87000EB18
:204B40000510C068010CB176206800F5D87000EB0510C068000EF0764DB920202168C8608C
:204B60002068406920F00A002168486108E02020216808612068406920F0500021684861DB
:204B800094F83C70222F01D0322F05D12068406920F40F4021684861CDB994F83C00422806
:204BA00004D0622806D072280CD107E0122084F83C000BE0322084F83C0007E0522084F8AF
:204BC0003C0003E0012084F83C0000BF19E094F83C00522804D0622806D072280CD107E051
:204BE000122084F83C000BE0222084F83C0007E0422084F83C0003E0012084F83C0000BF6A
:204C000000BF204604F01AFE0020BDE8F08100002DE9F34F83B0044660790B287EDB0021D2
:204C2000204610F0F5FA00906449009808700121204610F0EDFA8246604981F801A0009840
:204C400055286CD1BAF1AA0FFBD12088000A88702078C8700221204610F0DAFA06465749A7
:204C60000E71112E03D0162E01D00C2E7ED10321204610F0CDFA8046504880F80580052133
:204C8000204610F0C5FA83460421204610F0C0FA0BEB00201FFA80F94FEA1920474988713E
:204CA00081F807900521204610F0B2FA0546A8EB0500022872D1617908F10900814217DACC
:204CC000207C012804D105F0F1FCE0600020207405F0ECFCE168411A0498814205D96179CC
:204CE000204610F051FA0120207405B0BDE8F08F0120207400270EE0B81DC1B2204610F0FD
:204D000087FA2F49C8550846C15D07F108002B4A1154781C87B2AF42EEDB01E04CE047E07C
:204D2000A81DC1B2204610F073FA4FEA006BE81DC1B2204610F06CFA0BEB004B05F1080041
:204D4000C1B2204610F064FA0BEB002B05F10900C1B2204610F05CFA0BEB0001019105F14E
:204D60000801164800F038F9029000E01BE0DDE90110081A0CD12088114B4A46314600F06D
:204D8000A3FE08F10900C1B2204610F0FDF9ACE70121204610F0F8F90EE0FFE70121204639
:204DA00010F0F2F908E00121204610F0EDF903E00121204610F0E8F900BF96E72B0B0020D4
:204DC0002C0A002030B50A4600211CE00F4B5B6B14335B5CC57884686355C3785B1CDBB2ED
:204DE000C3708478A34201DB0023C37043795B1CDBB243718478A34203DD83784371012365
:204E000083714B1CD9B29142E0DB30BD4C1B00202DE9F047824688461446002C5FDD20469F
:204E2000E11704EB5171C910A4EBC1018FB237B90827E11704EB5171C1F3CF0907E02046BD
:204E4000E11704EB5171C910491C1FFA81F92548006BC0F800A000202249096BC860214917
:204E6000096B886000261CE008201E49096B086100250AE0082000FB065018F8001019483F
:204E8000006B14304155681C85B2082DF2DB0A21144804F043FD012801D10BF06BFC701C6C
:204EA00086B2A9F10100B042DEDC0E48006B076100250AE0082000FB065018F80010094851
:204EC000006B14304155681C85B2BD42F2DB0A21044804F023FD012801D10BF04BFCBDE899
:204EE000F08700004C1B002010B504462068406920F001002168486194F83C00122805D159
:204F00002068406920F40F402168486194F83C00422804D0522806D072280CD107E02220D5
:204F200084F83C000BE0322084F83C0007E0622084F83C0003E0012084F83C0000BF00BF69
:204F4000204604F043FE002010BD000010B5014600224C69CB69552008600A68552A01D013
:204F6000002010BDA82008600A6802F0A802A82A01D00020F5E70A4848614A69824201D024
:204F80000020EEE7074848614A69824201D00020E7E74C61CB614FF4004008600120E0E742
:204FA000550501002A8A020030B503460C460021002200BF09E0985C80EA1120C0B2054D22
:204FC00035F8100080EA0121521CA242F3D388B230BD0000E0600108F0B502460B4600251D
:204FE000681E00210FE0565C7040002407E0060E064F57F8265000026840661CB4B2042CBE
:20500000F5DB4E1CB1B29942EDDBF0BDE062010800B585B000BF1848806940F004001649D3
:2050200088610846806900F00400009000BF00BF00BF0846806940F0080088610846806900
:2050400000F00800009000BF00BF08200190002002900120039001A9084805F087F94FF479
:2050600000400190002002900120039001A9044805F07CF905B000BD00100240000C014088
:20508000000801402DE9F84F04460D4616461F4600F0ECF8009000F0E9F8804600F0E6F843
:2050A00081460098404504D1C84502D1644880F800906448007830B9614800786049487014
:2050C0000120604908705E4800785D494978884238D05B4840785A49097801F003015A4A1F
:2050E000515C884209D10020607058490880584908806068401C606024E05148407850494B
:20510000097801F00301534A515C88420DD14F480088401C4D49088008460088042811DBA0
:2051200001206070002008800CE049480088401C47490880084600880A2803DD0120607084
:20514000002008804FF0020A3D48007800F001003B49497801F00101884227D005F0A6FAE0
:205160003D490968401A4FF47A71B1FBF0F03B49088005F09BFA3849086017B94FF0010A8B
:2051800000E0B246607858B935480078401C3449087008460078504504DB0120A07001E0BC
:2051A0000020A07005F082FA2E4908602E4800682A490988C0EB81202B49096801EB202030
:2051C0002949086008460068C0F3872020704FF0640B22480088142802DA4FF496700DE067
:2051E0001E480088282801DD642007E01B48008800EB80004FF4FA71A1EB40001FFA80FBC4
:205200000BFB05F0642190FBF1F085B205F04EFA14490968401AA8420BD90020A0700220E6
:205220006070002020700D4908800F4908600C4908700348007802494870BDE8F88F000091
:205240003403002036030020C47A0108380300203A030020C87A01083C030020440300208E
:2052600046030020480300204003002070B54FF40041084805F008FA05462C4608210648D3
:2052800005F002FA064644EA4600C4B204F0030070BD000000080140000C014000BF084A1C
:2052A0001268526A91B201EB810292004FF47A7392FBF3F202800022014B1B685A627047EC
:2052C0008815002010B54FF4FA710948FFF7A0FC4FF4FA710748FFF79BFC4FF4FA71064835
:2052E000FFF796FC4FF4FA710448FFF791FC10BD94040020A8040020BC040020D004002084
:20530000F0B58DB007460E46154618A103C9CDE90B0118A103C9CDE9070109AB00223146D8
:205320000BA80FF0DFFF05AB0022314607A80FF0D9FF002405E009A8005D01A90855601C74
:20534000C4B2082CF7DB002407E005A8015D01AA04F108001154601CC4B2082CF5DB294649
:2053600001A801F0CEFB0DB0F0BD000039FF6C063454333029270957FFFFFFFF30B50246F2
:205380000B460021002400BF0EE0481C84B207E0505C155DA84201D1002030BD601C84B2B0
:2053A0009C42F5DB481C81B29942EEDB0120F4E731B581B0BDF80400ADF80000BDF90400D9
:2053C00044F6E61500FB05F1C913BDF9060000FB05F2D2130C4613466042C01AC01A00B285
:2053E000ADF8020000983CBD10B590B01022694640480CF035FA044624B9102269463E484E
:20540000FEF74DFB102269463A4814300CF028FA04462CB91022694637481030FEF73FFB8C
:2054200020226946334828300CF01AFA044624B9202269463148FEF732FB102269462D488F
:205440004C300CF00DFA044624B9102269462C48FEF725FB10226946264860300CF000FA67
:20546000044624B9102269462648FEF718FB10226946204874300CF0F3F9044624B9102280
:2054800069462148FEF70BFB20226946194888300CF0E6F9044624B9202269461B48FEF7A4
:2054A000FEFA202269461348AC300CF0D9F9044624B9202269461648FEF7F1FA10226946C7
:2054C0000C48D0300CF0CCF9044624B9102269461048FEF7E4FA3C2269460648E4300CF019
:2054E000BFF9044624B93C2269460B48FEF7D7FA10B010BD08FC0108D40700202C090020BD
:205500004C0900205C0900206C0900209C080020BC080020DC0800203E13002010B50446D0
:20552000684B0C220421204602F0ACFC401C28B9644B0C220421204602F0A4FC624B01225E
:205540001221204602F09EFC401C28B95E4B01221221204602F096FC5B4B183B1822152197
:20556000204602F08FFC401C30B9574B183B18221521204602F086FC544B01222F2120464C
:2055800002F080FC401C28B9504B01222F21204602F078FC4D4B183B18223221204602F0B6
:2055A00071FC401C30B9494B183B18223221204602F068FC464B01224C21204602F062FC32
:2055C000401C28B9424B01224C21204602F05AFC3F4B183B18224F21204602F053FC401C39
:2055E00030B93B4B183B18224F21204602F04AFC384B30226921204602F044FC401C28B96D
:20560000344B30226921204602F03CFC31480068401C304908600B463022692120460DF0F1
:20562000AEFC401C28B92B4B3022692120460DF0A6FC294B10229B21204602F023FC401CF7
:2056400028B9254B10229B21204602F01BFC234B1022AD21204602F015FC401C28B91F4B1E
:205660001022AD21204602F00DFC1D4B0822C321204602F007FC401C28B9194B0822C32149
:20568000204602F0FFFB174B1022CD21204602F0F9FB401C28B9134B1022CD21204602F0D7
:2056A000F1FB114B0222DF21204602F0EBFB401C28B90D4B0222DF21204602F0E3FB002031
:2056C00010BD0000B009002008130020221300203C130020EC0800201C0900200C0A002096
:2056E0007A0100201C0A0020860300201CB52D492D4801F09DFC10222C492B4808300DF08B
:20570000DDFB10222949103127481C300DF0D6FB20222749244830300DF0D0FB102225495D
:20572000214854300DF0CAFB102223491E4868300DF0C4FB102221491B487C300DF0BEFB01
:2057400020221F49184890300DF0B8FB20221D491548B4300DF0B2FB10221B491248D83044
:205760000DF0ACFB3C2219490F48EC300DF0A6FB1748007800061649497800EB014014492E
:20578000897800EB01201249C9780844009004210F48FFF721FC019002226946024801F056
:2057A000A5FF1CBDFFFF010800FC0108D40700202C0900204C0900205C0900206C09002081
:2057C0009C080020BC080020DC0800203E130020CC7A010838B5054600240FF07BFB0FF08D
:2057E00053FB284601F0AEFA284601F067FA1F48008800909DF800200021284601F08EFB57
:20580000401C28B99DF800200021284601F086FB9DF801200121284601F080FB401C28B9A6
:205820009DF801200121284601F078FB02216846FFF7BAFB044622120221284601F06EFBD9
:20584000401C20B922120221284601F067FBE2B20321284601F062FB401C20B9E2B203219A
:20586000284601F05BFB002038BD0000D07A010810B5094A0949A2F10C00FFF741FD064B7D
:205880000C22042106480DF07AFB0648006820F400100449086010BDB00900207A01002025
:2058A000B40300206C01002070B50546002639480078C8B9002404E03748C0880644601CDF
:2058C00084B20A2CF8DB0A20B6FBF0F03349088004F0ECFE3249086004F0E8FE314908604D
:2058E00001202C4908704FE004F0E0FE2D490968401AB0F5FA7F03D904F0D8FE28490860BB
:205900002868C0F3804000283ED104F0CFFE24490968401AB0F5FA6F36D9002404E01E48C9
:20592000C0880644601C84B20A2CF8DB0A20B6FBF0F01A49088008460088B0F57A7F05DB20
:205940000846008840F6B831884219DD286820F4802000F5802028600720134948800F488F
:2059600000888880084601F037FC00200F4908700F484089401C0E49488102200D490870A9
:2059800004F094FE0649086004F090FE0549086070BD00004000002008160020380400206B
:2059A000440000204800002024120020040300201C0900207901002010B5024804F088F93B
:2059C00010BD0000941600203FB5044600252068009060680190A0680290E06803900020C7
:2059E000206045F2555020602568854202D0002004B030BD0020206042F6AA202060256835
:205A0000854201D00020F3E70020206045F25550606005200CF0E8FE656845F25550854241
:205A200001D00020E4E74AF6AA20606005200CF0DBFE65684AF6AA20854201D00020D7E799
:205A40004FF05530A060A568B5F1553F01D00020CEE74FF0AA30A060A568B5F1AA3F01D00F
:205A60000020C5E74FF05530E060E568B5F1553F01D00020BCE74FF0AA30E060E568B5F1EF
:205A8000AA3F01D00020B3E7019860600298A0600398E060009820600120A9E730B590F88E
:205AA00040500124AC40C56B6C60046863604468102C04D10468A2600468E16003E00468F3
:205AC000A1600468E26030BD2DE9F84306460F4615461C4605F0FF0940F23171701A8E4250
:205AE00072D00ADCA6F2516000286BD0CF280DD0D0280CD0DF287DD165E00F287BD01028D6
:205B00007AD01F2879D02028F5D1DAE200BF41F20C61681A8D4236D00BDCA5F58050A0F149
:205B2000100070B1B0F53E7F23D0B0F5806F45D123E0B0F5807F2CD0A0F5C850F93878BB81
:205B40002FE04A462146FE48FDF7A9FFFC48407AFC49C8730020FC49887604F0A7FDFA49A1
:205B6000C8610020F949087004F0A0FDF749486025E001200BF060FB21E04A462146F448F9
:205B8000FDF78DFF1BE04A462146F248FDF787FF15E04A462146EF480C30FDF780FF0EE01F
:205BA0000CE04A462146ECA0FDF7B0FF28B9EC48007820F00100EA49087000E000BF00BF2C
:205BC000FEE301E0FDE300BF43F20821681A8D4278D01CDC41F20C31A5EB01008D4233D0A2
:205BE0000CDCA5F58050A0F1080018B3B0F5017F67D123E0E6E322E122E161E2A0F5E050B8
:205C0000F63840B3A0F203100028F1D14BE0B0F53E7F7DD005DCF82862D0B0F5007FE7D1EB
:205C200080E0A0F2FD30002873D0A0F2FB200028DED1D7E001200BF0FFFAFEE04A462146B5
:205C4000C848FDF72CFFF8E04A462146C5480C30FDF725FFF1E0C448007868B94A46214678
:205C6000C248FDF71CFFC1480078C043C0490870BE484078C0434870BC480078B14948735C
:205C8000BA48407888730B464FF481520C214FF4E2600DF00BFA0020B649087004F006FDA6
:205CA000B4494860C9E04A462146ABA0FDF72EFF28B9AB48007820F00200A9490870BCE0CF
:205CC00000E0B9E04A462146AB48FDF7E8FEABA345F203320C2140F213700DF0E7F9ACE082
:205CE00020222146A6480BF0BBFD20222146A548FDF7D5FEA348007B2070A2484078607095
:205D0000A0480079A0709F48C07EE070234601E02BE033E045F208420C2140F213700DF0D5
:205D2000C5F98AE0207840B29649C876084690F91B000A2801DD0A20C876924890F91B00AC
:205D400010F10A0F02DAF6208E49C87660788D49487000208C49087088A345F203320C218B
:205D600040F213700DF0A2F967E0884B41F210520C214FF4E2600DF099F95EE04A462146B1
:205D800083A0FDF7C3FE60BB002080498860C8600922814981A0FDF7B9FE80B17B480068FA
:205DA000B0F57A7F03D2002078490860486009227AA17948FDF797FE002073490870734BDD
:205DC0001022AD2178480DF0DAF86CA345F203320C2140F213700DF069F90020594908832B
:205DE00048832AE07148007828BB10227049644888380BF035FD10226D49103160487438B9
:205E00000BF02EFD0C216B48FFF7E6F880466848C0F82C8003464FF492520C214FF4E260AC
:205E20000DF044F9644B4FF4B9520C214FF4E2600DF03CF900BF00E000BF00BFC0E600BFC5
:205E4000B5F5445F60D010DCA5F58050A0F58670C8B1B0F5807F1CD0B0F57F7F20D0A0F5B3
:205E6000F050F438002867D122E0A5F548500838E8B3FD2861D0B0F5FC7F5FD0A0F2FD20F3
:205E80000028F0D1E1E04A4621464C48FDF707FE14E14A46214649480C30FDF700FE0DE13B
:205EA00000204749087004F001FC4549486005E13E48007838BB10223D49314888380BF0D0
:205EC000CFFC10223A4910312D4874380BF0C8FC0C213848FFF780F880463548C0F82C805F
:205EE00003464FF492520C214FF4E26000E071E00DF0DCF8304B4FF4B9520C214FF4E26003
:205F00000DF0D4F800BFD9E0202221461C480BF0A7FC202221461B48FDF7C1FD1948007BFB
:205F2000207018484078607016480079A0701548C07EE070234645E0BFE06FE07CE000003F
:205F400034080020B4070020B4020020A80100205C08002044080020524541445900000006
:205F6000700100206C080020C4000020C6000020C8000020980100207101002041434B0030
:205F800090FC01089C080020AD0300200C0A0020434C4541520000004C090020434C4541B1
:205FA000525F4F444F000000B4030020BE010020D4070020A40900201408002084080020E8
:205FC000A001002047F208320C2140F214700DF06DF873E0207840B2FB49C876084690F912
:205FE0001B000A2801DD0A20C876F74890F91B0010F10A0F02DAF620F349C8766078F24992
:2060000048700020F1490870AFF2900347F203420C2140F214700DF049F84FE04A462146FD
:20602000AFF2CC00FDF772FD28B9E948007820F00400E749087041E0E64B41F210520C2136
:206040004FF4E2600DF032F838E04A462146AFF2C000FDF75BFD78BB0020DE498860C8604E
:206060000922DD49AFF2CC00FDF750FD88B1D9480068B0F57A7F03D20020D649086048609D
:206080000922AFF2E801D448FDF72DFD0020CF490870D04B1022AD21D0480CF070FFAFF222
:2060A000241347F203420C2140F214700CF0FEFF0020CB490883488300BF00BF00BF7FE524
:2060C00000BF42F20550291A854270D053DCB5F5D05F6DD028DCB5F5A85F6AD015DCB5F55F
:2060E000905F67D008DCB5F5805F77D0A5F588500838002873D1B1E0B5F5985F70D0A5F59C
:20610000A05010380028F5D106E1A5F5B0501038002879D0F02878D0B0F5007F76D0A0F2C3
:20612000F1200028E6D16DE1B5F5005F6FD013DC41F61051A5EB01008D4269D006DCB5F52D
:20614000D95F76D0B5F5E05FD4D19CE1F02871D0B0F5F87FCED1C8E1B5F5045F6BD0A5F517
:2061600008501038002867D0B0F5807F74D0B0F5047FBFD1F9E140F6FB22881A91426CD0A2
:206180002FDC40F2FD52A1EB020091427DD019DC40F2FD22A1EB0200914277D00BDCB1F54A
:2061A000807F74D0A1F203210029A3D12FE2EEE145E1C3E06DE0FE286AD0A0F2FF10002829
:2061C00098D164E2FF287DD0A0F2062000287AD0F82879D0B0F5FC7F8CD1AEE22DE0FCE310
:2061E00088E0B0F5A06F70D013DCB0F5907F6DD0A0F2012000286AD0B0F5807F68D0A0F2E0
:20620000012000288ED149E3A7E0B8E0C6E07BE148E1A0F2016000287BD0A0F2011000282F
:2062200078D0A0F20310002875D0B0F5827F8BD1F1E312E148E168E170E16A4B0822C321B5
:20624000664801F01FFE674B4AF208420C2140F215700CF02BFF18E274E177E24A462146A1
:206260006048FDF71CFC5F4B0822C3215B480CF086FEAFF2F8234AF603120C214FF4E260CC
:206280000CF014FFFFF7F4FAFBE301E2D9E199E1FCE15548007860BB1022544954480BF0A3
:2062A000DFFA102251491031514814300BF0D8FA0C215048FEF790FE80464C48C0F82C8048
:2062C000034606E0F9E1FCE12EE21AE34DE25EE2CEE24FF492520C214FF4E2600CF0E6FEF3
:2062E000454B4FF4B9520C214FF4E2600CF0DEFE00BFC6E3102238493D484C300BF0B0FA75
:20630000354B4AF210620C2140F215700CF0CEFEB7E305E31DE37FE34A4621462E48FDF75E
:20632000BEFB002029490870AFF2B0334AF603120C214FF4E2600CF0B9FEA2E310222F492D
:206340002B4860300BF08CFA2C4B4AF210720C2140F215700CF0AAFE93E34A462146274820
:20636000FDF79DFB002019490870AFF2F0334AF603120C214FF4E2600CF098FE81E31022A4
:206380001F491B4874300BF06BFA1D4B4AF610020C2140F215700CF089FE72E34A462146C1
:2063A0001748FDF77CFB002008490870AFF234434AF603120C214FF4E2600CF077FE60E357
:2063C00060E360E378E300009C080020AD030020700100200C0A00204C090020B403002035
:2063E000B40700207A010020BE010020D407002008FC0108A4090020140800205C090020B2
:206400006C0900202078F949087008460078C043F7490870F548007801280FD1F5480068B1
:2064200020F48060F34908600846006820F4805008600846006820F40060086021E32022EA
:206440002146ED480BF00CFA23464AF220020C2140F215700CF02AFE13E34A462146E748B4
:20646000FDF71DFB0020E6490870E449487B0EF02DFBAFF2F8434AF603120C2140F215701E
:206480000CF014FEFDE210222146DB4848300BF0E7F923464AF210120C2140F215700CF059
:2064A00005FEEEE24A462146D648FDF7F8FA0020D3490870AFF23C534AF603120C2140F276
:2064C00015700CF0F3FDDCE2CF4B4AF230220C2140F215700CF0EAFDCC4B4AF610420C2148
:2064E00040F215700CF0E2FDCBE22022C849C24860380BF0B5F9C64B4AF220520C2140F2A1
:2065000015700CF0D3FDBCE2BBE2C24B41F201420C214FF4E2600CF0C9FDB2E24A4621466D
:20652000BD48FDF7BCFA0020B5490870AFF2B4534AF603120C214FF4E2600CF0B7FDFFF7C1
:2065400097F99EE24A462146B3481030FDF7A7FA0020AB490870AFF2DC534AF603120C2186
:206560004FF4E2600CF0A2FD8BE24A462146A848FDF795FA0020A2490870AFF200634AF65D
:2065800003120C214FF4E2600CF090FD79E24A462146A2A0FDF7BAFA98B9AFF220634AF6BA
:2065A00003120C2140F215700CF080FD00200AF043FE642003F0E0FC01200EF0B7FD04F0F4
:2065C00097F95EE24A462146AFF23C60FDF79EFAE0B9FF2304220021924800F041FB924948
:2065E0008548903800F024FD9049914800F020FDAFF278634AF603120C2140F215700CF085
:2066000055FD01200EF092FD04F072F939E24A46214688A0FDF77AFA90B90EF05BFC814812
:2066200000F090FBAFF2AC634AF603120C2140F215700CF03BFD01200EF078FD04F058F9E9
:206640001FE24A4621467E48FDF729FA7C480078C0437C4908707A484078C0434870002094
:206660007949087004F022F87749486074480078764948737248407888730B464FF48152E8
:206680000C214FF4E2600CF011FDFAE1F9E1F8E14A4621466E48FDF702FA6D4B0222DF2137
:2066A00060480CF06CFCAFF22C734AF603120C2140F215700CF0FAFCE3E1207865490870E1
:2066C000DFE100BF20790006617900EB0140A17900EB0120E179084421780906627801EB5C
:2066E0000241A27801EB0221E2781144401A00F1010820780006627800EB0240A27800EB81
:206700000220E2788118424604F10800FDF7C7F94AF60830404482B223460C2140F21570AE
:206720000CF0C4FC00BFACE14B4B41F210520C214FF4E2600CF0BAFCA3E1484B41F208620E
:206740000C214FF4E2600CF0B1FC9AE120222146294824300BF084F823464AF620520C2136
:2067600040F215700CF0A2FC8BE14A4621463C48FDF795F9002022490870AFF600034AF674
:2067800003120C2140F215700CF090FC79E12078401E00EB4002C2EB40101530C1B2631CC7
:2067A0001822204801F06EFB2078012804D0022807D003280FD109E02A48C08AA4F81700E4
:2067C00009E02948C08AA4F8170004E02748C08AA4F8170000BF00BF23464AF61A620C2142
:2067E00040F215700CF062FC4BE10000C4000020C50000206C01002090FC01089C080020AD
:20680000AD030020DC080020EC0800201C0900202C09002070010020D4070020524553453B
:2068200054000000B4030020FFFF0108FFF3010800F001085245434F5645525900000000C3
:20684000C6000020C800002098010020B4070020860300208D0100200C0A0020B001002078
:20686000BC080020F01200200A130020241300202078401E00EB4002C2EB40101230C1B2A9
:20688000631C01228E4801F0FDFA23464AF602720C2140F215700CF009FCF2E02078012803
:2068A0000AD160788749087601F118030122122183480CF064FB1AE0207802280AD16078DF
:2068C0008149087601F1180301222F217C480CF056FB0CE02078032809D160787B4908763C
:2068E00001F1180301224C2175480CF048FBAFF674134AF603120C2140F215700CF0D6FBCD
:20690000BFE023460222DF216D4801F0BBFA23464BF202020C2140F215700CF0C7FBB0E014
:206920002078012814DB3C2269496A480AF098FF2078401E664901EB80000068C4F801001E
:2069400023464BF205120C2140F215700CF0AEFB97E0207801285DDB5F4801882078401E5B
:206960005B4A22F8201061782078401E02EB800081702078012815D12078401E114601EB1B
:2069800080008078C0EBC00041022078401E32F8200091FBF0F0C1B22078401E02EB80004F
:2069A000C17024E02078401E494901EB800081782078801E464A02EB80008078081AC0EBBD
:2069C000C00041022078401E32F820202078801E3F4B33F82000101A00E051E091FBF0F0A2
:2069E000C1B22078401E1A4602EB8000C17000203A4908702078401E354901EB80000068CD
:206A0000C4F8010023464BF205120C2140F215700CF04CFB35E01EE0207801281ADB207874
:206A2000401E2B4901EB8000D4F80110016000202A4908702078401E254901EB8000006897
:206A4000C4F8010023464BF205120C2140F215700CF02CFB15E04A46214621A0FDF756F8C6
:206A600068B90EF011FA164800F028F9AFF6F4234AF603120C2140F215700CF017FB00E09A
:206A800000BF00BF19E0A5F51450053820B1A0F5F840063828B900E000BF022013490870F2
:206AA00000E000BF00BF2B463A4640F25161104800940CF047FB00E000BF00BFBDE8F883FB
:206AC000B4030020F01200200A130020241300203E130020ECFC01083A040020AD03002099
:206AE0004C4F4720434C4541520000005D000020F4040020704700BF0100A0F10100FBD1C3
:206B0000704710B50246002016E0135C041D145D63400B54031DD35C00F10804145D634038
:206B2000041D0B55231DD35C0834145D634000F108040B55431CD8B20428E6DB10BD000015
:206B40001FB54FF46040009011200190022003906946194803F00AFC4FF4E060009011202A
:206B60000190022003906946144803F0FFFB00224FF48071114803F093FD00224FF40071CF
:206B80000E4803F08DFD00224FF480610B4803F087FD00224FF40051074803F081FD00227A
:206BA0004FF48041044803F07BFD00224FF40041014803F075FD1FBD000C01400008014054
:206BC00010B500210D4805F049F804210B4805F045F80821094805F041F80021074804F08E
:206BE000DDFC0421054804F0D9FC0821034804F0D5FC0C21014805F011F810BD481500208A
:206C0000F8B50446002000906A460021204600F02FF90DF101020121204600F029F90221C0
:206C20006846FEF7C1F906466A460221204600F01FF90DF101020321204600F019F99DF848
:206C400001009DF8001000EB012085B2A81B03D12046FEF763FCF8BD2046FEF7BBFDFAE751
:206C60002DE9F04780460C4616461F46301B00F0FF09002507E06019C1B23A46404600F0BD
:206C80004DF9681CC5B24D45F5DBBDE8F08700001FB5044602200090012001900390694671
:206CA000054803F063FB01220221034803F0F8FC204605F0BDFB1FBD000C014010B5044673
:206CC0001C4B3022692120460CF059F9401C28B9184B3022692120460CF051F9164B102202
:206CE0009B2120460CF04BF9401C28B9124B10229B2120460CF043F9104B1022AD2120464B
:206D00000CF03DF9401C28B90C4B1022AD2120460CF035F90A4B1022CD2120460CF02FF91E
:206D2000401C28B9064B1022CD2120460CF027F910BD0000EC0800201C0900200C0A0020C7
:206D40001C0A002010B50446424B0C22042142480CF015F9401C28B93E4B0C2204213E48CB
:206D60000CF00DF93D4B0122122120460CF007F9401C28B9394B0122122120460CF0FFF861
:206D8000364B183B1822152120460CF0F8F8401C30B9324B183B1822152120460CF0EFF88F
:206DA0002F4B01222F2120460CF0E9F8401C28B92B4B01222F2120460CF0E1F8284B183B7C
:206DC0001822322120460CF0DAF8401C30B9244B183B1822322120460CF0D1F8214B0122A4
:206DE0004C2120460CF0CBF8401C28B91D4B01224C2120460CF0C3F81A4B183B18224F214D
:206E000020460CF0BCF8401C30B9164B183B18224F2120460CF0B3F8134B0822C3212046DA
:206E20000CF0ADF8401C28B90F4B0822C32120460CF0A5F80D4B0222DF2120460CF09FF898
:206E4000401C28B9094B0222DF2120460CF097F810BD0000B0090020B403002008130020D4
:206E6000221300203C1300207A010020860300202DE9F04106460F4615460024304605F038
:206E80004AFBA021304605F08BFB00BF00BF601C84B240F6B830844203DD4FF0FF30BDE8F4
:206EA000F081304605F0A4FA0028F0D13946304605F076FB002400BF601C84B240F6B83061
:206EC000844202DD4FF0FF30E9E7304605F090FA0028F1D1304605F01EFBA121304605F03F
:206EE0005FFB002400BF601C84B240F6B830844202DD4FF0FF30D2E7304605F079FA0028B3
:206F0000F1D12946304605F0B0FA304605F0E0FA304605F020FB0020C1E700002DE9F04151
:206F200006460F461546002400220221294803F0B7FB304605F0EFFAA021304605F030FB2B
:206F400000BF00BF601C84B240F6B830844203DD4FF0FF30BDE8F081304605F049FA0028E3
:206F6000F0D13946304605F01BFB002400BF601C84B240F6B830844202DD4FF0FF30E9E7BA
:206F8000304605F035FA0028F1D12946304605F007FB002400BF601C84B240F6B830844218
:206FA00002DD4FF0FF30D5E7304605F021FA0028F1D1304605F0CFFA0A2002F0DDFF012209
:206FC0000221044803F06CFB034803F09DFB0020C0E70000000C0140E8050020F8B50E48EE
:206FE0000468001D0568200E8DF80000200C8DF80100200A8DF80200E0B28DF80300042146
:207000006846FDF7E9FF0646701B02D1FEF7ECF901E0FEF76BFBF8BD00FC010810B504465D
:20702000207818B9FEF762FB0120207010BD000038B504460D4600200C490860084684607E
:20704000281B401C800AC86003F018F900BF34200749C86000BF6946044802F0A1FF03F011
:207060008BF8642002F088FF38BD0000D80500200020024010B590B0042269460E480AF012
:20708000EFFB0446ACB9042269460CA0FCF73EFD78B928226946084808300AF0E1FB0446D6
:2070A0003CB9282269460748FCF7F9FC002010B010BD0120FBE7000000E80108464C4147F0
:2070C000000000007C09002010B54FF4805003F03FF910BD10B5042003F03AF910BD00005F
:2070E0001FB54FF4604000900220019003906946064803F03BF94FF4E06000900220019019
:2071000003906946024803F031F91FBD000C01400008014010B50021104804F07FFD042181
:207120000E4804F07BFD08210C4804F077FD0C210A4804F073FD0021084804F019FA042128
:20714000064804F015FA0821044804F011FA0C21024804F00DFA0AF0F5F810BD48150020C7
:207160002DE9F04107460C46207860BB384600F057F846B2701C48B11448402101FB060578
:207180004022394628460BF0CDFE1AE00F49491E0F48FFF74DFFF0220C4940310C4800F06C
:2071A000A5FA0C490948FFF743FFF0220849074800F09CFA074D3F3D4022394628460BF000
:2071C000B1FE01202070BDE8F081000000F0010800EC0108FFF3010810B504460B48006886
:2071E000A0600B484068E06020220A4904F11000FCF755FC0848016821634068606307487F
:207200000168A1634068E06310BD00006C010020EC080020B4070020B0010020CA00002012
:2072200010B50246002116E00F4C04EB811003884FF6FF7083420CD111B90120108006E00D
:207240004020C0EB8110084C035B581C1080084610BD481C41B21029E6DB04480388581C25
:2072600010804FF0FF30F3E700F00108C0F301080021074AD1610749096941F00401054A96
:2072800011611146096941F0400111617047000048050020002002402DE9F047044600258D
:2072A0004FF6FF763746B046B14600F0EDF80443E6B2C4F30727C4F307484FEA14694CF217
:2072C000503000F0DBF90546002D4FD12949C86102F0BEFE0546002D48D12748006940F0F0
:2072E000100025490861FF2E09D0244800883043224908804CF2503000F0C0F905466DB96F
:20730000FF2F0BD01D48801C008838431B49891C08804CF2503000F0B1F905467DB9B8F14D
:20732000FF0F0CD01548001D008840EA08001349091D08804CF2503000F0A0F905467DB95D
:20734000B9F1FF0F0CD00D48801D008840EA09000A49891D08804CF2503000F08FF90546EA
:207360000548006920F01000034908612846BDE8F0870000480500200020024008F8FF1F0B
:207380002DE9F047044600254FF6FF763746B046B14600F079F8C0432043C443E6B2C4F3F0
:2073A0000727C4F307484FEA14694CF2503000F065F90546002D4FD12949C86102F048FE6C
:2073C0000546002D48D12748006940F0100025490861FF2E09D024480088304022490880D0
:2073E0004CF2503000F04AF905466DB9FF2F0BD01D48801C008838401B49891C08804CF252
:20740000503000F03BF905467DB9B8F1FF0F0CD01548001D008800EA08001349091D0880B6
:207420004CF2503000F02AF905467DB9B9F1FF0F0CD00D48801D008800EA09000A49891D00
:2074400008804CF2503000F019F905460548006920F01000034908612846BDE8F087000084
:20746000480500200020024008F8FF1FA5200021044AD26902F00201022901D1002000E0BE
:20748000A5207047002002400148006A704700000020024070B504460D4601264CF250309B
:2074A00000F0ECF80646A6B900200B49C8610B48006940F010000949086125804CF2503096
:2074C00000F0DCF806460548006920F0100003490861304670BD000048050020002002409F
:2074E00070B5054600244CF2503000F0C7F804465CBB00201649C8611648006940F020006B
:20750000144908610846006940F0400008614CF2503000F0B3F804460E48006920F0200083
:207520000C4908618CB90846006940F010000861094805804CF2503000F0A0F80446054835
:20754000006920F0100003490861204670BD0000480500200020024000F8FF1F70B5044606
:2075600000254CF2503000F089F80546BDB900200C49C8610C48006940F010000A4908619F
:2075800044F08800094908804CF2503000F076F805460548006920F01000034908612846F5
:2075A00070BD0000480500200020024002F8FF1F0021074AD1610749096941F00201054ACE
:2075C000116111464861096941F040011161704748050020002002400022054BDA61054A61
:2075E000126942F00102034B1A61018070470000480500200020024000201E49C96801F062
:20760000100139B11C49C96941F002011A4AD16140F010001749C96801F0040139B11649FE
:20762000C96941F00101144AD16140F004001149C96901F0010169B10F49C96941F00401C8
:207640000D4AD16100BF0B49C96921F00101094AD16100BF00BF40F20111884206D1054913
:20766000C96921F00101034AD16101E00149C86000BF7047002002404805002070B504463F
:2076800003F014F8054609E0601C38B124B103F00DF8401BA04201D9032070BD1248C0689C
:2076A00000F001000028EFD10F48C06800F0200020B100BF20200C49C86000BF0A48C068DC
:2076C00000F0100048B90848C06900F0010020B90548C06800F0040018B1FFF78DFF012091
:2076E000DBE70020D9E70000002002402DE9F04104460E461746002502F0C0FD00BF0FE0C2
:2077000056F825C0624600232146022002F05EFD08B9241D03E002F02FFDBDE8F0816D1CF3
:20772000BD4202D203488442EAD902F025FD00BFF3E70000FBFF01080220054908700020EA
:207740000449088048800449088048807047000030000020280000202C00002001200149E9
:2077600008707047300000202DE9FF4704460E4617464FF0000A0BF0F3FA03900398FDF7E0
:2077800017FE029039B2029809F0F0FB00908B4800990160B0F9000089490968C1EB802044
:2077A0008749096801EBA0208549086008460068801200B2834908808048B0F9020082491A
:2077C0000968C1EB80208049096801EBA0207E49086008460068801200B27C4908807C48CC
:2077E000007C002849D17B480078042845D17A48408840F6B831884210DA7848046078480D
:20780000006810F1040F05DA75480068001D7449086077E000207249086073E06E4840883B
:2078200040F68A41884221DA6B484088A0F6B83000EB800040F21A41081A6A490860084606
:207840000068844201DA204601E0664800686349086063480068801E614908600846006835
:2078600010F5D27F4EDA604808604BE000205B4908605D485A49086044E05748408840F6B2
:207880001C41884210DA554804605548006810F1040F05DA52480068001D5149086031E0AC
:2078A00000204F4908602DE04B48408840F6EE41884221DA48484088A0F61C4000EB800061
:2078C00040F21A41081A4749086008460068844201DA204601E043480068404908604048F7
:2078E0000068801E3E4908600846006810F5D27F08DA3D48086005E00020384908603A4848
:2079000037490860394A2F48B0F900103348008800B209F0EBFA054635480068C0EB4520F9
:207920003349096801EBE0003149086031484088B7214843C0F3CF1947F698107043B9F527
:207940007A7F02DA4FF47A7100E0494690FBF1FA274800680AEB602547F69810854200DD65
:2079600000E02846054628B223490880234A1748B0F900101A48008800B209F0B7FA80460F
:207980001F480068C0EB48201D49096801EBE0001B49086008460068401200B216494880B5
:2079A000084609F0A3FF14480068009009F0C4FF019001980AF028FFBDE8FF872800002010
:2079C0000400002018000020080000201A000020C4050020CA000020081600202000002098
:2079E0001C000020240000205CFEFFFF1406002010000020DC0800202C0000203806002097
:207A00001400002004F01AFE08F0FCFE08F09CFF62B60020124981F83C0008F0ABFE72B690
:207A200008F072FF09F096FCFFF78AF800200D4908600846006820F4005000F50050086035
:207A40000DE0084B41F204120C214FF4E2600BF02DFBC8200AF0B8FE034802F055FEF0E7C9
:207A60004C1B00206C010020E805002000B587B00220009000208DF810000948C06900F028
:207A8000020002280AD002F0F9FB02F089FB684602F00EFB02F07AFB02F06EFB07B000BDA5
:207AA0000020024070B505460E46049CAC4204DA281B7043C0F5806108E0944202DA4FF4CB
:207AC000806103E0A01A5843C0F58061002901DC002000E00846014688B270BD87B0014677
:207AE00000220868009048680190C86803903D4881423AD04FF0553008600A68B2F1553F39
:207B000002D0002007B070474FF0AA3008600A68B2F1AA3F01D00020F4E74FF0553048604E
:207B20004A68B2F1553F01D00020EBE74FF0AA3048604A68B2F1AA3F01D00020E2E745F2A9
:207B40005550C860CA6890B245F25553984201D00020D7E74AF6AA20C860CA6890B24AF696
:207B6000AA23984235D00020CCE700986FF30B0000F2555008600A68C2F30B0040F2555376
:207B8000984201D00020BDE700986FF30B0000F6AA2008600A68C2F30B0040F6AA2398423A
:207BA00001D00020AEE7039820F00700C01DC860CA6802F00700072801D00020A2E7039819
:207BC00020F00700C860CA6802F0070008B1002098E700980860019848600398C8600120BE
:207BE00090E70000001401402DE9F04104460E46154629480078012812D128480178007823
:207C0000401C264A1070264820F8116010460078322810DB002020490870114608700AE054
:207C200032221F49304609F01BF8643087B22088B84200DD00BF2888C0F3C03050BB2088F5
:207C400040F2DC51884203DC02F030FD1549086002F02CFD13490968401A42F21071884276
:207C600018D9286820F4004000F50040286001200D494880208888800846FFF7ADFA002078
:207C80000A4908700A488088401C09498880022008490870BDE8F081FF03002000040020C2
:207CA000E41400200404002024120020040300201C09002079010020B1F5967F03DA01226D
:207CC000044B1A7002E00022024B1A7001F1640202807047FE03002038B5044601234FF4A0
:207CE0007A720A210248009404F062FD38BD0000D014002030B503460024002204E033F8C0
:207D000012502C44551CAAB28A42F8DBB4FBF1F5A8B230BD70B505462A480078012811D1E4
:207D200000202849087002F0C1FCB0F5E16F05D902F0BCFCC8302449088003E04FF4FA60A1
:207D40002149088002F0B2FC1F490988884236D91E480078012832D11D48007858B11D486A
:207D60000088C82807DC40F2C270854207DD40F63E00854203DA00201749C8721CE00120AA
:207D80001549C872002415E0144830F81400A8420EDB092212A11548FBF7A5FE1448015D3D
:207DA0001248203880F8271000200849087070BD601CC4B2092CE7DB00200449087000BFBF
:207DC000F5E700000803002006030020BE010020900100208A010020C4050020887A010844
:207DE00054544B5A303139412E000000F40700209A7A010810B502460B460020002107E06F
:207E000032F81140844201DD32F811004C1CA1B29942F5DB10BD10B502460B464FF6FF70C3
:207E2000002107E032F81140844201DA32F811004C1CA1B29942F5DB10BD00000246002147
:207E400008E0064830F81100904201DC08467047481CC1B2C829F4DB0020F8E7D27A010814
:207E60000246002108E0064830F81100904201DC08467047481CC1B2BF29F4DB0020F8E7E9
:207E8000627C01082DE9F047C2B082460D4614461F4600260FE002A88219A819C1B250463E
:207EA000FEF7E6FF401C20B94FF0FF3042B0BDE8F087701CC6B2A642EDDB214602A8FDF77E
:207EC00073F881462819C1B201AA5046FEF7D0FF2819401CC1B20DF105025046FEF7C8FF50
:207EE0009DF805009DF8041000EB01201FFA80F8B8EB090006D1224602A93846FBF7CFFDD0
:207F00000020D3E74FF0FF30D0E72DE9FC5F804689464FF0000A002549464046FFF7EAFEFB
:207F20008346002407E038F81400ABEB000505FB05AA601C84B24C45F5DB5046FBF79AFFAB
:207F400006460F46304639460DF072FCCDE90001FBF7DBFF05462846BDE8FC9FF8B50446AD
:207F600000260020009000BF94F82400012801D10220F8BD012084F8240000BF2046FCF711
:207F800089F90646002E62D1A06A20F4885040F00200A062022002F0CDFC30490968B1FB15
:207FA000F0F04000009002E00098401E009000980028F9D12046FCF7D5F92068806840F058
:207FC00008002168886002F071FB054611E002F06DFB401B0A280CD9A06A20F0020040F076
:207FE0001000A06200BF002084F8240000BF0120BFE72068806800F008000028E7D120689A
:20800000806840F004002168886002F04FFB054611E002F04BFB401B0A280CD9A06A20F097
:20802000020040F01000A06200BF002084F8240000BF01209DE72068806800F0040000288D
:20804000E7D1A06A20F0020040F00100A06200BF002084F8240000BF30468AE700000020D4
:2080600038B50246002300200090906800B100BF00BF92F82400012801D1022038BD0120F0
:2080800082F8240000BF906890B94868012809D11068806B6FF315000C6840EAC4301468A7
:2080A000A06338E0906A40F020009062012332E00C694868A0421ED84C680869001BC0F145
:2080C000030000EB80041F20A04040F440141068806BA0434D680C69641BC4F1030404EBED
:2080E00084050C68AC400D8A6D1E44EA055420431468A0630FE04C680869001BC0F1030029
:2081000000EB80041F20A04040F440141068806BA0431468A0631068806800F0010040B93A
:208120001068806847F20104A043CC6920431468A060886901280FD1C869B0F5E04F06D1D4
:208140001068406840F480601468606004E0906A40F0200090620123486901280DD18869C2
:2081600030B91068406840F480501468606004E0906A40F020009062012308680A2812D3EB
:208180001068C0680C780A3C04EB44050724AC40A0430D780A3D05EB45058C68AC402043FA
:2081A0001468E0600FE0106800690C7804EB44050724AC40A0430D7805EB45058C68AC40DE
:2081C0002043146820610868102802D00868112805D11068806840F400001468A060486886
:2081E000012806D002280DD0032814D004281BD11BE0106840696FF30B00CC6820431468B6
:2082000060611BE0106880696FF30B00CC6820431468A06112E01068C0696FF30B00CC688C
:2082200020431468E06109E000BF1068006A6FF30B00CC6820431468206200BF00BF0868A4
:20824000102802D00868112827D1174C1068A0421ED11068806800F40000F0B9106880686A
:2082600040F400001468A0600868102815D10F4800680F4CB0FBF4F000EB800040000090DC
:2082800002E00098401E009000980028F9D104E0906A40F020009062012300BF002082F84F
:2082A000240000BF1846E9E6002401400000002040420F0010B504460121204600F044F8D5
:2082C0004FF6FF7101EA00101A4948800221204600F03AF84FF6FF7101EA00101549888002
:2082E0000321204600F030F84FF6FF7101EA001010490880104800880988401A00B20F4976
:2083000008800D4840880B494988401A00B20B4948800948808807498988401A00B2074955
:2083200088800749054808F069FE01200549087010BD000014040020260400202C040020B3
:2083400032040020200400200246002001290FD0022909D0032904D0042908D11368986C89
:2083600009E01368586C06E01368186C03E000BF1368D86B00BF00BF7047000070B50446EC
:20838000002500BF94F82400012801D1022070BD012084F8240000BF2046FBF7E3FF0546FA
:2083A000002D5BD1A06A42F20101884340F48050A0622E492068884208D12D48006800F4E0
:2083C000702008B9012002E0002000E0012020B1A06A20F48010A06203E0A06A40F48010F6
:2083E000A062A06A00F4807008B90020E06200BF002084F8240000BF401F21680860206854
:20840000406840F08000216848602068406800F4806010BB2068806800F4E040B0F5E04FAC
:2084200015D112492068884208D11148006800F4702008B9012002E0002000E0012030B1C5
:208440002068806840F40210216888600BE02068806840F400402168886004E000BF0020F2
:2084600084F8240000BF284691E70000002801400424014038B5024600230020009000BF1E
:2084800092F82400012801D1022038BD012082F8240000BF4868072812D21068406B0C7933
:2084A000641E04EB84051F24AC40A0430D796D1E05EB85050C68AC4020431468606327E01C
:2084C00048680D2812D21068006B0C79E41F04EB84051F24AC40A0430D79ED1F05EB8505D2
:2084E0000C68AC4020431468206311E01068C06A0C790D3C04EB84051F24AC40A0430D7949
:208500000D3D05EB85050C68AC4020431468E06208680A2812D31068C0680C780A3C04EB36
:2085200044050724AC40A0430D780A3D05EB45058C68AC4020431468E0600FE01068006923
:208540000C7804EB44050724AC40A0430D7805EB45058C68AC4020431468206108681028BE
:2085600002D00868112827D1174C1068A0421ED11068806800F40000F0B91068806840F44B
:2085800000001468A0600868102815D10F4800680F4CB0FBF4F000EB80004000009002E00B
:2085A0000098401E009000980028F9D104E0906A40F020009062012300BF002082F82400EA
:2085C00000BF184661E70000002401400000002040420F002DE9F0478046FD480068401C04
:2085E000FB49086008460068B0F5967F01D900200860F8480078012805D14120F6494875E9
:208600008875C8759EE0F548C07A012808D1F4480078012804D10020F149087007F052FF5D
:20862000F0480088F04909680844EF490860ED488088EE4909680844EC490860E948408A1B
:20864000EB4909680844EA490860EA480088401CE84908800846008840F6B831884271DBB4
:20866000DE48C07A012825D1DF480068B0FBF1F01FFA80F94846FFF7F3FBD7494875DB485C
:20868000006840F6B831B0FBF1F01FFA80F94846FFF7E6FBD0498875D548006840F6B83116
:2086A000B0FBF1F01FFA80F94846FFF7D9FBCA49C8753EE0CC48006840F6B831B0FBF1F0AF
:2086C0001FFA80F94846FFF7B9FBC3494875C748006840F6B831B0FBF1F01FFA80F94846C5
:2086E000FFF7ACFBBC498875C348007801280ED10846407DC1490870BD48006840F6B83137
:20870000B0FBF1F0BE4908800020BB490870B848006840F6B831B0FBF1F0B9490988081ADA
:2087200000EB40008001B549097801EBA020AA49C8750020AF490880AB490860AB490860DA
:20874000AB490860A7484088AE490968C1EB8020AC49096801EB6020AA490860084600686F
:20876000801244F2CE714843C0F38F209A49C8800846C1880089C01101EBC0009649C88016
:20878000A148007803280BD10846C088A0F5F850A43840F27A514843C0F38F208E49C88019
:2087A0008E48C07A012809D18E48C08897490988401A49F619214843851208E08948C08821
:2087C00092490988401A4CF250314843C512002D01DC002005E04CF25030854200DB00E063
:2087E000284605468A480068C0EB85208849096801EB60208649086008460068C0F38F2039
:20880000754908818348007807287DD2DFE800F0045592DFCDDEDD00724800897E49C98AEA
:20882000401A642148437C49097E90FBF1F004B2002C01DC002000E0204604461C2094FBDC
:20884000F0F0654908772546664840897349C98A401A642148437149097E90FBF1F004B24D
:20886000002C01DC002000E0204604461C2094FBF0F05949487725445A4880896849C98A1B
:20888000401A642148436649097E90FBF1F004B2002C01DC002000E0204604461C2094FB92
:2088A000F0F04D4988772544002D01DC002002E0032095FBF0F005462CE14A4840895749E8
:2088C000C98A401A642148435449097E90FBF1F004B2002C01DC002000E0204604461C20A0
:2088E00094FBF0F03C49487725463E4880894C49C98A401A642148434949097E90FBF1F0F4
:2089000004B2002C03DC00E002E1002000E0204604461C2094FBF0F02F4988772819054675
:20892000002D01DC002103E0284600EBD07149100D46EFE02B4800893749C98A401A642166
:2089400048433549097E90FBF1F004B2002C01DC002000E0204604461C2094FBF0F01E499A
:20896000087725461F4880892D49C98A401A642148432B49097E90FBF1F004B2002C01DC44
:20898000002000E0204604461C2094FBF0F01249887728190546002D01DC002103E028461A
:2089A00000EBD07149100D46B4E00E4800891A49C98A401A642148431749097E90FBF1F0F9
:2089C00004B2002C2EDC00202DE088E06EE054E03C040020BE010020B4070020C405002091
:2089E0006804002008160020500400204C04002054040020480400205804002059040020EC
:208A00005A04002040040020B8010020380400204404002084030020F01200200A130020D1
:208A200024130020204604461C2094FBF0F0824908772546814840898149C98A401A642141
:208A400048437F49097E90FBF1F004B2002C01DC002000E0204604461C2094FBF0F07649F7
:208A6000487728190546002D01DC002103E0284600EBD07149100D464CE0704880897149B0
:208A8000C98A401A642148436E49097E90FBF1F004B2002C01DC002000E0204604461C20C4
:208AA00094FBF0F064498877254633E0634840896349C98A401A642148436149097E90FB84
:208AC000F1F004B2002C01DC002000E0204604461C2094FBF0F05849487725461AE0574837
:208AE00000895949C98A401A642148435649097E90FBF1F004B2002C01DC002000E02046D7
:208B000004461C2094FBF0F04B490877254601E0002500BF00BF4D480068C0EB85204B497D
:208B2000096801EBA0204949086008460068C0F38F2047490880002600BF07E0454830F86D
:208B40002600A84200DB03E0701CC6B20F2EF5DB00BF3EB93F4800EB8600C0786843C011D4
:208B600007B226E00E2E14DC701E3A4931F82000281A01EB8601C9784843C111701E354A50
:208B800002EB80008078C0EBC00001EB800007B20FE03048008F281A2E4991F83B104843D2
:208BA000C1112C4890F83A00C0EBC00001EB800007B2002F01DD384600E0002007462649D6
:208BC0000F8026480078D8B91C48008A24490988451A002D01DC002000E028460546214818
:208BE0000068C0EB85201F49096801EB20201D49086008460068C0F38F201749488002E0C8
:208C00000020154948800D48C08917490968C1EB80201549096801EB602013490860084606
:208C20000068C0F38F20114908800449488808F0C5FABDE8F0870000B4070020081600207F
:208C40000A13002024130020F0120020600400203A0400203E13002022040020FE030020A4
:208C6000FC0300205C04002064040020BC0100207047704710B504462068406800F0200033
:208C800020282FD12068006800F00200022829D1A06A00F0100018B9A06A40F40070A062FB
:208CA0002068806800F46020B0F5602F13D1E06888B92068406820F0200021684860A06A94
:208CC00020F48070A062A06A00F4805018B9A06A40F00100A0622046FFF77CFC6FF012006D
:208CE000216808602068406800F0800080283BD12068006800F00400042835D1A06A00F01F
:208D0000100018B9A06A40F40050A0622068806800F4E040B0F5E04F0DD02068406800F489
:208D20008060D0B92068806800F46020B0F5602F13D1E06888B92068406820F080002168FC
:208D40004860A06A20F48050A062A06A00F4807018B9A06A40F00100A0622046FFF7AAFA7F
:208D60006FF00C00216808602068406800F0400040280FD12068006800F0010050B1A06A03
:208D800040F48030A062204600F0A8F86FF001002168086010BD00002DE9F0410446002721
:208DA00000250026A84614B90120BDE8F081A06810B1606900B100BFA06A30B90020E0621F
:208DC00084F82400204600F08BF82046FBF762FA0746A06A00F01000002873D1002F71D132
:208DE000A06A20F4885040F00200A062E16960680843E16840EA41000643A068B0F5807F43
:208E000002D0A068012802D14FF4807000E0002005436069012811D1E06838B9A069401E8D
:208E20004FF4006141EA4030054307E0A06A40F02000A062E06A40F00100E062206840687B
:208E400020F469402843216848602068806821490840304321688860A068B0F5807F02D035
:208E6000A068012802D14FF4807000E00020B0F5807F03D1208A401E4FEA00582068C06AF8
:208E800020F4700040EA08002168C8622068806811490840B04208D10020E062A06A20F010
:208EA000020040F00100A06211E0A06A20F0020040F01000A062E06A40F00100E062012749
:208EC00005E0FFE7A06A40F01000A062012738466BE70000FDF7E1FFFE0E1FFF70470000CE
:208EE00010B586B004463249206888423CD100BF3048806940F400702E49886108468069F8
:208F000000F40070019000BF00BF3F2002900320039002A9284801F029FAB0200290032083
:208F2000039002A9254801F021FA254825490860002048600021234881608021C1604900F7
:208F4000016189004161202181610021C16100F08DFF20B140F22D111BA00CF00FF800BFE4
:208F600018482062446221E01C49206888421DD100BF1048806940F480600E498861084621
:208F8000806900F48060019000BF00BF0E2002900320039002A9094801F0E8F90122114647
:208FA000122001F052FC122001F042FC06B010BD002401400010024000100140000801400B
:208FC00008000240941600202E2E5C436F72655C5372635C6164632E63000000002801403A
:208FE00070B50446002500BF94F82400012801D1022070BD012084F8240000BF2046FBF74C
:20900000B1F90546002D77D1A06A40F20121884340F48070A0623C492068884208D13B4864
:20902000006800F4702008B9012002E0002000E0012078B1A06A20F48010A0622068406856
:2090400000F4806000B3A06A20F4005040F48050A06219E0A06A40F48010A0622B49091FB0
:209060002068884203D028492068884204D12748006800F4806000E0002028B1A06A20F491
:20908000005040F48050A062A06A00F4805020B1E06A20F00600E06201E00020E06200BF37
:2090A000002084F8240000BFC01E216808602068806800F46020B0F5602F16D11249206880
:2090C000884208D11148006800F4702008B9012002E0002000E0012038B12068806840F436
:2090E000A000216888600CE006E02068806840F480102168886004E000BF002084F8240085
:2091000000BF284675E7000000280140042401402DE9F04104460D46164600275749206865
:20912000884203D056492068884205D15348001D006800F4702000E0002000287ED100BFF1
:2091400094F82400012802D10220BDE8F081012084F8240000BF2046FBF704F90746002FDA
:209160006DD1A06A40F60161884340F48070A06243492068884209D14048001D006800F465
:20918000702008B9012002E0002000E0012078B1A06A20F48010A0622068406800F480607D
:2091A00000B3A06A20F4005040F48050A06219E0A06A40F48010A06230492068884203D021
:2091C0002F492068884205D12C48001D006800F4806000E0002028B1A06A20F4005040F4A7
:2091E0008050A062A06A00F4805020B1E06A20F00600E06201E00020E06200BF002084F8BE
:20920000240000BF1F48216A88621F48216AC8621E48216A08636FF002002168086020683D
:20922000806840F4807021688860226802F14C0133462A46206A00F051FE01E01AE014E066
:209240002068806800F46020B0F5602F06D12068806840F4A000216888600CE0206880680E
:2092600040F480102168886005E000BF002084F8240000E00127384667E70000002401401C
:2092800000280140E7420008574300083943000830B5024600230C7D012000FA04F31068AB
:2092A000D0F8000220F47C5001254C6A45EA042420431468C4F800021068D0F81C029843FB
:2092C0001468C4F81C02C869E8B91068D0F80C0298431468C4F80C02888880B28C8940EA76
:2092E0000444106800F510704D6940F83540088880B20C8940EA0444106800F510704D696A
:2093000000EBC5004460C86901281DD11068D0F80C0218431468C4F80C02888880B20C88EC
:2093200040EA0444106800F510704D6940F83540888980B20C8940EA0444106800F5107034
:209340004D6900EBC5004460886938B91068D0F8040298431468C4F8040206E01068D0F89C
:20936000040218431468C4F80402086938B91068D0F8140298431468C4F8140206E010680F
:20938000D0F8140218431468C4F81402086A012806D11068D0F81C0218431468C4F81C02C5
:2093A0001068D0F8000220F001001468C4F80002002030BD0168496941F0020102685161A8
:2093C000704700002DE9F0410446002500260027A8462068C068C0F3001520684069C0F389
:2093E000C0062DB126B148F4007810202168C86020680069C0F3001520684069C0F380162A
:209400002DB126B148F480681020216808612068406900F0010000283BD0206880687A49C9
:209420000840884201D1012000E0002005462068806876490840884201D1012000E00020A8
:2094400006462068806872490840884201D1012000E0002007460DB906B9D7B120688068C6
:20946000C0F3400520688068C0F340262068806800F001070DB906B91FB12046FBF734FD25
:2094800001E048F400682068806862490843216888602068C06800F0030520684069C0F3E4
:2094A000400625B11EB100212046FBF7CFFA2068006900F0030520684069C0F3001625B1C6
:2094C0001EB101212046FBF7C1FA206C40EA080020642068806900F0010520684069C0F3FB
:2094E000002620684069C0F3C0372DB126B11FB1206C40F00100206420688069C0F340053C
:2095000020684069C0F3402620684069C0F3C0372DB126B11FB1206C40F0020020642068D7
:209520008069C0F3800520684069C0F3802620684069C0F3C0372DB126B11FB1206C40F064
:20954000040020642068806900F0700008B9012000E00020054620684069C0F3C026206833
:209560004069C0F3C03795BB8EB387B32068806900F07005402D1BD006DC102D09D0202D5A
:209580000CD0302D24D10EE0502D16D0602D1FD118E0206C40F0080020641AE0206C40F0D9
:2095A0001000206415E0206C40F02000206410E0206C40F0400020640BE0206C40F080002B
:2095C000206406E0206C40F48070206401E007E000BF00BF2068806920F070002168886144
:2095E000206C78B1042021684860012084F83C002068406948F65B718843216848612046EA
:20960000FFF7D8FEBDE8F081010000040001000800000110090501002DE9F0410446002782
:209620000026002514B90120BDE8F08194F83C0028B9002084F83D00204600F0A5F8022044
:2096400084F83C002068006820F00200216808602068006840F001002168086001F026F83E
:2096600006460EE001F022F8801B0A2809D9032084F83C0000BF002084F83D0000BF0320A1
:20968000D2E72068406800F001000028EAD02068406800F00100002867D0A069012802D189
:2096A00045F0800501E025F08005E069012802D145F0400501E025F04005206A012802D1F5
:2096C00045F0200501E025F02005606A012802D145F0100501E025F01005A06A012802D1F4
:2096E00045F0080501E025F00805E06A012802D145F0040501E025F004052068006820F0A2
:20970000FC00284321680860D4E90201084321690843616908436168491E08432168C861CF
:209720002068006820F001002168086000F0BEFF06460EE000F0BAFF801B0A2809D90320D5
:2097400084F83C0000BF002084F83D0000BF03206AE72068406800F001000028EAD12068FA
:20976000406800F0010000B90127012F06D100202064012084F83C00002055E7042084F8EF
:209780003C00012050E7000010B586B0044624492068884242D100BF2248C06940F000702C
:2097A0002049C8610846C06900F00070019000BF00BF8815029000200390049002A91A48AE
:2097C00000F0D4FD4FF400700290022003900320059002A9144800F0C9FD00BF134948688E
:2097E00020F4C04040F0E06040F48040486000BF01221146142001F028F8142001F018F896
:209800000B4820630B486063FBF7D2F80A480068406940F0020008490968486106B010BD1D
:209820000064004000100240000C014000000140101700202C1700204C1B002010B5044664
:20984000606B806810B9606B006940B92E480068406940F002002C490968486110BD606B7F
:20986000006840F23172811A904214D009DCA0F2516080B3CF2818D0D02817D0DF2837D132
:2098800008E00F291CD010291BD01F2924D020292ED122E000BF606B00881C490880606B48
:2098A000017C1A48FBF78EFA23E000BF606B008817490880606B017C1548FBF783FA18E046
:2098C00000BF606B008813490880606B017C1148FBF778FA0DE001E000BF00BF606B0088EE
:2098E0000D490880606B017C0B48FBF76BFA00E000BF00BF04480068406940F00200024960
:209900000968486100BFA9E74C1B002094040020A8040020BC040020D00400202DE9F041B8
:2099200004460E46042500272068806800F08060B0F1806F0DD02068806800F00060B0F12B
:20994000006F06D02068806800F08050B0F1805F7ED100BF94F83D00012802D10220BDE878
:20996000F081012084F83D0000BF94F83C00222804D0322806D062280CD107E0422084F89B
:209980003C000BE0522084F83C0007E0722084F83C0003E0122084F83C0000BF00BF206872
:2099A000806800F0806008B1002507E02068806800F0006008B1012500E00225206800F507
:2099C000C07000EB0510006800F00101206800F5C07000EB05100160206B806898B92068A3
:2099E00000F5C07000EB05100068216BC968226B128841EA42510843216801F5C07101EB51
:209A00000511086015E0206800F5C07000EB05100068216B8968226B526841EAC201226B7F
:209A2000D26811430143206800F5C07000EB05100160206B007C00F00F00216B08612068C3
:209A400000F5C07000EB0510406820F00F0100E0B1E0206800F5C07000EB051041602068D2
:209A600000F5C07000EB05104068216B09690843216801F5C07101EB05114860206BC07DAE
:209A80000106206B807D41EA0041206B407D41EA0020216B097D0843216801F5C07101EB3F
:209AA00005118860206BC07E0106206B807E41EA0041206B407E41EA0021206B007E014301
:209AC000206800F5C07000EB0510C160206800F5C07000EB0510006840F00101206800F5F4
:209AE000C07000EB0510016000F0E0FD074620E0701CF0B126B100F0D9FDC01BB04218D933
:209B0000032084F83C001DB980202168886009E0012D03D1E8032168886003E04FF4000016
:209B20002168886000BF002084F83D0000BF032015E74DB92068806821490840884201D17A
:209B4000012016E0002014E0012D09D1206880681C490840884201D101200AE0002008E006
:209B60002068806818490840884201D1012000E000200028BCD094F83C00422804D05228DB
:209B800006D072280CD107E0222084F83C000BE0322084F83C0007E0622084F83C0003E09E
:209BA000012084F83C0000BF00BF00BF002084F83D0000BFD3E6042084F83C000120CEE68D
:209BC000010000040001000800000110704710B504460CB9012010BD607920B9002020718A
:209BE000204600F005F8012060710020F3E7000008B5094A016891420DD100BF074949693B
:209C000041F04001054A51611146496901F04001009100BF00BF08BD0030024000100240FE
:209C200070B50446002594F82100022803D00420A063012548E02068006820F00E002168DA
:209C400008602068006820F00100216808601F492068884201D1012026E01C4914312068C5
:209C6000884201D110201FE0184928312068884201D1801518E015493C312068884201D1BF
:209C8000801411E0114950312068884202D14FF4803009E00D4964312068884202D14FF410
:209CA000801001E04FF08070084908394860012084F8210000BF002084F8200000BF606B07
:209CC00010B12046616B8847284670BD0800024070B50446E06B05682068066894F84010E4
:209CE000042088402840002846D006F00400002842D02068006800F0200028B920680068CD
:209D000020F004002168086057492068884201D1042027E0544914312068884201D14020E9
:209D200020E0514928312068884201D1001519E04D493C312068884202D14FF4804011E0E2
:209D4000494950312068884202D14FF4802009E0454964312068884202D14FF4800001E013
:209D60004FF08060404908394860E06A00287AD02046E16A884776E094F8401002208840FA
:209D80002840A0B306F0020088B32068006800F0200040B92068006820F00A0021680860E1
:209DA000012084F8210030492068884201D1022028E02D4914312068884201D1202021E0FE
:209DC000294928312068884201D140151AE026493C312068884202D14FF4005012E0224954
:209DE00050312068884203D14FF400300AE017E01D4964312068884202D14FF4001001E014
:209E00004FF0007018490839486000BF002084F8200000BFA06A30B32046A16A884722E0E0
:209E200094F84010082088402840E0B106F00800C8B12068006820F00E002168086094F85B
:209E4000401001208840E16B48600120A06384F8210000BF002084F8200000BF206B10B18E
:209E60002046216B884770BD080002400146002209B901207047184B0868C01A1423B0FB18
:209E8000F3F08000086414480838C863022081F821000868026843F6F0708243D1E901037A
:209EA0001843CB6818430B6918434B6918438B691843CB69184302430868026000208862DC
:209EC000C862086348638863012081F82100002081F8200000BFCDE7080002402DE9F041DF
:209EE00004460D4616461F464FF0000800BF94F82000012802D10220BDE8F081012084F881
:209F0000200000BF94F8210001282CD1022084F821000020A0632068006820F00100216823
:209F200008603B46324629462046FBF7B7FDE06A30B12068006840F00E00216808600BE010
:209F40002068006820F00400216808602068006840F00A00216808602068006840F00100D0
:209F60002168086006E000BF002084F8200000BF4FF002084046BFE770B5044600F096FB6B
:209F800006462546681C10B104480078054400BF00F08CFB801BA842FAD370BD580000208B
:209FA0002DE9F04104460E460127002500BF2648007E012802D10220BDE8F0810120224904
:209FC000087600BF2068022813D14CF25030FDF755FB90BB0120FDF74BF94CF25030FDF756
:209FE0004DFB07461948006920F004001749086123E04CF25030FDF741FBF0B94FF0FF301D
:20A000003060A56812E02846FDF7D2FA4CF25030FDF734FB07460D48006920F002000B4931
:20A0200008610FB1356007E005F58065D4E9021001EB8020A842E6D800BF00BF00200249B0
:20A04000087600BF3846B7E7480500200020024070B5A5250124FDF709FAC5B24CF2503098
:20A06000FDF70CFB0446ECB900200F49C8610F48006940F020000D4908610846006940F09F
:20A08000400008614CF25030FDF7F8FA04460748006920F02000054908611CB92846FDF753
:20A0A0001FFA0446204670BD480500200020024070B50446012500BF2E48007E012801D198
:20A0C000022070BD01202B49087600BF207800F0010098B16068012804D1A068FDF750F982
:20A0E000054603E0A068FDF7D7F8054635B100BF00202049087600BF2846E2E7207800F0F2
:20A10000020002280BD1207CFDF7EAF9054635B100BF00201749087600BF2846D1E7207859
:20A1200000F0040004280BD1607CFDF717FA054635B100BF00200F49087600BF2846C0E788
:20A14000207800F0080008280CD1217E6069FDF7A1F9054635B100BF00200649087600BFD0
:20A160002846AEE700BF00200249087600BF2846A7E70000480500200348006940F08000A8
:20A180000149086100207047002002400348006920F40070014908610020704700200240AF
:20A1A0000748006900F4007028B90648044988600548886001E0012070470020FCE700002E
:20A1C0000020024023016745AB89EFCD2DE9FE4F05468B46174698460126002400200290A6
:20A1E00000BF2448007E012802D10220BDE8FE8F01202049087600BF4CF25030FDF73EFAB5
:20A20000064686BB012D02D10120029006E0022D02D10220029001E00420029000241EE0A8
:20A220002201B946C24648465146F9F728FC80B20190022000FB04B000900199FDF7CCF944
:20A240004CF25030FDF71AFA06460B48006920F001000949086106B104E0601CC4B202983D
:20A260008442DDDB00BF00BF00200249087600BF3046BBE7480500200020024000200849E2
:20A28000096901F0800151B10649054A5160064951601146096901F0800101B101207047C4
:20A2A0000020024023016745AB89EFCD10B50446042C3BD100202149C8700846807840B930
:20A2C00000F0F4F91D494860601F88600120887011E000F0EBF919494968401A1749886099
:20A2E000084680684B2802D215480068886000F0DDF91249486011488068114908600F4811
:20A3000080684B2818D30F480068401C0D4908600D48007E08B9012001E00B48007E094965
:20A320000968B1FBF0F00549C86005E0B4F5805F02D101200549087010BD0000580300203B
:20A34000900400208C0400209C0800207802002010B5044604480068204020B10248046099
:20A360002046FFF7A3FF10BD140401402DE9F84703460024002000258446002700226EE150
:20A380004FF0010808FA02F4D1F8008008EA0400A0427DD1DFF8D0A2D1F80480A8EB0A09D2
:20A3A000D0453AD014DCB8F1030F50D009DCB8F1000F31D0B8F1010F1CD0B8F1020F49D19C
:20A3C00020E0B8F1110F18D0B8F1120F42D11EE0B9F5881F25D006DCB9F5803F20D0B9F5BA
:20A3E000801F37D11AE0B9F5001F18D0B9F5041F30D117E0D1F80CC02DE0D1F80C8008F14E
:20A40000040C28E0D1F80C8008F1080C23E0D1F80C8008F10C0C1EE000BF00BF00BF00BF5F
:20A4200000BF00BFD1F80880B8F1000F02D14FF0040C0BE0D1F80880B8F1010F03D14FF06B
:20A44000080C1C6102E04FF0080C5C6103E04FF0000C00E000BF00BFFF2801D8984601E02E
:20A4600003F104084646FF2802D84FEA820803E0A2F108084FEA88084746D6F800804FF023
:20A480000F0909FA07F928EA09080CFA07F900E088E048EA0908C6F80080D1F8048008F06A
:20A4A0008058B8F1805F7DD100BFDFF8C081D8F8188048F00108DFF8B491C9F81880C846EB
:20A4C000D8F8188008F00108CDF8008000BF00BF4FEAB9384FEA920958F829504FEA827856
:20A4E0004FEA18794FF00F0808FA09F825EA0805DFF87C81434502D14FF0000816E0DFF8DA
:20A500007481434502D14FF001080FE0DFF86881434502D14FF0020808E0DFF86081434528
:20A5200002D14FF0030801E04FF004084FEA82794FEA197908FA09F848EA0505DFF84081FC
:20A540004FEA920948F82950D1F8048008F48038B8F5803F0AD1DFF82C81D8F8008048EA20
:20A560000008DFF82091C9F8008009E0DFF81481D8F8008028EA0008DFF80891C9F800809A
:20A58000D1F8048008F40038B8F5003F10D1DFF8F48008F10408D8F8008048EA0008DFF8BC
:20A5A000E49000E05AE009F10409C9F800800DE0DFF8D08008F10408D8F8008028EA000842
:20A5C000DFF8C09009F10409C9F80080D1F8048008F48018B8F5801F0ED1DFF8A88008F108
:20A5E0000808D8F8008048EA0008DFF8989009F10809C9F800800DE0DFF8888008F10808A1
:20A60000D8F8008028EA0008DFF8789009F10809C9F80080D1F8048008F40018B8F5001F78
:20A620000ED1DFF8608008F10C08D8F8008048EA0008DFF8509009F10C09C9F800800DE0F9
:20A64000DFF8408008F10C08D8F8008028EA0008DFF8309009F10C09C9F80080521C102A5D
:20A66000FFF48EAEBDE8F887000011100010024000080140000C01400010014000140140D8
:20A680000800014000040140024693680B400BB1012000E000207047C2684A40C26070477D
:20A6A0000AB1016101E00B040361704701480068704700005000002070B504460CB9012045
:20A6C00070BD4CF6CC402168086045F2555021680860D4E9001048602168A0688860FFF75D
:20A6E000E5FF054606E0FFF7E1FF401B302801D90320E5E72068C0680028F4D14AF6AA204C
:20A70000216808600020DBE701464AF6AA200A6810600020704700000348006803490978DC
:20A720000844014908607047500000205800002010B50848006840F01000064908600320E5
:20A7400000F0C2F8002000F007F800F02BF8002010BD00000020024070B504460E480078A1
:20A760004FF47A71B1FBF0F00C490968B1FBF0F5284600F06DFE08B1012070BD102C07D2E3
:20A7800000222146501E00F060F80548046001E00120F2E70020F0E758000020000000205F
:20A7A0005400002008B500BF1F48806940F001001D4988610846806900F00100009000BF62
:20A7C00000BF032000F080F8002211466FF00B0000F03BF8002211466FF00A0000F035F82A
:20A7E000002211466FF0090000F02FF800221146501F00F02AF800221146101F00F025F8B2
:20A8000000221146901E00F020F800221146501E00F01BF800BF0549486820F0E06040F0E2
:20A820000070486000BF08BD001002400000014000BF00F01F02012191404209920002F156
:20A84000E022C2F8001100BF70472DE9F05F80460D461646002706F01FFA074639462A4669
:20A86000334601F00700C0F1070ABAF1040F02D94FF0040A01E0C0F1070AD14600F1040A06
:20A88000BAF1070F02D24FF0000A01E0A0F1030AD4464FF0010A0AFA09FAAAF1010A0AEA56
:20A8A000020A0AFA0CFA4FF0010B0BFA0CFBABF1010B0BEA030B4AEA0B042146404606F05A
:20A8C000F3F9BDE8F09F000000BF00F00702064B19684FF6FF031940044B0B4343EA022141
:20A8E000014B196000BF70470CED00E00000FA0500BF00BF00BF00BF00BFBFF34F8F00BF3B
:20A9000000BF00BF0948006800F4E06008490843001D0649086000BF00BF00BFBFF34F8F8F
:20A9200000BF00BF00BF00BF00BFFDE70CED00E00000FA052DE9F04385B006463DA30FCB1C
:20A9400001AC0FC43FA0006800904FF00008002500270024A146012E30D0022E58D0102E3D
:20A9600061D139484468006800F0807000B301A8C4F38341475C04F4803070B132484068CB
:20A98000C0F340401DF8008004F4803040B12F48B0FBF8F000FB07F502E02D4807FB00F507
:20A9A0002948406800F48000B0F5800F01D1A94603E068000321B0FBF1F935E02248046A24
:20A9C00004F44070B0F5807F05D104F0020010B14FF400491BE004F44070B0F5007F07D173
:20A9E0001948406A00F0020010B149F640490EE004F44070B0F5407F07D11348006800F448
:20AA0000003010B14FF2244901E04FF000090BE000F0A0F90C494968C1F38131491C4900E0
:20AA2000B0FBF1F900E000BF00BF484605B0BDE8F083000002030405060708090A0B0C0D6E
:20AA40000E0F1010010200000010024000127A0000093D00F8B5044600260025207800F0C8
:20AA6000010000286BD000274348C06900F0805070B900BF4048C06940F080503E49C8618E
:20AA80000846C06900F08050009000BF00BF01273A48006800F48070B0B93848006840F4F6
:20AAA000807036490860FFF701FE064606E0FFF7FDFD801B642801D90320F8BD2F480068F0
:20AAC00000F480700028F2D02B48006A00F440752DB3A08800F44070A84220D02648006AC4
:20AAE00020F44075012026490860002008602248056205F0010090B1FFF7D8FD064608E006
:20AB0000FFF7D4FD801B41F28831884201D90320D3E71948006A00F002000028F0D0164863
:20AB2000006A20F440706168084313490862012F04D10846C06920F08050C86100BF207831
:20AB400000F00200022807D10B48406820F44040A168084308494860207800F01000102855
:20AB600007D10548406820F48000E1680843024948600020A1E70000001002400070004043
:20AB80004004424270B504460D4600266248006800F00700A8420ED25F48006820F007000C
:20ABA00028435D4908600846006800F00700A84201D0012070BD207800F00200022807D1DA
:20ABC0005648406820F0F000A168084353494860207800F0010000285DD06068012806D1F1
:20ABE0004E48006800F4003090B90120E2E76068022806D14948006800F0007040B90120C4
:20AC0000D8E74648006800F0020008B90120D1E74248406820F00300616808433F4948606A
:20AC2000FFF744FD06466068012810D108E0FFF73DFD801B41F28831884201D90320B9E7B9
:20AC40003648406800F00C000428F0D123E06068022810D108E0FFF729FD801B41F2883184
:20AC6000884201D90320A5E72C48406800F00C000828F0D10FE008E0FFF718FD801B41F2C8
:20AC80008831884201D9032094E72448406800F00C000028F0D12048006800F00700A8420F
:20ACA0000ED91D48006820F0070028431A4908600846006800F00700A84201D0012079E7AA
:20ACC000207800F00400042807D11448406820F4E060E168084311494860207800F0080066
:20ACE000082808D10D48406820F46050216940EAC1000A49486000F03DF808494968C1F33F
:20AD00000311074A515CC840064908600020FFF723FD00204EE70000002002400010024023
:20AD2000E05801080000002001480068704700000000002000B5FFF7F7FF04494968C1F3D7
:20AD40000221034A515CC84000BD000000100240F058010800B5FFF7E7FF04494968C1F32B
:20AD6000C221034A515CC84000BD000000100240F0580108F0B585B00FF26C0C9CE8E010C7
:20AD800001A8A0E8E0101CA52D68009500210022002300240020194D696801F00C05F5B11E
:20ADA000042D02D0082D19D101E0154819E001ADC1F38346AC5D01F4803555B10F4D6D6825
:20ADC000C5F340451DF805200D4D6543B5FBF2F302E00C4D04FB05F3184602E000BF0848E4
:20ADE00000BF00BF05B0F0BD02030405060708090A0B0C0D0E0F1010010200000010024087
:20AE000000127A0000093D00F8B504460025207800F00100002878D0F848406800F00C0067
:20AE200004280CD0F548406800F00C00082811D1F248406800F48030B0F5803F0AD1EF481B
:20AE4000006800F4003000285FD0606800285CD10120F8BD00BF6068B0F5803F06D1E7482B
:20AE6000006840F48030E549086028E0606858B9E248006820F48030E04908600846006872
:20AE800020F4802008601AE06068B0F5A02F0BD1DA48006840F48020D849086008460068E7
:20AEA00040F4803008600AE0D448006820F48030D24908600846006820F48020086000BF00
:20AEC000606888B1FFF7F2FB054606E0FFF7EEFB401B642801D90320BBE7C848006800F48C
:20AEE00000300028F2D010E0FFF7E0FB054606E0FFF7DCFB401B642801D90320A9E7BF48FE
:20AF0000006800F400300028F2D1207800F00200022857D1B948406800F00C0050B1B74839
:20AF2000406800F00C00082818D1B448406800F4803098B9B148006800F0020020B120690E
:20AF4000012801D0012084E7AC48006820F0F800616940EAC100A949086033E02069E8B1C3
:20AF60000120A7490860FFF7A1FB054606E0FFF79DFB401B022801D903206AE79F480068E5
:20AF800000F002000028F2D09C48006820F0F800616940EAC1009949086013E0002098498E
:20AFA0000860FFF783FB054606E0FFF77FFB401B022801D903204CE79048006800F002002D
:20AFC0000028F2D1207800F0080008282DD1A069B8B101208B490860FFF768FB054606E06F
:20AFE000FFF764FB401B022801D9032031E78348406A00F002000028F2D0012006F0C6F93B
:20B0000013E000207F490860FFF750FB054606E0FFF74CFB401B022801D9032019E77748FD
:20B02000406A00F002000028F2D1207800F00400042873D100267148C06900F0805070B99C
:20B0400000BF6E48C06940F080506C49C8610846C06900F08050009000BF00BF01266A4856
:20B06000006800F48070B0B96748006840F4807065490860FFF71AFB054606E0FFF716FB87
:20B08000401B642801D90320E3E65F48006800F480700028F2D000BFE068012806D1574880
:20B0A000006A40F001005549086227E0E06858B95248006A20F00100504908620846006ABD
:20B0C00020F00400086219E0E06805280BD14B48006A40F00400494908620846006A40F093
:20B0E000010008620AE04548006A20F00100434908620846006A20F00400086200BFE068C0
:20B10000A0B1FFF7D3FA054609E0FFF7CFFA401B41F28831884202D903209AE622E0374818
:20B12000006A00F002000028EFD012E0FFF7BEFA054608E0FFF7BAFA401B41F2883188423E
:20B1400001D9032085E62D48006A00F002000028F0D1012E05D12948C06920F080502749DE
:20B16000C86100BFE069C8B32448406800F00C00082860D0E069022848D100202049086630
:20B18000FFF794FA054606E0FFF790FA401B022801D903205DE61948006800F00070002864
:20B1A000F2D1206AB0F5803F07D11448406820F40030A168084311494860D4E90801084357
:20B1C0000E49496821F4741108430C49486001200B490866FFF76AFA054607E02DE0FFF713
:20B1E00065FA401B022801D9032032E60348006800F000700028F2D01FE000000010024008
:20B2000000004242800442420070004000200C490866FFF74BFA054606E0FFF747FA401B11
:20B22000022801D9032014E60648006800F000700028F2D101E001200BE6002009E60000EA
:20B240000000424200100240042808D14FF0E021096941F004014FF0E022116107E04FF052
:20B26000E021096921F004014FF0E022116170470EB55A480078012800D10EBD5848407EDB
:20B2800008B9022001E05648407E02465448418801235448F9F7F6FE5348007830B9534AA4
:20B2A0001188534A1088534A02F086FF524853490978CDE90010524802784D48006802908C
:20B2C0005048037848480078029902F04DFD4A480078C0434C49087047488079C0438871DE
:20B2E0004548B0F90200C04348804348B0F90400C043888045480078D0B94548027E4548E0
:20B3000001893C4B4248163008F0ACFD4248027E40484189374B4048163008F005FE3F487D
:20B32000027E3C488189334B3C48163008F05EFE3B48007828B93748018A2E4A3948FCF791
:20B3400053FC39493948F9F74FF8394804F05AFF38480088401C3749088008460088052827
:20B3600001DB0020088034480088401C32490880084600880A2801DB002008802F4800885B
:20B38000401C2E49088008460088322804DB002008802B48F9F782FF2A480088401C2949EF
:20B3A000088008460088642809DB002008800D4908780A22244905F053FC0C4988722348AA
:20B3C0000088401C2149088008460088B0F57A7F01DB0020088000BF4FE700005C0000202E
:20B3E0009C08002028030020C4000020B4070020220400206C010020CA000020C5030020DA
:20B40000C6000020C4030020D200002088030020F0120020081600200A13002024130020CE
:20B42000FE030020FC0300201A0400201E160020BC0900205E0000206000002062000020D5
:20B440008A01002064000020641200206600002070B504462546681EB0F1807F01D30120AC
:20B460000FE0681E4FF0E02148610F214FF0FF3005F01AFC00204FF0E021886107200861EC
:20B48000002070BD10B5FFF7F3FE10BD7047704710B50346002200BF93F83C00012801D1C7
:20B4A000022010BD012083F83C0000BF22F0FF00CC6840EA040222F440708C6840EA0402A7
:20B4C00022F480604C6840EA040222F400600C6840EA040222F480500C6940EA040222F4D7
:20B4E00000504C6940EA040222F480408C6940EA040222F400408C6940EA0402186842647B
:20B5000000BF002083F83C0000BF00BFC9E7024600BF92F83C00012801D1022070470120A5
:20B5200082F83C0000BF022082F83D001068406820F0700013685860106840680B681843FC
:20B54000136858601068806820F0800013689860106880684B68184313689860012082F8D9
:20B560003D0000BF002082F83C0000BF00BFD5E770B504460D4604222946206808F0DCF913
:20B580002068406C40F40040216848642068006840F0010021680860002070BD70B5044600
:20B5A0000D4600222946206808F0C6F900BF2068006A41F21111084050B92068006A891086
:20B5C000084028B92068406C20F400402168486400BF00BF2068006A41F21111084050B96F
:20B5E0002068006A8910084028B92068006820F001002168086000BF002070BD10B504468A
:20B600000CB9012010BD94F83D0028B9002084F83C00204600F00CF8022084F83D00211D82
:20B62000206808F041F9012084F83D000020E9E710B586B0044632492068884233D100BFB1
:20B640003048806940F400602E4988610846806900F40060019000BF00BF881402900020AD
:20B660000390049002A92848FEF780FE4FF46040029002200390059002A92348FEF776FED7
:20B680004FF47060029002200390059002A91F48FEF76CFE012211461920FFF7D6F819209A
:20B6A000FFF7C6F829E02068B0F1804F25D100BF1448C06940F001001249C8610846C0696F
:20B6C00000F00100019000BF00BF00BF0846806940F0040088610846806900F0040001909B
:20B6E00000BF00BF012002900020039004900220059002A90548FEF739FE06B010BD000074
:20B70000002C014000100240000C0140000801400146022081F83D000868006840F00100AC
:20B720000A681060012081F83D000020704701460868C06840F001000A68D06008680068EF
:20B7400040F001000A681060002070472DE9F04104460D46002600BF94F83C00012802D172
:20B760000220BDE8F081012084F83C0000BF022084F83D002068866826F0770626F47F4636
:20B7800020688660286850283BD00CDC202860D004DC002853D0102865D155E030285DD075
:20B7A000402860D141E0602835D070280DD0B0F5805F03D0B0F5005F55D115E020688068E7
:20B7C00020F00700216888604EE0D5E902136A68206808F0BFF82068866826F0770646F098
:20B7E0007706206886603FE0D5E902136A68206808F0B0F82068806840F48040216888609D
:20B8000032E0EA686968206808F082F95021206808F0ACF828E0EA686968206808F08DF932
:20B820006021206808F0A2F81EE0EA686968206808F06EF94021206808F098F814E00021DF
:20B84000206808F093F80FE01021206808F08EF80AE02021206808F089F805E030212068CD
:20B8600008F084F800E000BF00BF012084F83D0000BF002084F83C0000BF00BF71E77047F8
:20B8800010B5044620680069C0F34000D8B12068C068C0F34000B0B16FF0020021680861D5
:20B8A000012020772068806900F0030018B12046FFF7E5FF05E0204600F0D6F8204600F004
:20B8C000ABF90020207720680069C0F38000D8B12068C068C0F38000B0B16FF00400216830
:20B8E0000861022020772068806900F4407018B12046FFF7C4FF05E0204600F0B5F82046DB
:20B9000000F08AF90020207720680069C0F3C000D8B12068C068C0F3C000B0B16FF0080025
:20B9200021680861042020772068C06900F0030018B12046FFF7A3FF05E0204600F094F828
:20B94000204600F069F90020207720680069C0F30010D8B12068C068C0F30010B0B16FF008
:20B96000100021680861082020772068C06900F4407018B12046FFF782FF05E0204600F0D0
:20B9800073F8204600F048F9002020772068006900F0010058B12068C06800F0010030B181
:20B9A0006FF0010021680861204600F095F920680069C0F3C01058B12068C068C0F3C010A1
:20B9C00030B16FF08000216808612046FFF75EFD20680069C0F3801058B12068C068C0F35E
:20B9E000801030B16FF0400021680861204600F055FA20680069C0F3401058B12068C068F3
:20BA0000C0F3401030B16FF02000216808612046FFF73DFD10BD00001FB504460E49206871
:20BA2000884218D140200090022001900320039069460A48FEF79AFC00BF0949486820F499
:20BA4000406040F0E06040F44060486000BF0021044800F00BF81FBD0004004000100140CA
:20BA600000000140C81500207047000030B504460D4601222946206807F050FF0A49206814
:20BA8000884201D1012000E0002028B12068406C40F40040216848642068006840F0010012
:20BAA00021680860002030BD002C014070B504460D46164600BF94F83C00012801D1022059
:20BAC00070BD012084F83C0000BF022084F83D0036B1042E1BD0082E31D00C2E5ED145E0FD
:20BAE0002946206807F04CFF2068806940F00800216888612068806920F0040021688861FB
:20BB000020688069296908432168886147E02946206807F067FF2068806940F4006021685C
:20BB200088612068806920F480602168886120688069296940EA0120216888612FE0294607
:20BB4000206807F087FF2068C06940F008002168C8612068C06920F004002168C861206846
:20BB6000C069296908432168C86118E02946206807F0A6FF2068C06940F400602168C8618B
:20BB80002068C06920F480602168C8612068C069296940EA01202168C86100E000BF00BFB0
:20BBA000012084F83D0000BF002084F83C0000BF00BF85E710B504460CB9012010BD94F8DC
:20BBC0003D0028B9002084F83C00204600F00CF8022084F83D00211D206807F065FE0120F9
:20BBE00084F83D000020E9E708B5094A016891420DD100BF0749C96941F00201054AD1617C
:20BC00001146C96901F00201009100BF00BF08BD00040040001002407047000030B5044657
:20BC20000D4601222946206807F078FE0A492068884201D1012000E0002028B12068406C85
:20BC400040F40040216848642068006840F0010021680860002030BD002C014030B5044680
:20BC60000D4600222946206807F058FE19492068884201D1012000E0002090B100BF2068DC
:20BC8000006A41F21111084050B92068006A8910084028B92068406C20F400402168486423
:20BCA00000BF00BF2068006A41F21111084050B92068006A8910084028B92068006820F0BA
:20BCC00001002168086000BF012084F83D00002030BD0000002C014038B5044660480088F8
:20BCE000401C5F49088008460088B0F5967F01DB002008805B4840785B4B0090DA799979AE
:20BD000058795A4B1B7800F02BFE59480078401C574908700846007805280ADB5548006897
:20BD2000806840F0010053490968886000205049087051480068401C4F49086000F02AFA53
:20BD40004D48C08842F6FF7188420CDA4A480089494989880844484908810846C0888988E3
:20BD600008444549C880444A917A108904F014FF424948804249434803F0D2FC424800783C
:20BD8000424909784840FF281AD13F4880793F4989794840FF2813D13B4880883B49898840
:20BDA000484080B24FF6FF71884209D13648408836494988484080B24FF6FF7188420AD0C7
:20BDC000FEF774FC32490968401AC82807D902203049087003E0FEF769FC2D4908602D4845
:20BDE0000078012802D0022837D132E02648807901282DD128480078012804D1FBF770F9BD
:20BE000000202549087020480078012811D0022804D003280ED0042818D10CE0164B1A8926
:20BE2000164BB3F90210184BB3F90200FBF79CFC0DE000BF00BF104B1A89104BB3F90210C6
:20BE4000114BB3F90400FBF78FFC00E000BF00BF04E001201049087000E000BF00BF38BDD2
:20BE600010040020C6000020BC080020C40300200804002034160020C4050020B407002083
:20BE80006C01002078020020CA000020D20000200C04002030000020090400207047704784
:20BEA0002DE9F0470446206805682068C668206847694FF00008C14605F00F08B8F1000FF6
:20BEC0000AD105F0200038B106F0200020B1204608F00EFBBDE8F087B8F1000F6DD007F033
:20BEE000010018B906F49070002866D005F0010030B106F4807018B1E06B40F00100E063CF
:20BF000005F0040030B107F0010018B1E06B40F00200E06305F0020030B107F0010018B12D
:20BF2000E06B40F00400E06305F0080030B107F0010018B1E06B40F00800E063E06B68B374
:20BF400005F0200028B106F0200010B1204608F0CFFA20684069C0F38019E06B00F0080035
:20BF600010B9B9F1000F22D0204608F052FA2068406900F04000B0B12068406920F0400060
:20BF800021684861606B50B11748616B4863606BFDF746FE10B1606B416B88470CE0204671
:20BFA000FFF77DFF08E02046FFF779FF04E02046FFF775FF0020E0638CE705F0800030B173
:20BFC00006F0800018B1204608F0D8FB82E705F0400030B106F0400018B1204608F029FAF2
:20BFE00078E700BF76E70000C142010810B504460CB9012010BDA06900B100E000BF94F813
:20C00000390028B9002084F83800204600F028F8242084F839002068C06820F40050216826
:20C02000C860204608F0C6FA2068006920F49040216808612068406920F02A002168486156
:20C040002068C06840F400502168C8600020E063202084F8390084F83A000020CAE700001C
:20C0600010B586B004462B49206888424FD100BF2948C06940F480202749C8610846C06958
:20C0800000F48020019000BF00BF0815029002200390012004900320059002A91F48FEF725
:20C0A00065F94FF400600290002003900120049002A91A48FEF75AF900BF1949486820F04F
:20C0C000300040F0E06040F01000486000BF012211462720FEF7B9FB2720FEF7A9FB114876
:20C0E0000068C06840F480700E490968C8600D480068406940F001000A4909684861094847
:20C100000068C06840F0200006490968C86006B010BD0000004800400010024000100140A9
:20C1200000000140901D00207047704710B500F011F9054931F8100041F2555108440349CC
:20C1400008810020086010BDB47A0108C405002000B585B000BF0D48806940F010000B4966
:20C1600088610846806900F01000009000BF00BF4FF460700190002002900120039001A9DD
:20C180000348FEF7F3F805B000BD00000010024000100140F8B500F0DDF8064600F0DAF8DF
:20C1A000044600F0D7F80546A64203D1AC4201D15E4805705E48007830B95C4800785B49CD
:20C1C000487001205A4908705848007857494978884210D0FEF76AFA5649086056480078D2
:20C1E00028B155480078401C5349087017E001205249887213E0FEF759FA4E490968401A97
:20C20000C8280CD900204D4988724B4908704B498881C8814A4908700120484908744748DF
:20C22000807A10B9002047490870404800783F494978454A515C884245D14048006840B1CD
:20C240003E48006842F6AA21B1FBF0F03B49888002E00120394988803A480078401C394970
:20C2600008700846007802280DDD3448006844F63E11B1FBF0F031498881002030490870DF
:20C2800001202E4908742F4800780F280CDA274800782E4931F8100041F255510844274952
:20C2A00008810020888009E00F20264908701F480078264931F810002049088100201F49CD
:20C2C0000860C88026E019484078184909781E4A515C88421ED100201A490870174988807C
:20C2E00012480078194931F8100041F255510844124908814FF6FF70086011480078401C7F
:20C30000C0B20F490870052804DD0620087000200A490874054800680D49009002F002FBB6
:20C320000248007801494870F8BD00000C0300200E030020100300200F030020C4050020D6
:20C340001403002015030020A47A0108B47A01086C01002010B51E48C07AA8B94FF4007109
:20C360001C48FEF791F904464FF480711948FEF78BF944EA4000C4B280211648FEF784F92D
:20C3800044EA8000C4B220E04FF400711148FEF77BF908B9012000E0002004464FF48071A3
:20C3A0000C48FEF771F908B9012000E0002044EA4000C4B280210748FEF766F908B90120DE
:20C3C00000E0002044EA8000C4B204F0070010BDC40500200010014007E0044803F0DDF83C
:20C3E000002004F0C9FEFAF7ABFBF6E7EC00002070B50446204608F080FEA1890122A06842
:20C40000FEF74EF90120FAF776FBA1882068FEF73BF90546A1890022A068FEF741F9012094
:20C42000FAF769FB012D01D1012070BD0020FCE71FB50446A06808F0DDFD206808F0DAFD07
:20C44000A089009001200390112001906946A068FDF78CFFA0880090012003901120019049
:20C4600069462068FDF782FF1FBD2DE9F04704460F464FF000084FF08009204608F03DFEA0
:20C4800000251CE0A1890122A068FEF709F93220FAF731FBA1882068FEF7F6F80646012EB1
:20C4A00003D149FA05F040EA0808A1890022A068FEF7F6F83220FAF71EFB681CC5B2082D73
:20C4C000E0DB87F800800120FAF715FBBDE8F08710B50446204608F018FEA188012220680D
:20C4E000FEF7DEF80120FAF706FBA1890122A068FEF7D6F83220FAF7FEFAA1890022A068B7
:20C50000FEF7CEF8A18800222068FEF7C9F80120FAF7F1FA10BD10B50446204608F0F5FDAE
:20C52000A1890122A068FEF7BBF8A18801222068FEF7B6F83220FAF7DEFAA1880022206899
:20C54000FEF7AEF83220FAF7D6FAA1890022A068FEF7A6F810BD10B50446204608F0D5FD3A
:20C56000A18800222068FEF79BF8A1890122A068FEF796F83220FAF7BEFAA18801222068B9
:20C58000FEF78EF83220FAF7B6FAA18800222068FEF786F8A1890022A068FEF781F810BD58
:20C5A0002DE9F04104460D46A8468026204608F0ACFD002736E006EA0800C0B1A18801220A
:20C5C0002068FEF76DF83220FAF795FAA1890122A068FEF765F83220FAF78DFAA1890022EA
:20C5E000A068FEF75DF83120FAF785FA17E0A18800222068FEF754F83220FAF77CFAA1893A
:20C600000122A068FEF74CF83220FAF774FAA1890022A068FEF744F83120FAF76CFA761052
:20C62000781CC7B2082FC6DBA18801222068FEF737F80120FAF75FFABDE8F0810148024908
:20C64000086070470030000808ED00E0012023490978052910D12149103109789B290BD1C5
:20C660001E4914310978522906D11C4918310978052901D1032030E018490978042910D1E9
:20C68000164910310978C3290BD1144914310978B42906D11149183109780B2901D102208E
:20C6A0001BE00E49097881B90C491031097810290BD10A4914310978042906D1074918318B
:20C6C00009780A2901D1012007E005490968054A914201D1042000E000207047D0FF0FE080
:20C6E000002004E01004031300B585B000BF2B48806940F01000294988610846806900F045
:20C700001000009000BF00BF2548264908604014888008468088019000200290012003900E
:20C72000086801A9FDF722FE00201E4988714872C860C87108721A481B4908604FF4804085
:20C7400088800846808801900020029001200390086801A9FDF70AFE00201349887148723F
:20C76000C860C87108720E48104908604FF4004088800846808801900020029001200390EF
:20C78000086801A9FDF7F2FD0020084988714872C860C871087205B000BD000000100240D9
:20C7A00000100140A8140020BC140020D01400202DE9F04104460F4616469846069DB8F1EC
:20C7C000000F04D10121204608F078FC03E00221204608F073FCE07900F0010020B1012072
:20C7E0006072FDF763FFE060607A01281BD1207A50B9FDF75BFFE060FDF758FF20610020C5
:20C800006072012028700EE0FDF750FFE168401AB84208D9FDF74AFFE060002060722870D7
:20C82000FDF744FF2061287868B966B1FDF73EFF2169401AB04206D9FDF738FF20610020B6
:20C84000607201202870BDE8F0812DE9F04105460E4617469846B8F1F10F13D100240EE077
:20C86000BC4201D1012300E000231A4605EBC403998855F83400FDF713FF601CC4B2B4421A
:20C88000EEDB0DE0002409E005EBC402918855F834000022FDF704FF601CC4B2B442F3DBB6
:20C8A000BDE8F08110B586B000BF2A48806940F00400284988610846806900F00400019003
:20C8C00000BF00BF00BF0846806940F0080088610846806900F00800019000BF00BF002461
:20C8E00033E01D4A02EBC40291881B4A52F834000022FDF7D5FE184800EBC400808802907D
:20C900000120039002200590134951F8340002A9FDF72CFD114A02EBC40291880F4A52F841
:20C9200034000022FDF7BCFE0C4800EBC400808802900120039002200590084951F834001D
:20C9400002A9FDF713FD601CC4B2032CC9DB06B010BD000000100240C8030020E0030020A0
:20C960002DE9F0470746894692461C46DDF82080B9F1060F06D0B9F10C0F05D0B9F1FF0FB8
:20C9800006D103E0002505E0012503E0022501E0002500BF00BFBAF1060F06D0BAF10C0FC3
:20C9A00005D0BAF1FF0F06D103E0002605E0012603E0022601E0022600BF00BF43462A4672
:20C9C00003217548FFF741FF072F43D2DFE807F04204436F7AA6AD004CB9F12332460321BD
:20C9E0006E48FFF732FF00206D49088031E0B8F1F10F22D16B48408969490988884206DDE3
:20CA0000F123324603216548FFF71FFF0FE06548808963490988884206DDF0233246032167
:20CA20005E48FFF712FF02E000205D4908805C480088401C5A4908800BE0B8F1F00F08D1FA
:20CA4000F023324603215548FFF7FFFE0020544908809DE000BF04BB51480088B0F5167FFC
:20CA600006DAF123324603214C48FFF7EEFE0EE04B480088B0F5966F06DAF023324603216E
:20CA80004648FFF7E2FE02E000204549088044480088401C4249088008E04346324603218A
:20CAA0003E48FFF7D2FE00203D49088070E00CB9F12000E0F0200346324603213748FFF78C
:20CAC000C4FE65E004BB36480088B0F5167F06DAF123324603213148FFF7B7FE0EE0304836
:20CAE0000088B0F5966F06DAF023324603212B48FFF7ABFE02E0002029490880284800886F
:20CB0000401C2749088008E0F023324603212348FFF79BFE00202249088039E0F123324678
:20CB200003211E48FFF791FE32E01F4800881D490989884222DB1B4840891949098888423D
:20CB400006DDF123324603211448FFF77EFE0FE01448808912490988884206DDF0233246FC
:20CB600003210E48FFF771FE02E000200C4908800B480088401C0A49088008E0002008498C
:20CB80000880F023324603210448FFF75EFE00BF00BFBDE8F0870000C8030020E003002038
:20CBA000F8030020BC080020580300207CB504460D46094903C9CDE90001084802F0E0FC3A
:20CBC00001208DF8060003208DF8000000982060019860607CBD0000F85E0108EC000020EC
:20CBE0002DE9F74F82B088461546FE4903C9CDE90001FD48008800B2FC490880FC48B0F97B
:20CC0000020064286EDD0846B0F90000002869DDF748B0F9020064214843F449B1F90010E5
:20CC2000B0FBF1F000B2F34908800846B0F90040F1480068C0EB0420EF49096801EBA01006
:20CC4000ED49086008460068001200B2EB490880E648B0F90000EA49B1F90010401A0528B5
:20CC600011DDE348B0F90200E649B1F90010401A002804DDDF48B0F90000E3490880DC48FC
:20CC80004088E0490880D948B0F90000DC490880DE48007828BBDE48B0F9040019282ADD08
:20CCA000DC480088401CDB49088008460088282821DB00200880D148008881B2D648D74AE3
:20CCC000128820F81210D5480088401CD34908800846008832280EDB002008800120CB49E5
:20CCE000087008E0C148B0F90000C5490880C0484088C4490880CA48408800B2C949088001
:20CD0000A8F13204B4F5006F02DD4FF4006000E02046044604FB04F0C11700EB5151CC12E4
:20CD2000C14800796043B849B1F9001048430A2190FBF1F0C01200B2BC490880BA48007965
:20CD400000EB8000142101EB4000A849B1F90010884202DA0020B5490880B448B0F900006B
:20CD6000002803DDB148B0F9000000E00020AF4908800846B0F90000AA49B1F9001088421B
:20CD800003DAAA48B0F9000002E0A648B0F90000A649088005F00F00012806D002280FD01F
:20CDA000032818D004282CD120E04FF4FA6201219C48B0F9000006F0D3FC9D4908602BE0CB
:20CDC00040F2DC5201219748B0F9000006F0C8FC9749086020E04FF47A7201219148B0F974
:20CDE000000006F0BDFC9249086015E04FF4FA7201218C48B0F9000006F0B2FC8C4908601D
:20CE00000AE04FF47A7201218648B0F9000006F0A7FC8749086000BF00BF4FF47A720121C0
:20CE20008048B0F9000006F09BFC824908607848807968B96E48B0F90200642808DD6C4861
:20CE400040887D4908800846008800047B49086005F00F00012806D0022814D0032824D086
:20CE6000042841D133E07149B1F9001001EBC1010811724B6F490A686D49096808F062F9C5
:20CE80006D4908803DE06949B1F9001001EB410202EBC1010811694B66490A6864490968E1
:20CEA00008F050F9644908802BE06049B1F9001001EB810202EBC1010811604B5D490A6894
:20CEC0005B49096808F03EF95B49088019E05B4B58480268564801685448B0F9000008F0F5
:20CEE00031F9554908800CE0544B52480268504801684E48B0F9000008F024F94E490880DF
:20CF000000BF00BF6FF0C7004D49086140F6340048614C4AD2895110474AB2F9002050104D
:20CF2000474A03F0E3FF484908806FF063004449086140F21A4048612D4A1289D1113A4A0D
:20CF4000127A4FF47A735A43D011404A03F0CEFF3F490880324A117B254AD0883D4A12884D
:20CF600000F0C0FF07463B48078001231A463A480188384601F006F9374908802A4A517A67
:20CF80001B4A907D00F09CFF8246274A527A0F3A91B2174A507D00F093FF83460AFB0BF08A
:20CFA0004FEA90291FFA89F001231A462B49098801F0E8F8294908802348B0F90000264916
:20CFC00009884843861225480088704386122448007828B923480068301A02284ADD43E007
:20CFE00054E00000E85E0108580300200E010020B407002014010020F000002016010020AD
:20D000001201002010010020F4000020F8000020CA000020FA000020EC060020F600002054
:20D02000DC080020180100209C0800201A0100201C010020200100202401002008010020C8
:20D04000A4060020C40500202E0100208006002030010020320100203401002036010020D8
:20D060002C0100202801002024480068801C2349086018E021480068301A10F1030F12DAC4
:20D080001E480068C01E1D4908600CE01B480068132805DD1948006810381849086002E086
:20D0A0000020174908701548006810F1C80F03DA6FF0C700114908601248008818B9124809
:20D0C00002F06BFA02E0104802F05AFA0B4800680E49B1F900100844401000B2ADF80400B6
:20D0E00001208DF8060004208DF800000099029801600199416005B0BDE8F08F28010020EA
:20D100002C01002024010020EC000020300100202DE9F04F8BB082460E469346F84903C98E
:20D12000CDE90901002008900790F6490870F6480068C0EB8620F449096801EBE010F2496D
:20D14000086008460068C0F38F20F049088008460088EF494880EF480088C82801DA6420AA
:20D1600002E0EC480088401005900598864204DBFDF79CFAE849086018E0E848B0F90200F2
:20D18000C82807DDE548B0F90200E54991FBF0F087B201E04FF49667FDF788FADE490968E1
:20D1A000401AB84202D90120D9490870DB4800883C2814DDD7480088C82801DA96200CE071
:20D1C000D4480088B0F52F7F02DD40F20D2004E0D048008800EB40008010069010E0CD4840
:20D1E0000088C82801DA962009E0CA480088B0F52F7F02DD40F20D2001E0C6480088069005
:20D200000698864202DB0020C1490870C5484078012802D0C348807810B90120BC490870FF
:20D22000BB480078012815D1B948B0F906000A2806DA0020B649C880BB4802F0AEF936E386
:20D24000B348C0880E3800B2B149C880B64802F097F92CE3B148B0F90200B0F5FA7F23DD00
:20D26000B04800780F281FDBA9484088C8281BDDAA48B0F9020064214843AA49097890FBC0
:20D28000F1F0AA490860AA4800680968C0EB0130A749096801EBA020A54908600846006892
:20D2A000C0F30F30A3490880BBF1030F7ED006DCBBF1010F0AD0BBF1020F78D183E0BBF16F
:20D2C000040F75D0BBF1330FF7D124E29A48007A08909948407A079090480088642804DC48
:20D2E0004FF480609549088016E08C480088F0280FDC8A48008800EBC00101EB80100A21A3
:20D3000090FBF1F040F2DA61081A00B28B49088002E0002089490880894800688749B1F9F5
:20D320000010C0EB81208649096801EB60208449086008460068801200B2824908807448A7
:20D340004088B1F900104843800A04B204EB440040000A2190FBF1F004B27748C088A042D7
:20D3600002DA7548C08800E0204604B2724840897549097A48434FF47A714843401400EB89
:20D38000C00101EB00104FF6FF7101EA8005012305226E480188284600F0F4FE6B49088095
:20D3A0006548C08840426A49086102E084E02BE226E1002048616048C088800240428861DA
:20D3C0000020C86125E25C48007D08905A48407D079052480088642804DC40F2335057496B
:20D3E000088016E04D480088F0280FDC4B480088C0EB401101EB80100A2190FBF1F040F62F
:20D40000E901081A00B24D49088002E000204B4908804B4800684949B1F90010C0EB81207F
:20D420004749096801EB60204549086008460068801200B24349088035484088B1F900107C
:20D440004843800A04B204EB440040000A2190FBF1F004B23848408AA04202DA3648408AF1
:20D4600000E0204604B23448C08A3749097A48434FF47A714843401400EBC00101EB0010A7
:20D480004FF6FF7101EA8005012305222F480188284600F077FE2D4908802748408A404290
:20D4A0002B490861002048612348408A8002404288610020C861ACE11F4890F82000089027
:20D4C0001D4890F82100079014480088642804DC40F26660194908803FE010480088F0285E
:20D4E00038DC0E480088752148430A2190FBF1F040F6F821081A00B2104908802DE0000071
:20D50000005F01084E010020480100204C010020DC0000208603002040010020B40700207D
:20D520002055030028030020EC0000206001002064010020BA010020D009002050010020D1
:20D5400054010020520100209C08002046010020C80600200020FE490880FE480068FC49E8
:20D56000B1F90010C0EB8120FA49096801EB6020F849086008460068801200B2F64908801B
:20D58000F6484088B1F900104843800A04B204EB440040000A2190FBF1F004B2F048C08BBD
:20D5A000A04202DAEE48C08B00E0204604B2EC48408CEC49097A48434FF47A7148434014E0
:20D5C00000EBC00101EB00104FF6FF7101EA800501230522E4480188284600F0D3FDE24925
:20D5E0000880DF48C08B4042E049086100204861DB48C08B8002404288610020C86108E1C7
:20D60000D74890F82C000890D54890F82D000790D748008832280DDCD5480088C0F13200C4
:20D6200000EB800040F6DE0101EB400000B2C84908801DE0CE480088642804DC40F6DE00D8
:20D64000C349088014E0CA480088F0280DDCC8480088A22148430A2190FBF1F040F6327151
:20D66000081A00B2BA49088002E00020B8490880B8480068B649B1F90010C0EB8120B54955
:20D68000096801EB6020B349086008460068801200B2B1490880B1484088B1F900104843C7
:20D6A000800A04B204EB440040000A2190FBF1F004B2AB48408DA04202DAA948408D00E04E
:20D6C000204604B2A648C08DA649097A48434FF47A714843401400EBC00101EB00104FF6FC
:20D6E000FF7101EA8005012305229F480188284600F048FD9C4908809948408D40429B496B
:20D700000861002048619648408D8002404288610020C8617DE0924890F83800089090488F
:20D7200090F83900079092480088642804DC40F639108749088014E08D480088F0280DDC9A
:20D740008B480088A82148430A2190FBF1F040F6CF71081A00B27E49088002E000207C4923
:20D7600008807C4800687A49B1F90010C0EB81207849096801EB60207649086008460068B1
:20D78000801200B27449088074484088B1F900104843800A04B204EB440040000A2190FBCE
:20D7A000F1F004B26E48C08EA04202DA6C48C08E00E0204604B26A48408F6A49097A4843D0
:20D7C0004FF47A714843401400EBC00101EB00104FF6FF7101EA80050123052262480188F1
:20D7E000284600F0CFFC604908805D48C08E40425E490861002048615948C08E800240428E
:20D8000088610020C86104E0002008900790002400BF00BF51488480B0F90400002802DCB1
:20D8200000204E4988804D48B0F904004B49B1F90610401A022807DD4848C1880898084466
:20D8400000B24649C88010E04448B0F904004349B1F90610401AB0F1FF3F06DA3F48C188E1
:20D860000798081A00B23D49C8803C48B0F90600062801DA062002E03848B0F90600374974
:20D88000C8803B4801883748007940F682225043B1EB202F08DD0120304908700020C88085
:20D8A000344801F07AFE02E0324801F069FE324A117B2F4AD088314A128800F013FB80461D
:20D8C0002E48A0F8008001231A462D480188404600F058FC2A490880224A517A244A907DC1
:20D8E00000F0EEFA03901F4A527A0F3A91B2204A507D00F0E5FA0290DDE902104843810A76
:20D900000491049988B201231A461E49098800F039FC1C4908801648C07B052801DC052045
:20D9200007E01348C07B0A2801DB0A2001E01048C07B0D49098848434FF47A7190FBF1F0B2
:20D9400000B201900A480089C111084A01981BE0500100205401002052010020DC0000209C
:20D96000D00900209C08002046010020C8060020B4070020EC000020DC0800205801002031
:20D980005A0100205C01002003F0B0FA144908801448B0F906001449098848434FEAA02987
:20D9A0001248008809FB00F04FEAA0290C48B0F9000048444FEA60090FFA89F0ADF8260017
:20D9C00001208DF82A0002208DF824000998CAF800000A98CAF804000BB0BDE8F08F000002
:20D9E00044010020DC0000205A0100205C0100202DE9FF5F82460E46874903C9CDE90201E9
:20DA0000002700BF0025012E56D184484088400141F2883190FBF1F0C5B2012D01DA0120D7
:20DA200000E0284605467D48408840017C4909784843642190FBF1F00A387A49496888423D
:20DA400005D97848406828447649486026E0734840884001724909784843642190FBF1F02B
:20DA60000A307049496888420DD26E484068A84205D96C484068401B6A4948600EE0002013
:20DA8000684948600AE0654840884001644909784843642190FBF1F062494860624A128949
:20DAA000D111624A127A4FF47A735A43D011604A03F01CFA044635E04FF000095B48C07F62
:20DAC00008B9872001E05948C07F8146554840680A21C1EB4911884205D252484068401CA1
:20DAE0005049486010E04F4840680A2101EB4911884205D94B484068401E4A49486003E0E6
:20DB00004FEA491047494860474A1289D111474A127A4FF4FA735A43D011454A03F0E6F981
:20DB2000044600BF404AB2F902103E4A5268520910B2404A03F0DAF90746381907B2012E60
:20DB400026D04FF000093948807F08B93C2001E03648807F814634480088A9F105018AB2E5
:20DB6000009088B280230021F9F79CFF7843800A07B22D480088484506DD002029494860E7
:20DB80002D4801F00AFD02E02B4801F0F9FC02E0294801F0F5FC214A117B234AD088274A7B
:20DBA000128800F09FF980462448A0F8008001231A4623480188404600F0E4FA204908803C
:20DBC0001A4A517A184A907D00F07AF9019001231A461C480188019800F0D4FA1949088001
:20DBE0001748008878434FEAA02B084600880BFB00F04FEAA02B0FFA8BF0ADF80C00012059
:20DC00008DF80E008DF808000298CAF800000398CAF80400BDE8FF9FF05E0108DC08002089
:20DC20008D010020E4000020B40700209C08002080060020A4060020EC00002038010020BE
:20DC40003A0100203C01002070B504460D461646FCF72CFD3C490968401A642870D3FCF7C0
:20DC600025FD394908603948006828443749086037480078401C364908700846007808281B
:20DC80000ADB32480068C0F3CF003249088000202F4908702D490860462C0BDA2D480088F6
:20DCA00041F27071884205DD2B480088401C2A49088002E0002028490880462C05DC254897
:20DCC000008841F28831884207DA962E05DA23480088401C2149088002E000201F4908804F
:20DCE0001D480088B0F5967F05DD00201A49088001201B49087019480088642804DD00201D
:20DD0000164908801649087015480078012814D1462C0EDA04F11E0012490870084600785C
:20DD2000642801DD642001E00E4800780D49087006E064200B49087002E064200949087012
:20DD40000848007870BD0000980000209C000020A0000020A2000020A4000020A60000204E
:20DD6000A8000020A90000202DE9FF4383B0074615469846DDE90E9408EA090202F00103A6
:20DD8000BDF81210434A10782A4601F0B9FB06462078B04223D04048007800BB05260120B2
:20DDA0003D4908702078042819D13C480068142806DD0426002008700120394908700EE0E1
:20DDC00000203849086038490860384908803349086033490870052601202F490870062E00
:20DDE00045D2DFE806F04412362A034505F00F02BDF8121001A8FEF7F3FE01982060029832
:20DE000060600020244908703FE029480078012807D12848B0F902004001254948600020A2
:20DE20000870394601A8FFF7E3FD019820600298606000201849087027E0294601A8FEF7EC
:20DE4000B5FE01982060029860600020124908701BE0BDF810102A4601A8FFF759F90198DF
:20DE600020600298606000200B4908700DE000BF114801F092FB1148F7F716FD052020704A
:20DE80000020A0716080A08000BF00BF07B0BDE8F08300009C08002068010020280100206E
:20DEA0002C010020F00000200801002024010020E4000020B4070020EC0000206C0100201F
:20DEC00010B502464FF480608A4208DD01FB01F4A302B3FBF2F4B4FBF2F4A0B201E04FF42C
:20DEE000806010BDF0B503460E461546002100244FF48060182E04D0242E12D0302E34D1BF
:20DF000021E0E721FC2401EBC10707EB0117B3EB870F02DD4FF4806701E0B3FBF1F73A46E6
:20DF200025E04FF4A5714FF4B47401EBC10707EB0117B3EB870F02DD4FF4806701E0B3FB8E
:20DF4000F1F73A4613E040F2AD114FF4EA7401EBC10707EB0117B3EB870F02DD4FF48067DA
:20DF600001E0B3FBF1F73A4601E0642200BF00BF02FB02F74FF0640CB7FBFCF75743B7FB2F
:20DF8000FCF75743BF0242F2107CB7FBFCF2B2F54D7F02D24FF44D7700E017463A46AA42DC
:20DFA00001D290B200E0284604EBC40707EB0417B3EB870F01DD4FF48060F0BD2DE9F0410E
:20DFC00005460E4617461C46002F7DD1552D66D14748007820BBFCF769FB45494968401ADB
:20DFE000B0F57A7F15D90120414908700020207040480078C043404908703E484078C0437D
:20E0000048703E48007820F00200801C3B49087018E03A48007820F002003849087011E0B2
:20E020000020207033480078C0433349087031484078C04348703148007820F00200801CBB
:20E040002E490870AA2E06D12C48007820F004002A49087023E02A480078C8B9FCF726FBB5
:20E0600027494968401AB0F57A7F0AD90120244908702248007820F00400001D1F490870AB
:20E080000DE01E48007820F004001C49087006E01A48007820F00400001D18490870194899
:20E0A0000078D8B9FCF702FB16494968401AB0F57A7F0CD90120134908701048007820F0A5
:20E0C0000100401C0D4900E00FE008700DE00B48007820F001000949087006E00748007806
:20E0E00020F00100401C05490870BDE8F081000098010020C6000020C800002070010020BF
:20E10000A0010020A80100200120114908700020486001200F490870002048808880C88091
:20E120000D4908600D4908600D4908600D4908600D4908600D4908620D4908620D490862E9
:20E140000D4908620D4908620D49086270470000E4000020DC00002004000020080000207C
:20E160000C000020100000201400002038060020140600205C060020C8060020A40600203D
:20E180008006002070B504461546661A32B2002A06DDAA4202DB4E19B0B20CE020460AE0D0
:20E1A000002A07DA56429E4202DBCE1AB0B202E0204600E0204670BD70B505460E461446DC
:20E1C00008216748FCF760FA664908704FF400416548FCF759FA6549087062480078644987
:20E1E00009784840634908705E480078604908705E480078604909784840604908705B481F
:20E2000000785D490870574800785849097848405B490870FCF74AFAB0F57A7F0CD2FCF7E5
:20E2200045FA58490860FCF741FA57490860FCF73DFA5649086070BD2088C0F380300028CF
:20E2400078D1B5F5966F7CDD462E7ADD4948007800BBFCF72BFA4B490968401A42F21071B2
:20E2600088421BD9206820F4804000F5804020600120474948800846F8F7AEFF002045493E
:20E28000087045484088401C43494880022043490870D0E7FCF70AFA3A490860374800784B
:20E2A00000BBFCF703FA38490968401A41F2883188421BD9206820F4804000F5804020602C
:20E2C0000220334948800846F8F786FF00203149087031484088401C2F49488002202F498D
:20E2E0000870A8E7FCF7E2F9274908602448007810BBFCF7DBF925490968401A41F28831D6
:20E3000088422AD9206820F4804000F58040206003201F4948800846F8F75EFF00201D492C
:20E3200008701D484088401C1B49488002201B49087080E711E004E0FCF7B8F9134908600E
:20E340000BE0FCF7B3F90F490860FCF7AFF90E490860FCF7ABF90D49086000BF6BE70000B3
:20E36000000C01407402002000080140750200205D0200205C0200206502002064020020D0
:20E380006C02002060020020680200207002002024120020040300201C09002079010020F5
:20E3A0001FB53948007890B93848807E55280ED1374A384800783849498889B2CDE90102AE
:20E3C00000913649887836490EC900F0ABFE3049344A30480078CDE902210190304880688D
:20E3E0000090314801782E480CC8304800F032FF274801902E488088ADF80000264B5B8841
:20E400009AB2254B1989234B9879294B1C6802949B88ADF80C30234600F0A4FD1E4A917D1D
:20E42000507D1B4A00F020FD20490839088A184900F076FA1E48016802918088ADF80C0085
:20E44000134ADDE9020100F0D3FB114800F03EF80F48134A009011780F4A528890B2154AB8
:20E4600012680392144A1388039A00F095FC084812490090CA8912490878124B12490988C4
:20E4800000F010FB1FBD0000C40000209C0800206C010020CA000020B40700205803002030
:20E4A0002803002084030020C6000020101600203204002022040020BA0100201E16002073
:20E4C00090010020CF0500208A01002010B50446FCF7ECF841F2883188420CD2FCF7E6F8A1
:20E4E000EE490860FCF7E2F8ED490860FCF7DEF8EC49086010BD2068C0F3804000286FD17C
:20E500004FF40041E848FCF7BFF800BBFCF7CEF8E3490968401A41F2883188421BD9206800
:20E5200020F4802000F5802020600120DF4948800846F8F751FE0020DD490870DD484089C9
:20E54000401CDC4948810220DB49087003E0FCF7ADF8D3490860D9480088002847D1D848AB
:20E560000078012843D1D748007805283FD0D548807901283BD1D348B0F90400C82804DC30
:20E58000D048B0F90200C82831DDCF48807A40BBCE480089C82825DAFCF788F8C149096832
:20E5A000401A41F28831884225D9206820F4802000F5802020600220BC494880BF4800887E
:20E5C00088800846F8F708FE0020B9490870B9484089401CB74948810220B74908700AE0E3
:20E5E0008DE0FFE7FCF762F8AE49086003E0FCF75DF8AC490860FCF759F8A8490968401A94
:20E6000014287CD3FCF752F8A4490860B048C088B04909680844AF490860AF480088AF4910
:20E6200009680844AD490860AB484088AC4909680844AB490860A8488088AA49096808444E
:20E64000A8490860A8480078401CA74908700846007820287EDB002008709E4800684FF4A5
:20E66000FA71B1EB501F2FD89A480068C900B1EB501F29D39948006841F28831B1EB501FC3
:20E6800022D8964800684EF66021B1EB501F1BD39348006841F28831B1EB501F14D890487E
:20E6A00000684EF66021B1EB501F0DD38D48006841F28831B1EB501F06D88A4800684EF6B2
:20E6C0006021B1EB501F16D2206820F4802000F5802020600320754948800846F8F77CFD16
:20E6E00000207349087073484089401C714948810220714908707D480068C82100E0C2E077
:20E70000B1EBA02F36DA7A48008872490968C0EB511019282AD277480078401C75490870F6
:20E72000084600780A2828DD206820F4802000F58020206004205D49488066480068C0F330
:20E740004F1088800846F8F747FD002058490870584800E01AE04089401C5649488102206F
:20E760005549087000206349087006E000206149087002E000205F490870002055490860CF
:20E780005649086056490860564908604F48407B00287AD14D484088002876D1FBF786FF5C
:20E7A00055490968401A41F28831884274D94848C0885249524A127821F812004648008813
:20E7C00050494F4A127821F81200434841884E484B4A127820F812103F4881884B48484A5A
:20E7E000127820F8121046480078401C444908700846007832284FDB0020087032213F4832
:20E80000F9F783FB4249086032213E48F9F77DFB4049086032213C48F9F777FB3E4908603D
:20E8200032213A48F9F771FB3C49086038480068B0F5FA7F0DD83748006842F6E0618842A5
:20E8400007D835480068884203D834480068884222D9206820F4802000F580202060052030
:20E86000124948802A48008888800846F8F7B4FC00200F4908700F484089401C0D494881FB
:20E8800002200D49087007E0FFE700201C490870FBF70CFF1849086000BF2BE60002002006
:20E8A00004020020080200200010014024120020040300201C0900207901002082010020B8
:20E8C00030000020CA000020C4050020B40700201E160020100200201A0400201402002040
:20E8E000180200201C0200200C02002004000020380400200D020020340200201410002029
:20E900002002002078100020DC1000204011002024020020280200202C0200203002002060
:20E920007047000013B50C465448007860B9FBF7BDFE534908609DF8012006215148F5F7C6
:20E94000C0F801204D4908702078C0F3C01000287ED19DF8000018B19DF80000072821D12A
:20E96000FBF7A4FE46490968401AB0F57A7F1DD9206820F080008030206001204249488059
:20E980009DF8000088800846F8F726FC00203F4908703F48C08A401C3D49C88201203D49B7
:20E9A00008701CBDFBF782FE354908609DF800009DF8011088425FD09DF8001036480278DD
:20E9C0000078401C344B18702E48815418460078062851DB00201946087006212948F6F765
:20E9E000CDFC28B92D480068401C2C49086006E000202A490860FBF759FE294908602748E4
:20EA00000068322838D9FBF751FE2549096801F5FA71884230D9206820F080008030206087
:20EA20000220194948801748007800021549497800EB011013498978084413498880114830
:20EA4000C07800020F49097900EB01100D4900E012E0497908440C49C8800846F8F7BCFBDF
:20EA600000200A4908700A48C08A401C0849C88201200849087094E700BF92E74602002013
:20EA800048020020500200202412002004030020EC0800207901002056020020580200207D
:20EAA0004C0200202DE9F04105460E4614469846069FFBF7FBFDB0F57A6F01D2BDE8F081C4
:20EAC000FBF7F4FD42F21071884220D23868C0F3804000287CD1FBF7E9FD3E490968401A30
:20EAE000142875D3FBF7E2FD3A49086098F80000A8BB0DB1C82E0BDD40F2C270844207DD39
:20EB000040F63E00844203DA0020334908705FE031480078401C3049087008460078FA2865
:20EB200056DB00200870386820F4802000F58020386008202949488005EB8600888008465D
:20EB4000C480F8F749FB00202549087025484089401C2449488102202349087038E0FFE76C
:20EB60000DB1C82E03DD002088F8000030E040F68B60844202DCB4F5BA7F26DA1B480078CF
:20EB8000401C1A49087008460078FA2820DB00200870386820F4802000F580203860092019
:20EBA0000E49488005EB860088800846C480F8F713FB00200A4908700A484089401C094975
:20EBC000488102200849087002E000200749087000BF73E740020020440200202412002080
:20EBE000040300201C090020790100204502002037B514466048007801280CD0FBF756FDF8
:20EC00005E490860FBF752FD5D490860FBF74EFD5C4908603EBD2068C0F30040002875D168
:20EC2000BDF90000002801DB014600E0414244F62062914228DDFBF739FD50490968401A50
:20EC4000B0F57A7F24D9206820F4803000F58030206001204C494880BDF90000002801DB70
:20EC6000014600E04142484A91801046F8F7B4FA0020464908704648C088401C4449C88026
:20EC8000022044490870C5E7FBF710FD3B490860BDF90200002801DB014600E0414244F616
:20ECA0002062914228DDFBF701FD35490968401AB0F57A7F24D9206820F4803000F5803035
:20ECC0002060022030494880BDF90200002801DB014600E041422C4A91801046F8F77CFAA9
:20ECE00000202A4908702A48C088401C2849C8800220284908708DE7FBF7D8FC2049086024
:20ED0000BDF90400002802DB014601E031E0414244F62062914228DDFBF7C8FC194909685B
:20ED2000401AB0F57A7F24D9206820F4803000F580302060032014494880BDF90400002843
:20ED400001DB014600E041420F4A91801046F8F743FA00200D4908700D48C088401C0C4905
:20ED6000C88002200B49087054E7FBF79FFC0549086000BF4EE7000030000020E801002092
:20ED8000EC010020F001002024120020040300201C090020790100202DE9FF4105460E4604
:20EDA0001F460A9C2068C0F3805000284DD1FBF77DFC27490968401A142846D3FBF776FC98
:20EDC00023490860B5F5FA7F3CDD0F2E3ADBBDF80800C82836DDBDF80A00322832DA40F2BA
:20EDE000DC5087422ADD1B480088401C1949088008460088FA2828DB00200880206820F4A7
:20EE0000800000F580002060012013494880BDF808008880BDF80A00C8800846F8F7DCF95A
:20EE200000200E4908700E4890F82400401C0C4981F8240001200B49087006E00020054952
:20EE4000088002E0002003490880BDE8FF810000380200203C0200202412002004030020FA
:20EE6000EC0800207901002070B504460E461546FBF71CFC41F28831884201D35A2C08DDC7
:20EE8000FBF714FC31490860FBF710FC2F49086070BD2888C0F34020002855D1052C01DB65
:20EEA000BE2C22DDFBF702FC28490968401A41F2883188421DD9286820F4007000F5007018
:20EEC000286001202249488008468480C680F8F783F900201F4908701F48408B401C1E495E
:20EEE000488301201D490870D2E7FBF7DFFB17490860052E01DBBE2E22DDFBF7D7FB1849DC
:20EF00000968401A41F2883188421DD9286820F4007000F50070286002200D4948800846EB
:20EF20008480C680F8F758F900200A4908700A48408B401C08494883012008490870A7E74F
:20EF4000FBF7B4FB0649086000BFA1E7E00100202412002004030020EC08002079010020E6
:20EF6000E40100200FB42DE9F04105460E4617460B9C2088C0F30020002877D1012D76D17F
:20EF800041F28830864272DDB7F5FA7FFBDDBDF92400002801DB014600E04142B1F5967F2F
:20EFA0002CDAFBF783FB58490968401A41F28831884227D9206820F4807000F580702060C8
:20EFC000012052494880BDF92400002801DB014600E041424D4A91801046F8F7FDF8002023
:20EFE0004B4908704B48008B401C4A490883012049490870BDE8F0015DF814FBFBF756FB05
:20F0000041490860BDF92600002801DB014600E04142B1F5967F2BDAFBF748FB3F49096886
:20F02000401A41F28831884226D9206820F4807000F580702060022034494880BDF926008D
:20F04000002801DB014600E04142304A91801046F8F7C2F800202E4908702E48008B401C0C
:20F060002C49088301202C490870C3E73CE03CE0FBF71CFB29490860BDF92800002801DBDB
:20F08000014600E04142B1F5967F29DAFBF70EFB23490968401A41F28831884231D920688E
:20F0A00020F4807000F580702060032017494880BDF92800002801DB014600E04142134AB3
:20F0C00091801046F8F788F80020114908701148008B401C0F49088301200F49087089E7E4
:20F0E000FBF7E4FA0E4908600BE0FBF7DFFA06490860FBF7DBFA09490860FBF7D7FA08497F
:20F10000086000BF76E70000D40100202412002004030020EC08002079010020D801002052
:20F12000DC0100202DE9FF410646DDE90A870C9C00252078C0F34010002878D1052F08D1F3
:20F14000FBF7B4FA3B490860FBF7B0FA3A4908606DE0012F01D0042F32D1B8F1320F2ADD27
:20F160004EBB364890FBF8F085B242F21070854200DA00E028460546FBF798FA2D49096805
:20F18000401AA84253D9206820F020002030206001202B4948800846F8F71EF80020294935
:20F1A00008702948408A401C27494882012027490870BDE8FF81FBF779FA1E49086036E08E
:20F1C0009DF8040005282EDB9DF8050058BB56BB9DF804001E4991FBF0F085B242F210704B
:20F1E000854200DA00E028460546FBF75FFA12490968401AA8421AD9206820F0200020307F
:20F20000206002200E4948800846F7F7E5FF00200C4908700C48408A401C0B494882012067
:20F220000A490870C5E7FBF741FA0349086000BFBFE70000C8010020CC01002048F13E00C4
:20F240002412002004030020EC08002079010020D8B805000FB42DE9F84305460E46DDE975
:20F260000D840F9FFBF722FA41F28831884203D35C480078012819D1FBF718FA5A49086077
:20F28000FBF714FA58494860FBF710FA56490864FBF70CFA54494864FBF708FA5249C1F895
:20F2A0008000FBF703FA5049C1F88400FBF7FEF94E490968401A142847D3FBF7F7F94B49F2
:20F2C0000860222E27D006F00F0020B39DF828001E2820DD9DF82900E8B9B8F1020F1AD1A3
:20F2E00000949DF8283028883F4A012100F088F800949DF8283068883B4A4032022100F047
:20F300007FF800949DF82830A888374A8032032100F076F819E0FBF7C9F933490860FBF78D
:20F32000C5F931494860FBF7C1F92F490864FBF7BDF92D494864FBF7B9F92B49C1F8800042
:20F34000FBF7B4F92849C1F884003878C0F38010F0BB207800F001002178C1F3400108445F
:20F360002178C1F380010844022838DD386820F0400040303860207800021D4948801A4812
:20F38000418FB0F87A0001EB80011748B0F8BA0001EB001016494988084315494880124856
:20F3A000818F90F87C0001EB0020114988800E48B0F8BC00C8800846F7F70EFF00200D490A
:20F3C00008700D48808A401C0B498882012000E005E00A490870BDE8F8035DF814FB00BF28
:20F3E000F9E70000C4000020540F0020D00100202412002004030020EC08002079010020AA
:20F400002DE9F0470546884614469946089E002708E004F10800791C30F8111020F817107E
:20F42000781C87B2182FF4D32587192104F10800F8F76BFDE063E06B0A2812D2FBF736F9F2
:20F440002168401A43F6982188420DD93078A8F1010101228A401043307001206087BDE857
:20F46000F087FBF723F92060322D03DB40F6D270854210DDFBF71AF96168401AB0F57A7F58
:20F480000CD93078A8F1010101228A401043307002206087E3E7FBF709F9606000BFDEE759
:20F4A00010B51149487B01F03BFC0F49487B05F00DFB0E4803F0D2FB0C48F6F7F5F90C4891
:20F4C00001890C4804F0F4FD094841890A4804F0EFFD07488189094804F0EAFD01F020FE88
:20F4E000012001F049FE10BD9C0800206C01002008160020F01200200A13002024130020A1
:20F500002DE9F04107460E46154698461948006818BBEDB1B8F1010F1AD1FBF7C7F840F605
:20F52000B831884214D9642E03DDAA2F01D104240FE0322E0DDA222D01D1012409E005F08C
:20F54000F00018B1332D01D0032402E0022400E00524012001F010FE08E0052400200649E9
:20F56000087008460078C043044908702046BDE8F08100006C010020C6000020C8000020AE
:20F5800010B50446207838B9F7F7C4FDFCF7CEFDF8F7E4F80120207010BD10B5044601F01D
:20F5A000D9FEF8F7C9F8FEF7AFFD0020207010BD2DE9F04107460D46144605EB4500C0F37D
:20F5C0004F06207800F0010050BBB74203DAFBF76DF81C490860FBF769F81A490968401AC7
:20F5E00041F2883188422AD9206820F00100401C206002201449488008468680F7F7ECFD6B
:20F6000000201249087012480089401C10490881012010490870FBF749F80F4908600EE003
:20F62000FBF744F80C490968401A41F28831884205D90A48006820F0010008490860BDE8BF
:20F64000F0810000A80200202412002004030020EC08002079010020AC0200206C010020E9
:20F660001CB528492848808B10B940F6B83001E02548808B254CCDE90001237B244C2478BB
:20F6800014B9244C248801E0234CE4882246224CE17B1F4C207800F0F7F91C4A117B224656
:20F6A000127812B91B4A128801E01B4AD2881046144A00F0FFF8194A917A174A1089114AF8
:20F6C00000F060F90F48104C0090A37A124CA27D617DE07D00F04EF822461189D088094AE6
:20F6E00000F094FA084A127A02EB4203C3EBC2124FF6FF7303EAC20122461089014AFFF751
:20F7000057FF1CBD6C0100209C080020DC080020A801002034080020B4070020C40500207C
:20F7200070B504460D46207868B900200F4908700F480078C0B90E480078401C0C4908701F
:20F74000F7F7CEFC10E000200949087007480078012802DB0020207001E0F7F7F1F9034896
:20F760000078401C0149087070BD0000B0020020B10200202DE9F04180460E4617461C4601
:20F78000069DFAF793FF40F6B831884207D2FAF78DFF40490860FAF789FF3F49086028780A
:20F7A000C0F3001000283DD13C48C07A58B9A4F11900B04215DD601D874212DAFAF776FF57
:20F7C000344908600DE0A4F12300B04209DD601D874206DA1938404503DDFAF767FF2D491E
:20F7E0000860FAF763FF2B490968401A41F2883188424CD9FAF75AFF27490860286820F072
:20F800001000103028602648F7F7E6FC0020254908702548008A401C2349088201202349F6
:20F82000087034E01D48C07AB8B9A4F12300B0422DDD0F30B8422ADDFAF738FF1649096840
:20F84000401A1B49884222D9286820F010002860FAF72CFF0F49086019E0A4F12D00B04264
:20F8600015DD1930B84212DD0A3840450FDDFAF71DFF09490968401A0D49884207D92868F7
:20F8800020F010002860FAF711FF02490860BDE8F0810000980200209C020020C405002095
:20F8A0002412002004030020EC08002079010020E09304002DE9F04105460E46144600273F
:20F8C000182E04D0242E05D0302E09D105E047F60C3707E04AF6C87704E04EF2844701E014
:20F8E0002F4600BF00BF2078C0F3800030BBBD4203DCFAF7DBFE1D490860FAF7D7FE1B49BF
:20F900000968401A41F28831884212D9206820F00400001D20601648F7F75EFC002015491E
:20F92000087015488089401C13498881012013490870FAF7BBFE1249086014E0A7F5FA70CC
:20F94000A84203DAFAF7B2FE0D490860FAF7AEFE0B490968401A41F28831884203D92068AB
:20F9600020F004002060BDE8F0810000840200202412002004030020EC080020790100200C
:20F980008802002070B505460E4614462078C0F3C000002848D1012E08D1FAF787FE30495C
:20F9A0000860FAF783FE2F49086014E040F6C410854208DAFAF77AFE29490860FAF776FE3E
:20F9C0002849086007E041F64C50854203DAFAF76DFE24490860FAF769FE21490968401A32
:20F9E000B0F5FA5F08D8FAF761FE1E490968401A40F6B831884232D9206820F008000830DB
:20FA000020601948F7F7E8FB0020184908701848C089401C1649C881012016490870FAF7A5
:20FA200045FE154908601AE0FAF740FE12490968401A41F28831884211D91048007870B9D5
:20FA40000F4800880A280ADA0D4840880A2806DA0C48807818B9206820F00800206070BD18
:20FA60008C020020900200202412002004030020EC0800207901002094020020C60000205F
:20FA800022040020280300202DE9F0470746884615469A46DDE908940026BAF1180F06D002
:20FAA000BAF1240F07D0BAF1300F11D10AE0C9EBC90086B20EE009EB89004FF6FF7101EA1B
:20FAC000400607E009EB890000EBC90086B201E02E4600BF00BF002F48D12078C0F34000EA
:20FAE00058BBB8F1010F05DBB54203DBFAF7DEFD40490860FAF7DAFD3E490968401A41F27B
:20FB00008831884214D9206820F00200801C2060394845808780F7F75FFB00203749087012
:20FB200037484089401C36494881012035490870FAF7BCFD344908605AE0B8F1010F03DB62
:20FB400006F57A70854203DAFAF7B0FD2E490860FAF7ACFD2C490968401A41F2883188420F
:20FB600046D9206820F00200206041E02078C0F3400040BBB54203DBFAF798FD1D4908607C
:20FB8000FAF794FD1B490968401A41F28831884214D9206820F00200801C20601648458038
:20FBA0008780F7F719FB00201449087014484089401C13494881012012490870FAF776FD49
:20FBC0001149086014E006F57A70854203DAFAF76DFD0D490860FAF769FD0B490968401A57
:20FBE00041F28831884203D9206820F002002060BDE8F0877C020020241200200403002022
:20FC0000EC08002079010020800200202DE9F0410746884614460026FAF748FD2B49096897
:20FC2000401A642850D3002507E02949681C31F8100021F81500681C85B2092DF5D324482D
:20FC400047820A21F8F761F906462068C0F3404090BBB8F1320F2BDAB6F57A7F28D91D481C
:20FC60000078322830DD206820F4003000F500302060C6F30F20184948800A211448F8F7AD
:20FC8000B9F8154988800A211148F8F7C4F81249C8800846F7F7A0FA00201049087010485C
:20FCA0000089401C0E49088102200E4908700BE000200849087007E0FFE7B6F57A7F03D86E
:20FCC000206820F400302060BDE8F081A002002068050020A4020020241200200403002030
:20FCE0001C0900207901002010B5FAF7DFFC93490968401AC8287DD3FAF7D8FC8F490860A8
:20FD00008F48008900EBC00101EB00118D48007A64225043B1FBF0F08949888008468088B6
:20FD2000142801DA002001E08548808884498880854840780873854800881C2190FBF1F003
:20FD40007F49C8728248007848738148407888738048007800F0010068B10846C08800EB5D
:20FD6000C00080007C49097B90FBF1F084B22046F4F73CFD01E07948407A7149C8737548C0
:20FD8000007800F0010010B14EF6EE6001E07448C08A6B4908826B48807EEE2816D171481B
:20FDA0008078012824D16F48806844F62061B1FBF0F06D49096808446B4908600846006802
:20FDC0006421B0FBF1F06749C86011E05D48807EAA280DD15C4840685A49897948435949D8
:20FDE000C979B0FBF1F03221B0FBF1F05D49C860544800E0A0E0007B524991F91B10084475
:20FE000042F2107191FBF0F05649C968574A1268891A884206D80120554908705148C06893
:20FE20005249086052480078012838D100205049087050480068401C4E49086008468068B9
:20FE4000401C8860084680684B49884203D9002048498860C8603A48008B401C38490883B8
:20FE6000444800680A21B0FBF1F03549488243480078401C41490870084600781E280EDB39
:20FE80003F4B302269213F4803F079F8394B1022AD213C4803F073F8002038490870284822
:20FEA00000881E281ADB38480078401C3649087008460078052814DB0020087033480088B7
:20FEC000401C324908801E48408B401C1C4948832F480078401C2E49087002E000202A4957
:20FEE00008702B4800783C280BDB00202849087020484068401C1F4948600846C068401CFE
:20FF0000C86022480088B0F5167F0EDB00201F4908801B4B302269211A4803F030F8154B75
:20FF20001022AD21174803F02AF80D48808A0A2190FBF1F00249087510BD0000680000203A
:20FF4000B40700209C0800202803002022040020C600002070010020DC080020340800209A
:20FF6000B402002058030020780000206C000020700000200C0A00209F8601007C00002084
:20FF8000EC080020B403002071000020740000207200002010B50446FAF788FB1049096872
:20FFA000401A4EF66021884218D3FAF77FFB0C4908602068401C20600A480078401C094969
:20FFC0000870084600780A2808DB074B30226921064802F0D4FF00200249087010BD0000DD
:20FFE000B4000020B8000020EC080020B403002001B511480078022800D108BD0098A0B13A
:020000040801F1
:20000000FAF754FB0D490968401AB0F5FA7F10D9FAF74CFB094908606B4641F204120C215F
:200020004FF4E26003F042F803E0FAF73FFB0349086000BFE1E700005D00002080000020A8
:2000400010B50446012C13D1FAF730FB0B490968401AC82810D30A4B4FF481520C214FF497
:20006000E26003F023F8FAF721FB0449086003E0FAF71CFB0149086010BD00008400002060
:20008000B407002010B5FCF763F8FCF74FF8F4F7BFFF03F0A3F9FCF727FB0A4801890A48BD
:2000A00004F068F807484189084804F063F805488189074804F05EF80248018A0548F7F734
:2000C000FBFD10BD08160020F01200200A13002024130020FC0300201CB50446FAF7E6FA5C
:2000E00040490968401AB0F5FA7F7AD33E480088401C3D49088008460088142837DB3B4822
:20010000007800F0010010B900203949487437480088C0F3002010B9002035490874334817
:200120000078C0F3801010B90020314908812F480078C0F3C01010B900202D4948812B480B
:200140000078C0F3001010B900202949888127480078C0F3401010B900202549C8814FF433
:2001600080512448FAF798FA00201F4908802248007868B900204FF408430C2240F2FF712E
:2001800000901E4802F0DEFF01201B49087024E019480078012820D100200190184801781C
:2001A0000078401C164A107005290CDC01A841F20133162240F2FF710090104802F0C2FFF0
:2001C0000A20F9F7D9FE41F214030C2240F2FF710A48009402F0B6FF00BFFAF767FA01492C
:2001E00008601CBD900000209400002082010020BC090020001001405D000020F4040020EC
:200200009600002070B504464D48007880BB08214C48FAF739FA4C4908704FF400414B486C
:20022000FAF732FA4A49087080214A48FAF72CFA494908704FF480714648FAF725FA4749E0
:2002400008704FF400514348FAF71EFA4449087004214448FAF718FA434908700020208180
:200260006081A081E081207460740120344908703E48C08860803D488088A0804FF400609F
:20028000E0803A480089208008212E48FAF7FCF905462D480078A84202D02089401C208134
:2002A000294805704FF400412848FAF7EDF9054627480078A84202D06089401C608124480D
:2002C000057080212348FAF7DFF9054622480078A84202D0A089401CA0811F4805704FF426
:2002E00080711C48FAF7D0F905461C480078A84202D0E089401CE081184805704FF400517D
:200300001448FAF7C1F9054615480078A84202D0207C401C20741248057004211148FAF730
:20032000B3F9054610480078A84202D0607C401C60740D4805704FF47A70608270BD000028
:200340008E000020000C0140880000200008014089000020001001408A0000208B00002062
:200360008C000020001401408D0000201E16002010B5FAF79BF942F21071884204D2FAF7EB
:2003800095F94149086010BDFAF790F93E490968401A41F28831884274D3FAF787F93A4953
:2003A00008603A48407D3A4991F82310884207DA3648407D364981F8230000203549087040
:2003C0003248407D324991F82210884207DD2F48407D2F4981F8220000202E4908702B4839
:2003E000807D2B4991F82910884207DA2748807D274981F829000020264908702348807D32
:20040000234991F82810884207DD2048807D204981F8280000201F4908701C48C07D1C498C
:2004200091F82B10884207DA1848C07D184981F82B000020174908701448C07D144991F834
:200440002A10884207DD1148C07D114981F82A0000201049087010480088401C0E49088015
:20046000084600880C280DDD0A48007850B900200880012007490870054B302269210748A9
:2004800002F07DFD00BF7EE7BC000020B4070020EC080020C2000020C0000020B403002068
:2004A00010B50748007850B9FAF700F904494968401AB0F5FA6F02D901200149087010BDCC
:2004C0009001002000B587B0012003900320049003A90E48F9F74AFF0D480068806820F024
:2004E00001000B4909688860002000900A2001900720029069460648F7F7BCFF20B140F281
:20050000253104A004F03AFD07B000BD00080140341600202E2E5C436F72655C5372635C6E
:200520006164632E630000000EB55F485F49086081155E4881600021C16041614FF46021C3
:20054000C1610020594948600B2158480161F8F723FC18B1592156A004F010FD0A200090DF
:20056000012001900720029069465048F7F782FF18B163214EA004F001FD0B200090022050
:2005800001900720029069464848F7F773FF18B16D2147A004F0F2FC0C20009003200190E2
:2005A0000720029069464148F7F764FF18B177213FA004F0E3FC0D20009004200190012053
:2005C000029069463948F7F755FF18B1812138A004F0D4FC05200090019001200290694668
:2005E0003248F7F747FF18B18B2131A004F0C6FC04200090062001900120029069462B4811
:20060000F7F738FF18B1952129A004F0B7FC0F200090072001900120029069462348F7F794
:2006200029FF18B19F2122A004F0A8FC07200090082001900720029069461C48F7F71AFF6C
:2006400018B1A9211AA004F099FC0E200090092001900120029069461448F7F70BFF18B1CD
:20066000B32113A004F08AFC102000900A2001900220029069460D48F7F7FCFE18B1BD21B7
:200680000BA004F07BFC112000900B2001900720029069460548F7F7EDFE18B1C72104A0E4
:2006A00004F06CFC0EBD000000240140341600202E2E5C436F72655C5372635C6164632ECD
:2006C0006300000000B589B02348244908608115224881600021C1604161C16100201F491A
:2006E000486001211D480161F8F756FB18B1DB211BA004F043FC012001900290032005907A
:20070000002003904FF480500890002007900690049001A91148F7F7A3FC18B1EA2110A086
:2007200004F02CFC02200190029001A90B48F7F797FC18B1F3210AA004F020FC032001908F
:20074000029001A90548F7F78BFC18B1FC2104A004F014FC09B000BD002801406416002094
:200760002E2E5C436F72655C5372635C6164632E6300000010B50F480F49086030204860CB
:2007800000210D488160C1604FF4403101610021416181610121C1610021016241628162D8
:2007A000C162F8F739FF18B1542104A004F0E6FB10BD0000006400404C1B00202E2E5C4345
:2007C0006F72655C5372635C63616E2E6300000008B500BF0A48406940F00100084948618E
:2007E0000846406900F00100009000BF00BF022211460B20FAF729F80B20FAF719F808BD59
:200800000010024000B585B000BF3A48806940F01000384988610846806900F01000009001
:2008200000BF00BF00BF0846806940F0200088610846806900F02000009000BF00BF00BFF7
:200840000846806940F0040088610846806900F00400009000BF00BF00BF0846806940F0E5
:20086000080088610846806900F00800009000BF00BF002289142048F9F712FF4FF463403C
:2008800001900320029001A91B48F9F76FFD40F6087001900320029001A91848F9F766FD58
:2008A0004EF6024001900320029001A91448F9F75DFD4FF4805001901248029000200390D9
:2008C00001A90F48F9F752FD4FF480500190012002900220049001A90748F9F747FD00227C
:2008E00011462820F9F7B1FF2820F9F7A1FF05B000BD000000100240001001400008014083
:20090000000C01400000211010B50848084908600320486040F2E24105488160F9F7CCFE83
:2009200018B13A2103A004F029FB10BD00300040E80500202E2E5C436F72655C5372635C6D
:20094000697764672E63000000B595B03148324908600020486020212F4881604FF41661EA
:20096000C1600021016101214161FAF747FE4FF48050119011A92848FAF7E8FE2648FBF7C4
:2009800019F970200F90802010900FA92248FAF7BEFD4FF4006008904010099000200A902A
:2009A00039200B9000200C900D900E9008A91A48FAF76EFD6FF08000174909680861602044
:2009C00001904FF496600290002003900490059006900790002201A90F48FBF767F8042218
:2009E00001A90D48FBF762F8082201A90A48FBF75DF86020019040F65F1002900020039044
:200A0000082004900C2201A90348FBF74FF815B000BD0000002C01404815002000B587B066
:200A200000200390049005900690019002904FF08040194908600020486000211648816030
:200A40004FF6FF71C1600021016141618161FAF7D5FD18B17E2111A004F090FA4FF40050CC
:200A60000390002004900590069003A90A48FAF76DFE18B1862109A004F080FA0020019072
:200A8000029001A90448FAF742FD18B18C2103A004F074FA07B000BD881500202E2E5C55E5
:200AA0007365725C5372635C74696D2E6300000000B589B01C481D49086000204860002128
:200AC0001A4881604721C1600021016180218161FBF770F820B14FF48F7115A004F04EFAE5
:200AE00000200790089007A91048FAF710FD20B140F225110EA004F041FA60200090242037
:200B00000190002002900490002269460748FAF7CDFF20B14FF4977105A004F02FFA0348F8
:200B2000FAF77AFF09B000BD00040040C81500202E2E5C557365725C5372635C74696D2EE5
:200B40006300000010B50C480C4908604FF416504860002109488160C16001610C21416166
:200B600000218161C161FBF741FA18B1462104A004F004FA10BD000000480040901D00203B
:200B80002E2E5C436F72655C5372635C75736172742E630000BFFEE730B504460A46002130
:200BA000002329480078401C274D2870284600780F2841DB0020287024480089244D2D88B5
:200BC000411B002907DA214800894FF6FF7528441F4D2D88411B44F62060814200DD0021A0
:200BE0001A4800891A4D28804FF47A70414319480068081A174D2D6805EB2020154D28604C
:200C0000284600680314C3EB031040F35C0000B2114D28800D488089104D2D68C5EB80203F
:200C20000E4D2D6805EB60100C4D286028460068C0F38F20054DE88112B90020064D2880AA
:200C40000548B0F9000030BD16030020C4050020180300201C03002024030020200300208B
:200C60002DE9F04107460C46154629462046F7F741F88046002606E0701C34F8100024F881
:200C80001600701C86B2681EB042F5DC24F810704046BDE8F081704702480068C0F30220BB
:200CA000704700000CED00E010B5002807DA0A07140E054A00F00F031B1FD45403E00A07FC
:200CC000130E024A135410BD18ED00E000E400E010B5F9F7EBFC40F6B831884216D90C4802
:200CE0000078012812D10020094908700948C07AAA280BD133200849087008460078C04368
:200D00000649087004484078C043487010BD0000C30000209C080020C6000020C80000200B
:200D200010B50446012C06D0022C23D0032C40D0042C7DD15CE024224E494F48F2F7AFFE7D
:200D400024224E494E48F2F7AAFE24224D494E48F2F7A5FE24224D494D48F2F7A0FE242253
:200D60004C494D48F2F79BFE24224C494C48F2F796FE7CE024224B493F48F2F790FE242261
:200D800049493F48F2F78BFE242248493E48F2F786FE242246493E48F2F781FE2422454967
:200DA0003D48F2F77CFE242243493D48F2F777FE5DE0242241493048F2F771FE24224049EA
:200DC0002F48F2F76CFE24223E492F48F2F767FE24223D492E48F2F762FE24223B492E48EC
:200DE000F2F75DFE24223A492D48F2F758FE3EE0242238492048F2F752FE2422364920487F
:200E0000F2F74DFE242235491F48F2F748FE242233491F48F2F743FE242232491E48F2F7E1
:200E20003EFE242230491E48F2F739FE1FE0FFE7242210491048F2F732FE24220F49104846
:200E4000F2F72DFE24220F490F48F2F728FE24220E490F48F2F723FE24220E490E48F2F7A0
:200E60001EFE24220D490E48F2F719FE00BF00BF10BD0000F8580108140600201C59010808
:200E800038060020405901085C060020645901088006002088590108A4060020AC590108A2
:200EA000C8060020D0590108F4590108185A01083C5A0108605A0108845A0108A85A0108ED
:200EC000CC5A0108F05A0108145B0108385B01085C5B0108805B0108A45B0108C85B0108A4
:200EE000EC5B0108105C0108345C01082DE9F04304460D46601B06B2B2F9000000FB06FCD3
:200F0000908810B90020106212E0B2F9040000FB06F7106AC319D069984202DAD0691062D5
:200F200006E09069984202DD9069106200E0136250889CFBF0F0B2F80690D2F8208098FBCD
:200F4000F9F800EB0801002906DA1069884203DD108A00B2BDE8F083002905DD506988428E
:200F600002DC908A00B2F5E708B2F3E72DE9F34F83B00C46204603F043F900901D48009957
:200F80000160BDF90C001B49B1F9001000FB01F7FF13BDF90E001749B1F9021000FB01F837
:200FA0004FEAE8380FFA87FB0FFA88F001900198ABEB000000B2ADF80800BDF90C000D4995
:200FC000B1F9021000FB01F5ED13BDF90E000949B1F9001000FB01F6F6130FFA85F90FFA09
:200FE00086FA09EB0A0000B2ADF80A00029805B0BDE8F08F4C0000207047000030B502464F
:20100000B2F900303F4CB4F90040A34202DD13883C4C2380B2F902303B4CB4F90040A342BD
:2010200002DD5388384C2380B2F90430374CB4F90040A34202DD9388344C2380344B1B885C
:201040005B1C1BB2324C23802346B3F90030B3F5FA7F56DB2B4BB3F900000023294C238037
:20106000031E01DB1C4600E05C42B5256C43294D2D68C5EB8404274D2D6805EB6414254DE4
:201080002C602B461B689B121BB20B801E4BB3F9000000231C4C2380031E01DB1C4600E049
:2010A0005C42B5256C431C4D2D68C5EB84041A4D2D6805EB6414184D2C602B461B689B12DD
:2010C0001BB24B80114BB3F9000000230F4C2380031E01DB1C4600E05C42B5256C430F4D8D
:2010E0002D68C5EB84040D4D2D6805EB64140B4D2C602B461B689B121BB28B800023044CFC
:20110000238030BD70040020720400207404002076040020780400207C0400208004002003
:2011200000B585B000BF1148806940F004000F4988610846806900F00400009000BF00BF16
:20114000002289140A48F9F7ABFA4FF480500190012002900220049001A90548F9F706F9F6
:2011600000200449087005B000BD00000010024000080140FA03002010B50446012C0BD148
:201180000C480078A8B9012211030B48F9F788FA0120084908700CE05CB90648007801284C
:2011A00007D1002201030448F9F77AFA00200149087010BDFA0300200008014010B504465D
:2011C00019480078012816D1B4F5D16F0FDB17480088401C80B21549088047F23051884274
:2011E00020DD0020114908800F4908701AE000200E49088016E0B4F5BC6F10DA0C48008897
:20120000401C80B20A4908803C280BDDF5F798FC01200549087000200649087002E00020C9
:201220000349088010BD0000880400208404002086040020BF01002038B50446002031495E
:201240000870F020487008460078C0432E4908702C484078C04348702A4840782B4B00907F
:20126000DA79997958792A4B1B78FBF779FB29480078E0B928480068284908602648406881
:2012800048602548806888602348C068C8602448406808612822234801F010FE042222A194
:2012A0002048083801F00AFE01201A49087020A341F205320C214FF4E26001F0F7FE04B90F
:2012C00038BDF9F7F3F91C49086000201B49087012E0F9F7EBF918490968401A64280BD912
:2012E000F9F7E4F91449086014480078401C134908701348F9F708FA104800780A28E8DB46
:2013000000BFDDE7C6000020C8000020BC080020C4030020AA0000200C0A00207C0900200C
:20132000EC08002008E80108464C4147000000005245414459000000AC000020B000002075
:20134000E805002010B50248FAF7F1F910BD00004815002010B500210B48FAF77FFC042182
:201360000948FAF77BFC08210748FAF777FC00210548FAF713F904210348FAF70FF90821DB
:201380000148FAF70BF910BD4815002008B508490968C9084FF47A72B1FBF2F141430091A2
:2013A00000BF00BF00994A1E00920029F9D108BD000000202DE9F04705460E46174698461D
:2013C000F9F774F984490968401A052801D2BDE8F087F9F76BF9804908600FFA88F07F492E
:2013E00048807F480088281AC8810846007801287ED1F9F75BF97949C969401AB0F5FA6F6D
:2014000006D9F9F753F97549C8610120887601E0744886607148407E01281BD100206F49C4
:201420004876002405E000206F4921F81400601CC4B2192CF7DB00206C4908806C4908605D
:201440006C4908706548408A20B16448408A0002694908606148C0890A2849DB6048056030
:201460005E48807E00286FD15E4886600774C068002869D05B4880895A490989401A00B2E3
:201480005E4908800846B0F90000002803DD0846B0F9000000E00020584908800846B0F907
:2014A00000001E2803DA0846B0F9000000E01E20524908800846008818B94A48007C642890
:2014C00042D049484949098830F8110048490968081A47490860084600684849B1F90010F0
:2014E0000844434908604548008881B23F4800E06FE002880088401C3C4B18803A4820F887
:20150000121018460088192807DB002019460880012038490870314908763548006840B3AF
:2015200034480078012810D1314800684FF47A7148436421484329498989FA225143B0FB24
:20154000F1F02649088217E03FE02848008800EB80004100214880894143254800684FF4E9
:201560007A72504364225043B0FBF1F01B49088202E00020194908821C480088A0B91748C7
:20158000B0F810901C480068C0EB09201E2190FBF1F019490968084417490860084600681B
:2015A000C0F30F200D4948820C48408A002808DD0C4880680949898AB0FBF1F00749C88237
:2015C00003E04FF6FF700549C882064880680549C86000BFFBE60000E4020020B4020020B4
:2015E000E80200207C05002090050020D4020020D8020020DC020020E0020020DE0200209B
:201600002DE9F04104460D4617469846069E002013490860886043F2C82048600020C8602E
:201620000DB90846866000200E49087048800520888000208860084684810020C88108827E
:2016400048824FF6FF70C88200200876487601208876F9F72BF80349C861BDE8F0810000A9
:201660007C050020B40200202DE9F04106460F4606F00F0000287DD0052FFCD001206F49B8
:2016800008700846007E012864D1002008760846408A6B49098888425CD06848408A002815
:2016A00054D06648408A67490988401A642100FB01F56448008895FBF0F004B214F11E0FF1
:2016C00044DBB4F5E47F41DA04F164005D4909884843642190FBF1F0584988825A480588DE
:2016E00004F164006843642190FBF1F0574908805548458804F164006843642190FBF1F06E
:20170000524948805048858804F164006843642190FBF1F04D4988804B48C58804F16400F5
:201720006843642190FBF1F04849C8804648058904F164006843642190FBF1F0434908810E
:201740000B461022CD21424801F019FC3B48408A3B4908803F480078864203D13E48007896
:20176000874265D0032E1DD005DC012E08D0022E33D10EE054E0042E1DD0332E2DD123E08E
:20178000324800882D4948822F4800882D49088029E02E484088294948822B4840882949DA
:2017A000088020E02948808824494882264880882449088017E02548C0882049488222483D
:2017C000C088204908800EE0204800891B4948821D4800891B49088005E0002017494882BA
:2017E0001849088000BF00BF1448408A144908801248408A114988820846408A002807DDCB
:2018000016488068898AB0FBF1F00C49C88203E04FF6FF700949C88201200849487607E0FA
:20182000002006490870488288824FF6FF70C8820848067008480770BDE8F081B402002076
:20184000EE020020F0020020B05F01081C0A0020B4030020EC020020ED0200207C05002073
:201860002DE9F043A1B0064688461546AD10002423E056F8240011A941F8240011A850F8EB
:201880002400000E01AA02F8240011A850F82400C0F30741A000401C115411A830F82400C7
:2018A000C0F30721A000801C115411A810F82410A000C01C1154601CC4B2AC42D9DB56F8F4
:2018C0002590A10001A8F3F787FB0746B9EB070008D1AA0001A94046F2F7E1F8002021B03F
:2018E000BDE8F0834FF0FF30F9E7000010B5B0F900205243B0F9023003FB03210C4A914239
:2019000014D909163939CBB20A4C34F81320B0F9003003FB02F1CB131BB20380B0F9023044
:2019200003FB02F1CB131BB2438000BF10BD0000400AC139585C01082DE9F14181B0BDF98C
:201940000400DFF86880B8F9008000FB08F1C913BDF90600DFF85480B8F9028000FB08F234
:20196000D2130EB217B2F01900B2ADF80000BDF90400DFF83880B8F9028000FB08F3DB1339
:20198000BDF90600DFF82480B8F9008000FB08F4E4130FFA83FC25B2CCF10000284400B2B7
:2019A000ADF802000098BDE8FC8100004C00002010B504462078012808D10B4B302269217F
:2019C0000A4801F0DCFA002020700AE02078022807D1074B10229B21044801F0D0FA002053
:2019E0002070002010BD0000EC080020B40300201C0900204FF055301F4A106040001F4AF4
:201A000010601D480168B1F1553F01D0002070471A480168B1F1AA3F01D00020F7E74FF046
:201A2000AA30154A10604008144A106012480168B1F1AA3F01D00020E9E710480168B1F175
:201A4000553F01D00020E2E74FF055300A4A106040000A4A106008480168B1F1553F01D0EC
:201A60000020D4E705480168B1F1AA3F01D00020CDE70120CBE70000000600201006002076
:201A800001200C490968B1F1EE3F00D0002009494968B1F1CC3F00D0002006498968B1F11E
:201AA000BB3F00D000200349C968B1F1DD3F00D0002070471822002010B5214800780D2825
:201AC0002FD2DFE800F0070A0D101316191C1F2225282B00F1F772FB24E0F1F7A3FB21E029
:201AE000F1F7DFFB1EE0F1F721FC1BE0F1F764FC18E0F1F7A8FC15E0F1F7ECFC12E0F1F7BB
:201B000030FD0FE0F1F775FD0CE0F1F7BBFD09E0F1F7FCFD06E0F1F73DFE03E0F1F77EFEA9
:201B200000E000BF00BF06480078401C04490870084600780C2801DD0020087010BD000023
:201B40000405002010B5F1F739FBF1F76BFBF1F7A8FBF1F7EBFBF1F72FFCF1F774FCF1F781
:201B6000B9FCF1F7FEFCF1F744FDF1F78BFDF1F7CDFDF1F70FFEF1F751FE10BD10B53B4842
:201B80000068B0F1AA3F70D138480068384909684840401C002866D136490860C04336498C
:201BA000086034480068801C32490860FFF784FF31480068801E304908602E4800680D3066
:201BC0002C490860FFF75CFF08B9F5F71BFF2A4800680D3828490860264800680B30254999
:201BE000086000F0C5FC044634B1012C0AD0032C04D0042C05D100E007E006E0F5F702FFF3
:201C000003E000BFF5F7FEFE00BF00BF1A4800680B381949086017480068C01C154908607C
:201C200000F044F808B9F5F7EDFE13480068C01E114908600F480068401D0E490860FFF7AC
:201C4000D9FE08B9F5F7DEFE0B480068401F0A490860222003F032FB08B9F5F7D3FE00204F
:201C60000249086001E0F5F7CDFE10BDE01D0020041E0020D01D0020F41D002010B500F0FA
:201C800047FC00F055FC00F001F810BD4FF0EE30054908604FF0CC3048604FF0BB30886002
:201CA0004010C8607047000018220020F0B55527552F01D00020F0BDAA27AA2F01D00020BD
:201CC000F9E74FF05531B1F1553F01D00020F2E74FF0AA31B1F1AA3F01D00020EBE74FF4B4
:201CE0007A714A008C1840F6B830844201D00020E1E74FF0FF3102228C18012C01D0002019
:201D0000D9E74FF47A73F94D5E1916F57A7F01D00020D0E76FF0004301255E19B6F1004F35
:201D200001D00020C7E76FF0004302255E19981C864201D00020BEE76FF0004303255E1971
:201D4000D81C864201D00020B5E74FF4FA614A108C1AB4F57A7F01D00020ACE74FF4FA61D8
:201D60004A1C8C1A601C08B10020A4E7002101228C1A601C08B100209DE74FF47A735D0027
:201D80005E1B16F57A7F01D0002094E7002301255E1B701C08B100208DE74FF00043012517
:201DA0005E1B581E864201D0002084E74FF47A71491C0846814201D000207CE74FF0FF31A9
:201DC000491C09B1002076E70021491C012901D0002070E74FF47A735B1C1846834201D0D4
:201DE000002068E700235B1C012B01D0002062E76FF000435B1CB3F1004F01D000205AE736
:201E00004FF000435B1C1846834201D0002052E74FF47A71491E0846814201D000204AE7B4
:201E20000021491E481C00B145E74FF0FF31491E881C00B13FE74FF47A735B1E18468342BC
:201E400001D0002037E74FF000435B1E1846834201D000202FE76FF000435B1E1846834210
:201E600001D0002027E700235B1E581C00B122E764210A2201FB02F4B4F57A7F01D0002063
:201E800019E76FF07041112201FB02F49848844201D000200FE74FF0FF31012201FB02F4FC
:201EA000601C08B1002006E76421002201FB02F40CB10020FFE64FF47A710A22B1FBF2F499
:201EC000642C01D00020F6E601210A22B1FBF2F40CB10020EFE600210A22B1FBF2F40CB177
:201EE0000020E8E64FF47A710022B1FBF2F40CB10020E0E64FF0FF310122B1FBF2F4601CCF
:201F000008B10020D7E602214C00042C01D00020D1E602210C02B4F5007F01D00020CAE6EA
:201F20000221CC070CB10020C5E64FF6FF714C084810844201D00020BDE64FF6FF710C0A9D
:201F4000FF2C01D00020B6E64FF6FF71CC0F0CB10020B0E6012109B90020ACE6002109B155
:201F60000020A8E6FF2109B90020A4E664210A22914201D800209EE664216422914201D96E
:201F8000002098E60A216422914201D9002092E64FF0FF310022914201D800208BE66FF080
:201FA0000043DD07AB4201DC002084E60A216422914201D300207EE664216422914201D219
:201FC000002078E664210A22914201D2002072E600214A1E914201D300206CE64FF0004390
:201FE0005D1EAB4201DB002065E664210A22914201D200205FE664216422914201D20020A5
:2020000059E60A216422914201D3002053E64FF0FF310022914201D200204CE66FF00043A5
:20202000DD07AB4201DA002045E60A216422914201D900203FE664216422914201D900202E
:2020400039E664210A22914201D8002033E600214A1E914201D900202DE64FF000435D1E65
:20206000AB4201DD002026E664216422914201D0002020E64FF0FF310A46914201D0002011
:2020800019E600210022914201D0002013E64FF000431D46AB4201D000200CE60023002544
:2020A000AB4201D0002006E66FF000431D46AB4201D00020FFE564216422914201D00020C0
:2020C000F9E54FF0FF310A46914201D00020F2E500210022914201D00020ECE54FF000436E
:2020E0001D46AB4206D00020E5E5000030F8FFFFEFFFFF0F00230025AB4201D00020DAE5C9
:202100006FF000431D46AB4201D00020D3E50121002221B9022904D0032906D103E0921C73
:2021200004E0121D02E0083200E000BF00BF022A01D00020BFE502210022012904D00229E3
:2021400004D0032906D103E0921C04E0121D02E0083200E000BF00BF042A01D00020AAE5DC
:2021600003210022012904D0022904D0032906D103E0921C04E0121D02E0083200E000BFBA
:2021800000BF082A01D0002095E504210022012904D0022904D0032906D103E0921C04E027
:2021A000121D02E0083200E000BF00BF0AB1002081E50021002211B10AB100207BE501B93B
:2021C0000AB1002077E50021012211B10AB1002071E511B90AB900206DE50121012201B19B
:2021E0000AB9002067E511B90AB9002063E50121FF2201B10AB900205DE511B90AB90020F4
:2022000059E50021FF2211B10AB1002053E511B90AB900204FE54FF055310A4681EA020402
:202220000CB1002047E54FF055314A0081EA0204601C08B100203EE50021002281EA0204E9
:202240000CB1002037E54FF0FF310A4681EA02040CB100202FE500214A1E81EA0204601CEE
:2022600008B1002027E54FF05531CC43B4F1AA3F01D000201FE5E443B4F1553F01D00020D1
:2022800019E50021CC43601C08B1002013E5E4430CB100200FE501200DE5000008B500BF3C
:2022A0007148806940F004006F4988610846806900F00400009000BF00BF00BF0846806978
:2022C00040F0080088610846806900F00800009000BF00BF00BF0846806940F01000886181
:2022E0000846806900F01000009000BF00BF00BF0846806940F0200088610846806900F043
:202300002000009000BF00BF5848F5F7E7FB08B9002008BD5648F5F7E1FB08B90020F8E755
:202320005448F5F7DBFB08B90020F2E75248F5F7D5FB08B90020ECE74B48806920F00400EB
:20234000494988610846806920F0080088610846806920F0100088610846806920F0200023
:2023600088614648F2F7B0F900BF3F48C06940F000703D49C8610846C06900F0007000902F
:2023800000BF00BF3E48F2F7E1FD08B90020C0E73548C06920F000703349C86100BF084612
:2023A000406940F0010048610846406900F00100009000BF00BF3348F3F706FB08B900205D
:2023C000A7E72948406920F001002749486100BF0846806940F4007088610846806900F47D
:2023E0000070009000BF00BF00BF0846806940F4806088610846806900F48060009000BF12
:2024000000BF2148F2F778F808B9002081E71F48F2F772F808B900207BE71348806920F49D
:202420000070114988610846806920F48060886100BF0846806940F400608861084680692B
:2024400000F40060009000BF00BF114801F08BFB08B900205DE70448806920F40060024931
:202460008861012055E700000010024000080140000C014000100140001401400000014047
:2024800000640040080002400024014000280140002C014010B5002419480068194909688E
:2024A0004840401C48BB164800681749884210D316490846F1F7EAF9012801D1042400E0E7
:2024C000032411484B380E490860C0430D49086014E00E490A480068F1F7D8F901280AD1B7
:2024E0000748006810300649086008460068C0430449086002E0032400E00124204610BD7F
:20250000380500203C0500207B0000201805002004480549086008460068C04303490860B6
:202520007047000030000020380500203C05002010B50A480A490860C0430A4908600A48F4
:202540000A4908600846F7F742FB08480068806840F0010005490968886010BD00300008CA
:20256000EC1D0020101E0020003002400C05002010B502241F4800681F4909684840401CCA
:20258000002834D11B4800681C49884223D2002006E01849096851F82010194A1160401C9E
:2025A00018498908174A9209B1FBF2F18142F0D814498908134A9209B1FBF2F10D4A1268CD
:2025C00002EB81010B4A116011460968C9430A4A116000240CE00A480068084909688842D7
:2025E00001D1042400E00324FFF7A2FF00E00124204610BDEC1D0020101E00208083010888
:20260000003002408053010070B50A2050490870F8F78EF800F0E4FF00204E490860C043AA
:202620004D4908604B480068801C4A490860FFF789FA49480068801E47490860F0F772FDAC
:202640000C2043490870434800680B304149086042484349086008460068806840F00100DD
:20266000096888603E48F7F7B2FA002405E03D4951F8240039490860641C3B48B4EB900FBA
:20268000F5D33648056839480068854201D0F5F7B9F9314800680B382F4908600E202C49C1
:2026A00008702C480068C01C2A490860FFF7FEFA08B9F5F7A7F928480068C01E2649086047
:2026C00010202349087023480068401D21490860FFF790F908B9F5F795F91F480068401FFC
:2026E0001D49086012201A4908701A480068C01D18490860FFF7D2FD08B9F5F783F914206D
:2027000013490870FFF7CAFD08B9F5F77BF912480068C01F1049086016200D4908701C2065
:2027200002F0CCFD08B9F5F76DF91820084908704FF400510804F1F722F908B9F5F762F91F
:2027400000F0B8FFAA2005490871F0F7CFFC70BD08050020D01D0020F41D00200030024085
:202760000C05002000300008805301008083010810B5124800780A281EDB00200F4908705E
:202780004FF0AA300E49086040080E49086072B6FFF780FE044662B634B1012C08D0032C43
:2027A00005D0042C02D100E005E004E000BF00BFF5F728F900BF00BF10BD00005900002049
:2027C000E01D0020041E0020002107E041F64C5100BF0A00A1F1010399B2FAD10200A0F1B6
:2027E000010398B2F2D17047002106E0072100BF0A00A1F1010399B2FAD10200A0F10103D6
:2028000098B2F3D1704770472DE9F143BDF9000044F2F30100FB01F9BDF902004FF41651BB
:202820004843C0F10008444608EB09004710A8EB09004610002F0FDA002E03DA0520F749FD
:20284000088018E0002C03DC0420F449088012E00320F24908800EE0002E03DB0220EF49D8
:20286000088008E0002C03DC0620EC49088002E00120EA4908800020E9490870E7480088BB
:2028800007287BD2DFE800F07A044D97E0FCFB0004F51650801B4FF4966101EBA040E149A2
:2028A00008800846008800EB6640488008464088A0EB6440888008460088C0F5166080B2E1
:2028C000E22803DD40F65F10C88029E0D5480088D4494988401A85B2B5F58B7F05DBD14847
:2028E00000883338CF49C8801AE0CE480088C0F5166080B28A2813DDCA480088E230C94930
:20290000C8800846C088B0F5166F09DB0120C4490870C448C088C0F59650401EC149C88086
:2029200074E107F51650801B4FF4966101EBA040BC4908800846008800EB66404880084635
:202940000088A0EB6740888008464088C0F5166080B2E22803DD40F65F10C8802AE0B14868
:202960004088B0490988401A85B2B5F58B7F06DBAC4840883338AB49C8801BE045E1A9486A
:202980004088C0F5166080B28A2813DDA5484088E230A449C8800846C088B0F5166F09DBD0
:2029A00001209F4908709F48C088C0F59650401E9C49C8802AE1C4F5165038444FF4966161
:2029C00001EBA0409749088008460088A0EB674088800846808800EB6440488008464088F0
:2029E000C0F5166080B2E22803DD40F65F10C88029E08C4840888B498988401A85B2B5F5DE
:202A00008B7F05DB8748408833388649C8801AE084484088C0F5166080B28A2813DD81485D
:202A20004088E2307F49C8800846C088B0F5166F09DB01207A4908707A48C088C0F5965007
:202A4000401E7849C880E1E004F51650801B4FF4966101EBA040734908800846008800EB49
:202A60006640488008464088A0EB6440888008468088C0F5166080B2E22806DD01E078E0C2
:202A80002EE040F65F10C88029E06648808865494988401A85B2B5F58B7F05DB6148808827
:202AA00033386049C8801AE05E488088C0F5166080B28A2813DD5B488088E2305949C8806C
:202AC0000846C088B0F5166F09DB0120544908705448C088C0F59650401E5249C88095E0E7
:202AE00007F51650801B4FF4966101EBA0404D4908800846008800EB6640488008460088B0
:202B0000A0EB6740888008468088C0F5166080B2E22803DD40F65F10C88029E04148808857
:202B200040490988401A85B2B5F58B7F05DB3D48808833383B49C8801AE03A488088C0F559
:202B4000166080B28A2813DD36488088E2303549C8800846C088B0F5166F09DB012030498F
:202B600008703048C088C0F59650401E2D49C8804CE0C4F5165038444FF4966101EBA04099
:202B80002849088008460088A0EB674088800846808800EB6440488040F65F10C880084644
:202BA0000088C0F5166080B2E22803DD40F65F10C88029E01B4800881A498988401A85B260
:202BC000B5F58B7F05DB1748008833381549C8801AE014480088C0F5166080B28A2813DD8C
:202BE00010480088E2300F49C8800846C088B0F5166F09DB01200A4908700A48C088C0F564
:202C00009650401E0749C88000E000BF00BF0448007848B9002000F005FB08E03400002069
:202C20003600002038000020022000F0FBFA40F64C100949C880088800F0DCFA064948883E
:202C400000F0DEFA0449888800F0E0FA0249C88800F0E2FABDE8F883380000202DE9F0415F
:202C60000446002500260027F3F7AAFFA84618E000BF334800780128FBD100203049087067
:202C80003048008805442F48408806442D48808807440C212C48F8F7C1FF08F101001FFA37
:202CA00080F8B8F10A0FE3DB0A20B5FBF0F0274908800A20B6FBF0F048800A20B7FBF0F02B
:202CC00088800846008846F2A81188421DDB1F48008849F64041884217DC1C48408846F293
:202CE000A811884211DB1948408849F6404188420BDC1648808846F2A811884205DB13486F
:202D0000808849F64041884216DD206820F4802000F58020206006200D4948800846F4F760
:202D20005BFA00200B4908700B484089401C0A494881022009490870F3F742FFBDE8F08191
:202D40002004002014040020481500202604002024120020040300201C09002079010020D4
:202D600008B50020009053480088072870D2DFE800F0933362630405320000BF4E480088F8
:202D8000404201B211F5004F04DA4FF40040ADF8000009E0B1F5004F04DB47F6FF70ADF895
:202DA000000001E0ADF8001043484088404201B211F5004F04DA4FF40040ADF8020009E0AF
:202DC000B1F5004F04DB47F6FF70ADF8020001E0ADF8021061E000BF37484088404201B2B8
:202DE00011F5004F04DA4FF40040ADF8020009E0B1F5004F04DB47F6FF70ADF8020001E085
:202E0000ADF802102C488088BDF80220801A01B2B1F5004F04DB47F6FF70ADF8000009E04D
:202E200011F5004F04DA4FF40040ADF8000001E0ADF8001031E000BF1F480088404201B2AD
:202E4000B1F5004F05DB47F6FF70ADF800000AE022E011F5004F04DA4FF40040ADF8000005
:202E600001E0ADF8001014488088BDF80020801A01B211F5004F04DA4FF40040ADF80200D9
:202E800009E0B1F5004F04DB47F6FF70ADF8020001E0ADF8021000E000BF00BFBDF9000076
:202EA0000011ADF80000BDF902000011ADF80200009808BD340000202C0400202DE9F043A2
:202EC000C1B081460D4616463046F11706EB9171C1F38707002414E015F824000106A00068
:202EE000401C285C01EB0041A000801C285C01EB0021A000C01C285C08444DF82400601CC7
:202F0000C4B2BC42E8DB31462846F2F765F880464DF827807A1C69464846F4F7E7FB41B00C
:202F2000BDE8F0832DE9F04190B080460D4616463046F11706EB9171C1F38707002414E0B2
:202F4000A000C01C285C0106A000801C285C01EB0041A000401C285C01EB002015F82410B0
:202F600008444DF82400601CC4B2BC42E8DB3A4669464046F4F7BAFB10B0BDE8F0812DE9A8
:202F8000F84381460D4616461F46002000908046002420E02819C1B26A464846F3F768FF3E
:202FA000401C18B94FF0FF30BDE8F883385D9DF8001088420DD0385D00902819C1B29DF807
:202FC00000204846F3F7AAFF401C10B94FF0FF30EAE7601CC4B2B442DCDB31463846F1F7D0
:202FE000E3FF80464FEA28200090A819C1B29DF800204846F3F792FF401C10B94FF0FF3093
:20300000D2E708F0FF000090A819401CC1B29DF800204846F3F782FF401C10B94FF0FF309F
:20302000C2E70020C0E7000070B505460C4664BB1A4800691A4948600B46302269212846CE
:20304000FFF79DFF401C28B9154B302269212846FFF795FF11480068124908600F484068EA
:2030600048600E48806888600C48C068C8600B461022AD212846FFF782FF401C28B9094B17
:203080001022AD212846FFF77AFF064800680A21B0FBF1F004494882002070BD7C090020DD
:2030A000EC0800200C0A0020B40700202DE9F04706468846174699460025FCB255201F4998
:2030C0000870AA204870084680F80280A01CC870380A08710846447122464946801DF0F781
:2030E000DEFC552016490870AA20487030128870CE70221D1149891C1148001DF0F7CFFC4A
:2031000004F108010E48F1F767FF0546280EA11D0A4A5054C5F30741E01D1154C5F3072194
:20312000401C1154401C1554F021401C1154421C02493046F1F76CFEBDE8F0872A0C002054
:20314000290D00202DE9F047CCB081460E4690461F46DDF850A1982126A8F0F7B9FC982158
:203160006846F0F7B5FC0025FCB255208DF89800AA208DF89900300A8DF89A00F0B28DF83C
:203180009B008DF89C80A01CC0B28DF89D00380A8DF89E008DF89F402246514628A8F0F724
:2031A0007EFC04F1080226A96846F0F778FC04F108016846F1F710FF0546280E04F108019C
:2031C00026AA5054C5F3074104F109001154C5F30721401C1154401C1554F021401C1154E0
:2031E000401CC2B226A9484601F0D5F94CB0BDE8F087000001490968486370474815002031
:2032000001490968886370474815002001490968C8637047481500200149096808647047DC
:203220004815002008490968096A21F40051064A1268116204490968096A41EA0031024A60
:2032400012681162704700004815002010B51048007801281BD10F4A32210F4800F048F96F
:203260000446F0F702FE0D49086008460068F0F71FFE0B490860002005490870084800684B
:203280001E2804DA0348008800B20649088010BDF800002004010020EC060020FC00002076
:2032A00000010020F40000202DE9F04705460C4616461F46DDE90889F7F7F8F91949096825
:2032C000401A32282BD3F7F7F1F91649086005FB06F090FBF7F000FB08F000EBC000000196
:2032E00042F2107190FBF1F0208020880E49096808440D4908600D480078401C0B4908709E
:203300000846007808280ADB0020087006480068C0F3CF00A9F80000002003490860BDE8E8
:20332000F087000070030020780300207403002070B504460D461646F7F7B8F924490968B6
:20334000401A322841D3E07828B9F7F7AFF9214908600120E070F7F7A9F91E490968401AD1
:20336000B0F57A6F04D90020A0704FF6FF70A060208980B24FF6FF71884202D10020A070A1
:2033800001E00120A070A078012812D1A06810B94FF0FF30A0604FF4B4707043A168B0FBEA
:2033A000F1F0208020880A220B49FDF759FC288007E00020208028800A210748F1F70BFABD
:2033C00070BDF7F773F90249086000BFF8E700007C03002080030020DC12002000B585B0DB
:2033E00000BF1048806940F020000E4988610846806900F02000009000BF00BF0420019033
:20340000094802900120039001A90848F6F7AEFF002202210820F7F718FA0820F7F708FAFC
:2034200005B000BD0010024000001110001401402DE9F04104460D4617461E46F7F736F990
:2034400028490968401A32284AD3E07828B9F7F72DF9254908600120E070F7F727F92249AC
:203460000968401A4FF47A6191FBF6F1884201D90020A070A078012822D1A06810B94FF0D8
:20348000FF30A0604FF4B4707843B0FBF6F0A168B0FBF1F0208020880A221449FDF7E0FB15
:2034A0002880F7F703F96168411AA068B1EB400F12D940F20E41A0684843800AA0600BE0EF
:2034C0000020208028800A210848F1F784F94FF0FF30A060BDE8F081F7F7E8F801490860A0
:2034E00000BFF7E7680300206C030020C81200202DE9F74F88B0044689464FF0000BDA4604
:203500000020069000210F4688460D460E4600BF0FE034F81B00F0F7BEFC3A464346CDE9B5
:203520000401F0F78CFB074688460BF1010000F0FF0BCB45EDDB4846F0F7ADFC02460B4677
:20354000CDE9020138464146F0F720FCCDE90401F0F726FD06900698F0F7C3FC81B20A9836
:2035600001804FF0000A23E034F81A00F0F77DFC00900699F0F72BFB029034F81A00F0F7DD
:2035800074FC00900699F0F722FB01900299F0F724FB0390F0F7F1FC2A463346CDE904014B
:2035A000F0F74DFB05460E460AF1010000F0FF0ACA45D9DB2846314602F03AF9CDE90201C2
:2035C000F0F7C2FC80B20590F0F765FC05460E4628463146F0F7B8FC80B20BB0BDE8F08F07
:2035E00010B594B009200A904FF480300B9000200C9001200E90109002201190C10312912C
:203600004FF4E01113910AA8F7F7FEFB18B1CD211AA001F0B3FC0F2005900220069000208C
:2036200007904FF48060089000200990022105A8F7F7A8FA18B1DB2110A001F09FFC0220FC
:2036400001908003039001A8F7F704FA18B1E2210AA001F093FCF7F767FB4FF47A71B0FB0F
:20366000F1F42046F7F7F4FE0420F7F7EDFD00221146501EF7F7E9F814B010BD2E2E5C53D1
:20368000656C6654657374557365725C7372635F6D6964646C6577617265735C73746D333D
:2036A000326678785F535455737461727475702E6300000010B590B00220069001200A900B
:2036C00010200B9000200D9006A8F7F79DFB20B140F2031114A001F051FC0F200190002045
:2036E000029003904FF48060049000200590002101A8F7F747FA20B140F211110AA001F080
:203700003DFCF7F711FB4FF47A71B0FBF1F42046F7F79EFE0420F7F797FD00221146501E3B
:20372000F7F793F810B010BD2E2E5C53656C6654657374557365725C7372635F6D69646461
:203740006C6577617265735C73746D33326678785F535455737461727475702E630000000C
:20376000034618044843B0FBF2F0704710B5F6F7D3FFF7F787FE03480078401C014908703D
:2037800010BD00005900002010B594B009200A904FF480300B9000200C9001200E9010906E
:2037A00002201190C10312914FF4E01113910AA8F7F72AFB20B14FF4C0711CA001F0DEFB77
:2037C0000F20059002200690002007904FF48060089000200990022105A8F7F7D3F920B1E7
:2037E0004FF4C77111A001F0C9FB022001908003039001A8F7F72EF920B140F295110BA00D
:2038000001F0BCFBF7F790FA4FF47A71B0FBF1F42046F7F71DFE0420F7F716FD00221146BD
:20382000501EF7F712F814B010BD00002E2E2F436F72652F5372632F6D61696E2E630000C1
:203840001148006840F001000F490860084640680E4908400C494860084600680C490840D1
:20386000094908600846006820F4802008600846406820F4FE0048604FF41F008860C803F7
:203880000449086070470000001002400000FFF8FFFFF6FE08ED00E010B50248F7F7F0FFC0
:2038A00010BD00004815002000220268184B984208D0B0F1804F05D0164B984202D0164B6A
:2038C000984203D122F070024B681A43104B984208D0B0F1804F05D00E4B984202D00E4BF6
:2038E000984203D122F44072CB681A4322F080024B691A4302608B68C3620B688362044BFC
:20390000984201D10B6903630123436170470000002C0140000400400008004030B50023A1
:20392000012404FA01F3046A9C430462046A02FA01F52C43046230BD30B50023042404FA6D
:2039400001F3046A9C430462046A02FA01F52C43046230BD30B50C460021816821F47F4188
:2039600042EA032525432943816030BD0A460021816821F0700142F0070319438160704745
:2039800030B5002400220023056A25F001050562026A4368846924F0700424F003040D68CC
:2039A0002C4322F002028D682A430D4DA84206D100BF22F00802CD682A4322F00402084D1B
:2039C000A84207D123F4807323F400734D692B438D692B43436084614D684563026230BDD3
:2039E000002C014030B5002400220023056A25F010050562026A4368846924F4E04424F4B4
:203A000040740D6844EA052422F020028D6842EA05120F4DA84207D100BF22F08002CD6814
:203A200042EA051222F04002094DA84209D123F4806323F400634D6943EA85038D6943EAD3
:203A40008503436084614D688563026230BD0000002C014030B5002400220023056A25F425
:203A600080750562026A4368C46924F0700424F003040D682C4322F400728D6842EA05224F
:203A80000E4DA84207D100BF22F40062CD6842EA052222F48062094DA84209D123F480534E
:203AA00023F400534D6943EA05138D6943EA05134360C4614D68C563026230BD002C014003
:203AC00030B5002200230024056A25F480550562036A4468C26922F4E04222F440720D681B
:203AE00042EA052223F400538D6843EA0533074DA84204D124F480444D6944EA851444609F
:203B0000C2614D680564036230BD0000002C014030B50B46144600210022026A056A25F0E2
:203B200001050562816921F0F00141EA041122F00A021A438161026230BD30B50B461446AE
:203B400000210022056A25F0100505628169026A21F4704141EA043122F0A00242EA0312B1
:203B60008161026230BD0146002240F205100860086882B240F20510824201D000207047A3
:203B800040F28A200860086882B240F28A20824201D00020F3E70020086045F255504860C6
:203BA000486882B245F25550824201D00020E6E742F6A8204860486882B242F6A820824273
:203BC00001D00020DBE70020486045F255508860886882B245F25550824201D00020CEE73C
:203BE0004AF6A2208860886882B24AF6A220824201D00020C3E70020886045F25550C8604A
:203C0000C86882B245F25550824201D00020B6E742F6AA20C860C86882B242F6AA208242BE
:203C200001D00020ABE70020C86045F255508861886982B245F25550824201D000209EE7B9
:203C40004AF6AA208861886982B24AF6AA20824201D0002093E70020886145F25550C86105
:203C6000C86982B245F25550824201D0002086E74AF6AA20C861C86982B24AF6AA2082427B
:203C800001D000207BE70020C86141F255500862086A82B241F25550824201D000206EE7BE
:203CA00042F6AA200862086A82B242F6AA20824201D0002063E70020086245F255504862E1
:203CC000486A82B245F25550824201D0002056E74AF6AA204862486A82B24AF6AA208242C8
:203CE00001D000204BE70020486245F255508862886A82B245F25550824201D000203EE735
:203D00004AF6AA208862886A82B24AF6AA20824201D0002033E70020886245F25550C862A0
:203D2000C86A82B245F25550824201D0002026E74AF6AA20C862C86A82B24AF6AA20824217
:203D400001D000201BE70020C86255200863086B82B2552A01D0002011E7AA200863086B8F
:203D600082B2AA2A01D0002009E70020086345F255504863486B82B245F25550824201D0F0
:203D80000020FCE64AF6AA204863486B82B24AF6AA20824201D00020F1E60020486345F2ED
:203DA00055508863886B82B245F25550824201D00020E4E64AF6AA208863886B82B24AF695
:203DC000AA20824201D00020D9E60020886345F25550C863C86B82B245F25550824201D0BB
:203DE0000020CCE64AF6AA20C863C86B82B24AF6AA20824201D00020C1E60020C86345F26D
:203E000055500864086C82B245F25550824201D00020B4E64AF6AA200864086C82B24AF660
:203E2000AA20824201D00020A9E60020086441F215508864886C82B241F21550824201D00F
:203E400000209CE640F60A208864886C82B240F60A20824201D0002091E60020886408614B
:203E600001208CE62DE9F04104460E461746984627480078012812D1264801780078401CE1
:203E8000244A1070244820F811601046007832281CDB00201E4908701146087016E0322208
:203EA0001D493046FCF7DCFE05462088A84209DDF6F7FCFB19490968401AB0F57A7F05D909
:203EC000258003E0F6F7F2FB1449086040F634007843642190FBF1F0C0F5805021888842AD
:203EE00003DBF6F7E3FB0E490860F6F7DFFB0C490968401A42F21071884206D9094800784C
:203F000020F00100401C07490870BDE8F0810000890300208A0300207A130020900300209D
:203F20008C030020840300202DE9F04104460E461746984627480078012812D12648017831
:203F40000078401C244A1070244820F811601046007832281CDB00201E49087011460870BD
:203F600016E032221D493046FCF77AFE05462088A84209DDF6F79AFB19490968401AB0F599
:203F80007A7F05D9258003E0F6F790FB1449086040F634007843642190FBF1F0C0F58050EA
:203FA0002188884203DBF6F781FB0E490860F6F77DFB0C490968401A42F21071884206D9A5
:203FC0000948007820F00200801C07490870BDE8F08100009403002095030020DE1300200C
:203FE0009C03002098030020840300202DE9F04104460E461746984627480078012812D18D
:20400000264801780078401C244A1070244820F811601046007832281CDB00201E490870E4
:204020001146087016E032221D493046FCF718FE05462088A84209DDF6F738FB19490968CC
:20404000401AB0F57A7F05D9258003E0F6F72EFB1449086040F634007843642190FBF1F011
:20406000C0F580502188884203DBF6F71FFB0E490860F6F71BFB0C490968401A42F21071CC
:20408000884206D90948007820F00400001D07490870BDE8F0810000A0030020A103002018
:2040A00042140020A8030020A4030020840300202DE9F04704460F46E7824FF00908414625
:2040C0002046F3F717FEC01B0FFA80F919F1780F41DDB9F1780F3EDA002606E0701C34F862
:2040E000100024F81600701CC6B2A8F10100B042F4DC24F8107041462046F3F77BFE05B27B
:20410000608AA84200DA658241462046F3F783FE05B2A08AA84200DDA5821148844206D1ED
:204120002346182215210F48FEF729FF16E00E48844206D12346182232210A48FEF71FFFEE
:204140000CE00A48844209D1234618224F210548FEF715FF02E0002005490870BDE8F08734
:20416000F0120020B40300200A130020241300208803002003B5024664211176002006E0F5
:2041800002EB4001BDF804300B80411CC8B20C28F6D300201BE0411C01EB81014900C1EBCE
:2041A000C1014FF6FF7303EA8101144B23F82010411C01EB81014906090E03EB80039970C2
:2041C00080210E4B03EB8003D970411CC8B20728E1DB07200FE04FF6FF71084B23F8201000
:2041E000502103EB800399708021044B03EB8003D970411CC8B20F28EDDB0CBD3E1300201A
:2042000008B5024602F5004081B20846CB1701EB936399114FF6FE70014001F4407038B3EF
:20422000B0F5807F36D0B0F5007F03D0B0F5407F40D10DE0C8B2214B33F81000ADF80200B3
:20424000C8B2C0F1FF0033F81000ADF8000032E0C8B2C0F1FF00194B33F81000ADF80200D2
:20426000C8B233F81000404200B2ADF8000022E0C8B2124B33F81000404200B2ADF80200C1
:20428000C8B2C0F1FF0033F81000404200B2ADF8000010E0C8B2C0F1FF00084B33F8100038
:2042A000404200B2ADF80200C8B233F81000ADF8000000E000BF00BF009808BDE65C0108C3
:2042C00070B505466C6A0020E085E0842046F7F7E6FD70BD2DE9F04106460D4614460020EB
:2042E00025490870F6F7E2F92349486005F0FF08A5F50040083830B1A0F6FA70B8B1B0F5F7
:20430000545F2DD108E0424621461C48EFF7C7FB00201B4908702BE023462A46314640F280
:204320001560FEF7C3FE01201649087020E02178627801EB02218FB2002007E0124931F80C
:204340001010B94200DD03E0411CC8B20B28F5D300BF00F14601CAB20C4981F8272007E041
:2043600023462A46314640F21560FEF79FFE00BF00BFBDE8F08100009001002082010020CC
:204380008C0100205D000020D85F0108D407002010B50A46C37893421EDBC3681B68DB68A9
:2043A00023F02003C4682468E360C3789B1AC370C3681B68DB6843F02003C4682468E36067
:2043C000114683780B4499B203788B4202DC0378CB1A99B281701BE0C3681B68DB6823F030
:2043E0002003C4682468E360C1780023C370C3681B68DB6843F02003C4682468E3608378D3
:20440000194403788B4202DC0378CB1A99B2817010BD0168C96821F490710268D1600168FC
:20442000496921F0010102685161202180F83A10704710B504462068C06820F04000216849
:20444000C860202084F839002046F7F76EFE002010BD00BFC27803789A42FBD0C2681268D3
:20446000D26822F08002C3681B68DA60C2788AB9C26812681268C2F3C0125AB1C2681268B5
:204480005160C2681268D26842F08002C3681B68DA60704743788268D1544278521CD2B2C4
:2044A000427003789A4201D100224270C278521CC270C2681268D26842F08002C3681B6833
:2044C000DA6000BFE5E710B502460B461946D4789C4209DB94780C44A1B214788C4204DC63
:2044E00014780C1BA1B200E000219468605C10BD70B5044694F83A0022284AD1A068B0F5E9
:20450000805F13D1A56A206940B920684068C0F308002880A06A801CA06219E020684068E3
:20452000C0B22880A06A401CA06211E0206938B920684068C1B2A26A501CA062117007E009
:204540002068406800F07F01A26A501CA0621170E08D401E80B2E085C8B92068C06820F01D
:2045600020002168C8602068C06820F480702168C8602068406920F0010021684861202051
:2045800084F83A002046F7F7CFFD002070BD0020FCE70220FAE7F0B507460D46164600242D
:2045A00005E0295D3846FFF754FF601CC4B2B442F7DBF0BD2DE9F0410446002520680069BB
:2045C00020F44050E1680843216808612169A06808436169084305432068C06841F20C6127
:2045E000884328432168C8602068406920F44070A1690843216848615F49206888425CD131
:20460000F6F7A8FB00EBC00101EB001061688900B0FBF1F6F6F79EFB00EBC00101EB001050
:2046200061688900B0FBF1F06421B0FBF1F000EBC00101EB0010A6EB8000322101EB001083
:204640006421B0FBF1F000F0F006F6F783FB00EBC00101EB001061688900B0FBF1F06421ED
:20466000B0FBF1F006EB0016F6F774FB00EBC00101EB001061688900B0FBF1F7F6F76AFB6C
:2046800000EBC00101EB001061688900B0FBF1F06421B0FBF1F000EBC00101EB0010A7EB49
:2046A0008000322101EB00106421B0FBF1F000F00F003044216888605BE0F6F73BFB00EBED
:2046C000C00101EB001061688900B0FBF1F6F6F731FB00EBC00101EB001061688900B0FB7B
:2046E000F1F06421B0FBF1F000EBC00101EB0010A6EB8000322101EB00106421B0FBF1F0AF
:2047000000F0F006F6F716FB00EBC00101EB001061688900B0FBF1F06421B0FBF1F006EB2D
:204720000016F6F707FB00EBC00101EB001061688900B0FBF1F7F6F7FDFA00EBC00101EB6B
:20474000001061688900B0FBF1F06421B0FBF1F000EBC00101EB0010A7EB8000322101EB61
:2047600000106421B0FBF1F000F00F00304421688860BDE8F081000000380140014691F8D5
:20478000390021282CD18868B0F5805F0FD10A6A1088C0F308000B685860086918B9086AA0
:2047A000801C086209E0086A401C086205E00B6A581C086218780B685860C88C401E80B2FB
:2047C000C88458B90868C06820F080000B68D8600868C06840F040000B68D860002070471F
:2047E0000220FCE710B5054800F00EF8044800F040F80448F7F754FB10BD0000E4040020DA
:20480000F4040020901D002008B5C26812681268C2F3401262B3C26812685268D1B2C268B1
:20482000126812680022B2B943788268D1544278521CD2B2427003789A4201DB00224270C8
:20484000C278521CD2B2C27003789A4203DD0278C2700122027100BF00220092C26812686A
:2048600012680092C26812685268009200BF00BF08BDC16809680968C1F3C01139B3C16854
:204880000968C96801F0800109B36FF08001C26812681160C17891B1C178491EC17082780D
:2048A0008168895CC268126851608178491CC9B28170027891420ADB0021817007E0C168B7
:2048C0000968C96821F08001C2681268D160704710B50248F4F776FD10BD00004C1B002057
:2048E00010B54FF4FA71024800F004F810BD0000E40400202DE9F34F83B00398C0780D28A7
:2049000073DB00210398FFF7DEFD01906B490198087001210398FFF7D6FD8146674981F8F0
:204920000190019855287DD1B9F1AA0FFBD102210398FFF7C8FD6149887003210398FFF783
:20494000C2FD5E49C87004210398FFF7BCFD06465A490E71112E03D0162E01D00C2E7DD12D
:2049600005210398FFF7AFFD07465448477107210398FFF7A8FD834606210398FFF7A3FDB4
:204980000BEB00201FFA80F84FEA18204B49887181F8078007210398FFF795FD0446381B8A
:2049A00002287AD10398C17807F10B0081421DDA43480078012806D1F5F778FE414908609A
:2049C00000203F490870F5F771FE3E490968411A0498814206D9F5F769FE3A49086001206C
:2049E0003749087005B0BDE8F08F64E001203449087000250FE005F10800C1B20398FFF776
:204A000062FD314948550846415D05F108002B4A1154681C85B2A542EDDB04F10800C1B282
:204A2000039800E043E0FFF74EFD4FEA006B04F10900C1B20398FFF746FD0BEB004B04F178
:204A40000A00C1B20398FFF73EFD0BEB002B04F10B00C1B20398FFF736FD00E022E0584437
:204A6000029004F108011548F0F7B6FA82460298B0EB0A000CD1144A41463046FFF72AFC57
:204A800007F10B00C1B20398FFF782FCAAE704E001210398FFF77CFC0DE001210398FFF751
:204AA00077FC08E001210398FFF772FC03E001210398FFF76DFC00BF94E70000BE0E002055
:204AC000C4010020C0010020280E0020012806D002282CD0032851D0042878D178E05249E1
:204AE000524A13680B6053684B6092688A60504A1368CB6053680B6192684A610A464D49F8
:204B00000B6893614B68D3618968116211464A4A13684B6253688B629268CA620A46474922
:204B20000B6813634B685363896891637AE03E49434A13680B6053684B6092688A600A4650
:204B400040490B68D3604B6813618968516111463D4A13688B615368CB6192680A623B4A45
:204B600013684B6253688B629268CA62384A13680B6353684B6392688A6353E02A4A35495F
:204B80000B6813604B685360896891601146324A1368CB6053680B6192684A610A462F49DA
:204BA0000B6893614B68D3618968116211462C4A13684B6253688B629268CA620A462949BE
:204BC0000B6813634B685363896891632AE028E01549254A13680B6053684B6092688A608F
:204BE0000A4622490B68D3604B6813618968516111461F4A13688B615368CB6192680A6216
:204C00000A461C490B6853624B6893628968D1621146194A13680B6353684B6392688A63F8
:204C200000E000BF00BF7047D0090020EE5F0108FA5F010806600108126001081E6001083D
:204C40002A60010836600108426001084E6001085A60010866600108726001087E6001086C
:204C60008A60010896600108A2600108AE600108BA600108C6600108D260010800BFFEE7EF
:204C800010B5002048490860484908804849087007204849087018214748EEF719FF1821E6
:204CA0004648EEF715FF18214548EEF711FF102244494548EEF7F3FE444845490A680260A2
:204CC00049684160102243A14748EEF70CFF102246A145481030EEF706FF2E2142482038EC
:204CE00080F83F10202246A14E48EEF7FCFE4E48007828B930213C48203880F82A102CE075
:204D000049480078012805D131213748203880F82A1022E044480078022805D132213248DD
:204D2000203880F82A1018E03F480078032805D133212D48203880F82A100EE03A480078B6
:204D4000042805D134212848203880F82A1004E030212548203880F82A10102233A1224866
:204D60002038EEF7C0FE102236A11F481038EEF7BAFE082238A13B48EEF7B5FE08223AA1C0
:204D800038480830EEF7AFFE08223AA135481030EEF7A9FE3A483B4B0ECB0EC000F09AF84A
:204DA00000F072F810BD00006C01002082010020840300207001002044080020840800204C
:204DC0006C080020085F01085C08002071010020185F010854544B5A303130442E20202089
:204DE0002020202000000000F40700205634723172305F3230323330363238430000000010
:204E000054433031313030302D4D53303030302D563172302E202020202020202020202068
:204E20000000000014080020B8010020564C36355858265653373558584A30312E2020207C
:204E40002020200030303030303030303030303030303030000000004D4F54494E4F564185
:204E6000000000002C090020575548414E2E2020000000003230323130393031000000005D
:204E8000A4090020E8F7FF1F10B5302209490A48EEF705FE102209490948EEF700FE09489C
:204EA000094C1ECC1EC0102208490948EEF7F7FD10BD0000705F0108EC080020A05F010867
:204EC0001C0900200C0A0020C05F0108B05F01081C0A002010B50C2216A11A48EEF703FEDF
:204EE000194801891948FFF745F9174841891848FFF740F9144881891648FFF73BF916482E
:204F000016490A680260496841604FF4B87014490880202213491448EEF7C1FD2022134981
:204F20001348EEF7BCFD102212491348EEF7B7FD10BD0000303030303030303030303030EA
:204F400000000000B009002008160020F01200200A130020241300207A010020D05F0108B1
:204F600086030020205F01089C080020405F0108BC080020605F0108DC08002088B0044662
:204F80000D4631E01948FAF708FB0020FCF7F4F8F1F7D6FD20216846EEF79AFD2046EEF7E8
:204FA000AEFD0646324621466846EEF778FD2046EEF7A5FD694608440DA10A880280897868
:204FC00081702046EEF79BFD69460844C0F803506B464FF620720C214FF4E260FEF766F86A
:204FE000C820F4F7C9FF00BFCCE70000EC000020202C200008B52B4988420DD100BF2A4921
:20500000896941F00401284A91611146896901F00401009100BF43E0244988420DD100BF7E
:205020002149896941F008011F4A91611146896901F00801009100BF32E01D4988420DD1CC
:2050400000BF1949896941F01001174A91611146896901F01001009100BF21E015498842E4
:205060000DD100BF1049896941F020010E4A91611146896901F02001009100BF10E00E49BA
:2050800088420DD100BF0849896941F04001064A91611146896901F04001009100BF00BF28
:2050A00008BD00000008014000100240000C014000100140001401400018014070B50446D5
:2050C0000E46A1882068F5F7DFFA28B9A07908B9012506E0002504E0A07908B9002500E057
:2050E0000125012E04D1207A68402840E07102E0207A6840E071257270BD10B50446A1881A
:2051000001222068F5F7CCFA10BD00BF704702E008C8121F08C1002AFAD1704770470020C0
:2051200001E001C1121F002AFBD1704700F0010181F31388704700000149086070470000CD
:2051400014050020F0B504460E4619681F683D14A54206DA31440814A04212DD20460104E6
:205160000FE0A5420CDD02EB04473DB2A94202DA2046010405E0891A081410B9002100E0A9
:2051800020461960F0BD000010B50A46437993421EDB1E4B1B685B6923F002031B4C246829
:2051A000636143799B1A4371184B1B685B6943F00203164C24686361114603790B4499B205
:2051C00083788B4202DC8378CB1A99B201711BE00E4B1B685B6923F002030C4C2468636131
:2051E000417900234371094B1B685B6943F00203064C246863610379194483788B4202DC2A
:205200008378CB1A99B2017110BD00004C1B002010B502460B46194654799C4209DB1479C4
:205220000C44A1B294788C4204DC94780C1BA1B200E000219468605C10BD00007FB5064685
:20524000002404E0305D18490855601CC4B2082CF8DB3823154A02A9304600F00FFB002409
:205260001EE0002504E002A800F0A4FA681CC5B20F48005DA842F6DC40230E4A694602A870
:2052800000F0FCFA002507E01DF805000A4901EBC4014855681CC5B2082DF5DB601CC4B26F
:2052A000102CDEDB7FBD0000FC020020A0670108786A0108D8670108A4110020014601201F
:2052C000064A12688A4206D1044A1268044B1B685A40521C02B1002070470000D01D002028
:2052E000F41D00202DE9F04F87B082460F469046994600250AE0785D3A49495D884203D075
:205300003846FFF79BFF0725681CC5B2082DF2DB4023354A05A9504600F0B0FA012536E05A
:20532000002405E005A8005D03A90855601CC4B2082CF7DBB8F1000F04D1681E2B4901EBE6
:20534000C00B04E0C5F11000284901EBC00B002406E003A9201D085C05A90855601CC4B25C
:20536000042CF6DB01AA05A9584600F043F8002409E003A8005D01A9095D484005AA211D70
:205380005054601CC4B2042CF3DB681CC5B2112DC6DB9DF814609DF818008DF814008DF8CB
:2053A00018609DF815609DF819008DF815008DF819609DF816609DF81A008DF816008DF84B
:2053C0001A609DF817609DF81B008DF817008DF81B604023064A494605A800F04FFA07B01C
:2053E000BDE8F08FFC020020E0660108A411002020670108F0B587B005460E46174640237C
:20540000104A05A9304600F039FA002410E005A8005D295D484000F03F0003A908550A4835
:2054200000EB8410095D405C01A90855601CC4B2082CECDB2023054A394601A800F01EFA35
:2054400007B0F0BD1868010878680108586801081CB5F7F7F3F8F7F7F9F8B2490870F2F7C8
:2054600005FBF5F765F9FEF78FF9F7F71BFAFBF7C9F9FBF769FAFBF7D1FAFBF719FBFBF7A4
:20548000A7F9FBF751F8FBF71DF9FBF773F9FBF759FBFCF7F3FBEEF7FBFF1420F4F76CFD3D
:2054A000A148F6F735F9FFF7EBFBFBF72DFAFAF7E9FD9E48F1F7ECFBF1F790FD9B48F1F727
:2054C0009FFBF1F7D7FD9A490870084601789748FDF7AAFD97499848F1F7AAFDF9F7E0FFBC
:2054E0000020964908701CE195480078401C9449087008460078C82801DD0020087091482D
:205500000088F2F707FCFBF7E3FBEFF7DBFEFFF7E7F98D4A51788D4AD07A8D4B8D4A1278B8
:20552000F8F74CFDFAF7BCFF8848807EAA2841D18948007BC0B18848B0F902000B2190FBE6
:20554000F1F084B284498148007B804A92F91B20104480B2CDE900017C48C37982797F4993
:205560002046FDF7A1FE46E07B48B0F902000B2190FBF1F07849897A884206DD7648B0F92E
:2055800002000B2190FBF1F001E07348807A84B271496E48007B6D4A92F91B20104480B2B7
:2055A000CDE900016948C37982796C492046FDF77BFE20E06548807EEE280AD16348007B02
:2055C0006249C97E0844C2B263496448FDF7B0FE11E05E48007B5D49C97E0844C2B25B48BD
:2055E000007E08B9012001E05848007E03465A495A48FDF71DFF5A48F2F76EFB5948EFF733
:20560000B3F900BF5848007818BB5848007828B1F5F74CF842F21071884229D94E48C088B4
:205620000A2190FBF1F084B251488088474A0090127B464D95F91B502A4490B24D4A137BED
:205640004A4A11782246FBF7DBFF0120464908700EE0414C2389464C627AA1883F4CE06840
:20566000FBF7A8FE444A1178394A1078FBF7FCFF00BFFAF739FB4148FAF78CFCFAF778FE36
:20568000354B9A7D1989987AF8F7DEFA3C4908703948807910B93B48F1F7C0FC364880791A
:2056A00030B939493948F1F75BFD3948FCF780F938480078E8B938480068384908603648E9
:2056C000406848603448806888603348C068C8602A48001F40680861282217480830FDF7EC
:2056E000EDFB04222EA11448FDF7E8FB012029490870F8F755FEF9F7B3FF2B480068FAF7DF
:2057000077FC14480078FAF79BFC2848FAF7E4FCFDF79CFDFDF72CF8FCF730FA2448F4F760
:20572000F3FFE1E6B801002088150020B4030020AC030020FFEF010800E801085C00002010
:205740005A000020BC010020710100209C080020C6000020C4000020B4070020580300207C
:20576000C5030020C40300205B000020A801002034080020DC080020CA000020F0080020B4
:20578000DA000020AD030020040300202412002079010020BF0100200C0A00207C0900206D
:2057A000464C4147000000006C010020BC090020E80500200CB5002104E0425C0DF80120C6
:2057C0004A1CD1B20829F8DB002112E0425C5206120E425406290ADA4A1C1DF8022002F07B
:2057E0008002802A03D1425C42F0010242544A1CD1B20729EADB9DF8002002F0800222B166
:20580000C27842F01002C27003E0C27822F01002C2709DF8032002F0080222B1827942F0B1
:205820000102827103E0827922F0010282710CBD2DE9F04106460F46EEF783FC04000D4620
:2058400018BF0120284320F00040C0F17F6000F1E040C00F0ED0301C18BF0120384320F078
:205860000040C0F17F6000F1E040C00F04BF0120FFF762FC20462946BDE8F0812DE9F0410E
:2058800004461D46154E002000BF4FF000080746401C01F807800828F7DB002000BF12F8BE
:2058A000013B04EBE3073F7803F0070C16F80CC007EA0C0767B101EBE0073F7800F0070C93
:2058C00016F80CC047EA0C0701EBE00C8CF80070471C3846AF42E2DBBDE8F081886A01083E
:2058E000000000000000000001020304060708090000000001020304204E000403000004FD
:2059000000000004000000009CFFFFFFFF7F0000000000FE00FCFF0100000000204E000400
:205920000300000400000004000000000080FFFFFF7F0000000000FE00FCFF010000000066
:20594000400000040300000400000004000000000000FCFF00000000000000F0000000000D
:2059600000000000307500012C0100040000000400000000CCF7FFFF000000000030DFFF7D
:20598000000000000000000000100004010000040000000400000000E6FBFFFF1A040000ED
:2059A0000088FAFF0078050000000000307500042C0100040000000400000000E6FBFFFF2C
:2059C000000000000098EFFF0000000000000000204E0004030000040000000400000000C4
:2059E0009CFFFFFFFF7F0000000000FE00FCFF0100000000204E0004030000040000000419
:205A0000000000000080FFFFFF7F0000000000FE00FCFF0100000000400000040300000445
:205A200000000004000000000000FCFF00000000000000F0000000000000000030750001D1
:205A40002C0100040000000400000000CCF7FFFF000000000030DFFF000000000000000042
:205A600000100004010000040000000400000000E6FBFFFF1A0400000088FAFF007805000E
:205A800000000000307500042C0100040000000400000000E6FBFFFF000000000098EFFFC3
:205AA0000000000000000000204E00040300000400000004000000009CFFFFFFFF7F000052
:205AC000000000FE00FCFF0100000000204E00040300000400000004000000000080FFFFD1
:205AE000FF7F0000000000FE00FCFF010000000040000004030000040000000400000000DF
:205B00000000FCFF00000000000000F00000000000000000307500012C01000400000004BF
:205B200000000000CCF7FFFF000000000030DFFF000000000000000000100004010000047D
:205B400000000004000000009CFFFFFF1A0400000088FAFF007805000000000030750004E3
:205B60002C0100040000000400000000E6FBFFFF000000000098EFFF00000000000000008B
:205B8000204E00040300000400000004000000009CFFFFFFFF7F0000000000FE00FCFF0177
:205BA00000000000204E00040300000400000004000000000080FFFFFF7F0000000000FE6E
:205BC00000FCFF0100000000400000040300000400000004000000000000FCFF000000007F
:205BE000000000F00000000000000000307500012C0100040000000400000000CCF7FFFF19
:205C0000000000000030DFFF00000000000000000010000401000004000000040000000059
:205C20009CFFFFFF1A0400000088FAFF0078050000000000307500042C01000400000004D1
:205C400000000000E6FBFFFF000000000098EFFF0000000000000000657F367E107D807CBE
:205C6000657B527A467940784177C476CE75DF74F47310739F72C271EA701770486F7D6EC8
:205C80001A6E566D966CDA6B216B6D6A136A6469B8680F68696718677666D8653D65A4641C
:205CA0000E64C4633263A26215628A614561BE603960B55F345FB55E765EFA5D805D085DCC
:205CC000915C1C5CE25B705BFF5A905A235AED5981591859AF584858E357B1574D57EB5638
:205CE0008A562B56CC550000C90092015B022403ED03B6047F0548061107D907A2086A09B1
:205D0000330AFB0AC40B8C0C540D1C0EE30EAB0F72103A110112C8128F1355141C15E215B7
:205D2000A8166E173318F918BE19821A471B0B1CCF1C931D571E1A1FDD1F9F2061212322FD
:205D4000E522A62367242825E825A82667272628E528A329612A1F2BDC2B992C552D112EA9
:205D6000CC2E872F4130FB30B5316E322633DF3396344D350436BA366F372438D9388C3998
:205D8000403AF23AA53B563C073DB83D683E173FC53F73402141CE417A422543D0437A4499
:205DA0002445CD4575461C47C34769480F49B449584AFB4A9D4B3F4CE04C814D204EBF4E6B
:205DC0005D4FFB4F97503351CE51685202539B533254C9546055F5558A561D57B0574258AF
:205DE000D3586459F359825A0F5B9C5B285CB35C3E5DC75D4F5ED75E5D5FE35F6860EB60ED
:205E00006E61F0617162F1627063EE636C64E8646365DD655666CF664667BC673268A66889
:205E200019698B69FD696D6ADC6A4A6BB76B236C8E6CF86C616DC96D306E966EFB6E5E6FC9
:205E4000C16F22708370E27040719D71F9715472AE7207735E73B5730A745F74B2740475C9
:205E60005575A575F37541768D76D87622776B77B377FA773F788478C77809794A7989797F
:205E8000C879057A417A7C7AB67AEE7A267B5C7B917BC57BF87B297C597C887CB67CE37CB3
:205EA0000E7D397D627D897DB07DD57DFA7D1D7E3E7E5F7E7E7E9C7EB97ED57EEF7E097FFD
:205EC000217F377F4D7F617F747F867F977FA67FB47FC17FCD7FD87FE17FE97FF07FF57FCC
:205EE000F97FFD7FFE7F000005000000000000000500000000000000050000000000000022
:205F00000500000000000000A0282400000000000000000000000000045500000000000037
:205F200055026400180310100F87A555DB026464646464646464646401025500B80B3C8738
:205F40000000000055020606000000000000000000000000000000000000000000000000DE
:205F6000FA00B004C8000A000A00A08C240000000100000000000000000000000000000046
:205F800000000000000000000000000000000000000041410000000041414141000000007B
:205FA000000000000000000000000000000000006400A000BE000E01B4000000000000005C
:205FC0000000000000000000000000000000000041564F4E49544F4D7401E8025C04D105BF
:205FE0004507B9082D0AA20B160D8A0EFF0F4701000064007805020200048F0200006400C1
:206000007805020200040004000064007805030200041E0500006400780504020004E80314
:20602000D00764007805040200044701000064007805020200048F020000640078050202F7
:2060400000040004000064007805030200041E0500006400780504020004E803D00764001A
:20606000780504020004CA0200006400A903020100025A0500006400E2040302AE0234081E
:2060800030026400B30504026603800CBC0264003408050300040000CC010000340804023E
:2060A0000004CA0200006400A90302010002940500006400E2040302AE025E083002640067
:2060C000B30504026603800CBC0264003408050300040000CC010000340804020004000090
:2060E00000002110422063308440A550C660E770088129914AA16BB18CC1ADD1CEE1EFF1A0
:206100003112100273325222B5529442F772D662399318837BB35AA3BDD39CC3FFF3DEE35F
:206120006224433420040114E664C774A44485546AA54BB528850995EEE5CFF5ACC58DD51F
:206140005336722611163006D776F6669556B4465BB77AA719973887DFF7FEE79DD7BCC7DF
:20616000C448E5588668A7784008611802282338CCC9EDD98EE9AFF9488969990AA92BB99F
:20618000F55AD44AB77A966A711A500A333A122AFDDBDCCBBFFB9EEB799B588B3BBB1AAB5F
:2061A000A66C877CE44CC55C222C033C600C411CAEED8FFDECCDCDDD2AAD0BBD688D499D1F
:2061C000977EB66ED55EF44E133E322E511E700E9FFFBEEFDDDFFCCF1BBF3AAF599F788FDF
:2061E0008891A981CAB1EBA10CD12DC14EF16FE18010A100C230E32004502540467067609F
:20620000B9839893FBA3DAB33DC31CD37FE35EF3B1029012F322D23235421452776256725E
:20622000EAB5CBA5A89589856EF54FE52CD50DC5E234C324A014810466744764245405441E
:20624000DBA7FAB79987B8975FE77EF71DC73CD7D326F2369106B0165766767615463456DE
:206260004CD96DC90EF92FE9C899E9898AB9ABA94458654806782768C018E1088238A3289E
:206280007DCB5CDB3FEB1EFBF98BD89BBBAB9ABB754A545A376A167AF10AD01AB32A923A5E
:2062A0002EFD0FED6CDD4DCDAABD8BADE89DC98D267C076C645C454CA23C832CE01CC10C1E
:2062C0001FEF3EFF5DCF7CDF9BAFBABFD98FF89F176E367E554E745E932EB23ED10EF01EDE
:2062E00000000000B71DC1046E3B8209D926430DDC7604136B6BC517B24D861A0550471E0E
:20630000B8ED08260FF0C922D6D68A2F61CB4B2B649B0C35D386CD310AA08E3CBDBD4F38AD
:2063200070DB114CC7C6D0481EE09345A9FD5241ACAD155F1BB0D45BC2969756758B56524D
:20634000C836196A7F2BD86EA60D9B6311105A6714401D79A35DDC7D7A7B9F70CD665E74ED
:20636000E0B6239857ABE29C8E8DA191399060953CC0278B8BDDE68F52FBA582E5E664868D
:20638000585B2BBEEF46EABA3660A9B7817D68B3842D2FAD3330EEA9EA16ADA45D0B6CA02D
:2063A000906D32D42770F3D0FE56B0DD494B71D94C1B36C7FB06F7C32220B4CE953D75CACD
:2063C00028803AF29F9DFBF646BBB8FBF1A679FFF4F63EE143EBFFE59ACDBCE82DD07DEC6D
:2063E00077708634C06D4730194B043DAE56C539AB0682271C1B4323C53D002E7220C12A0D
:20640000CF9D8E1278804F16A1A60C1B16BBCD1F13EB8A01A4F64B057DD00808CACDC90CAC
:2064200007AB9778B0B6567C69901571DE8DD475DBDD936B6CC0526FB5E6116202FBD0664C
:20644000BF469F5E085B5E5AD17D1D576660DC5363309B4DD42D5A490D0B1944BA16D840EC
:2064600097C6A5AC20DB64A8F9FD27A54EE0E6A14BB0A1BFFCAD60BB258B23B69296E2B28C
:206480002F2BAD8A98366C8E41102F83F60DEE87F35DA9994440689D9D662B902A7BEA942C
:2064A000E71DB4E0500075E4892636E93E3BF7ED3B6BB0F38C7671F7555032FAE24DF3FECC
:2064C0005FF0BCC6E8ED7DC231CB3ECF86D6FFCB8386B8D5349B79D1EDBD3ADC5AA0FBD86C
:2064E000EEE00C6959FDCD6D80DB8E6037C64F643296087A858BC97E5CAD8A73EBB04B77CC
:20650000560D044FE110C54B383686468F2B47428A7B005C3D66C158E4408255535D4351EB
:206520009E3B1D252926DC21F0009F2C471D5E28424D1936F550D8322C769B3F9B6B5A3B0B
:2065400026D6150391CBD40748ED970AFFF0560EFAA011104DBDD014949B93192386521D2B
:206560000E562FF1B94BEEF5606DADF8D7706CFCD2202BE2653DEAE6BC1BA9EB0B0668EF4B
:20658000B6BB27D701A6E6D3D880A5DE6F9D64DA6ACD23C4DDD0E2C004F6A1CDB3EB60C96B
:2065A0007E8D3EBDC990FFB910B6BCB4A7AB7DB0A2FB3AAE15E6FBAACCC0B8A77BDD79A38B
:2065C000C660369B717DF79FA85BB4921F4675961A163288AD0BF38C742DB081C3307185AB
:2065E00099908A5D2E8D4B59F7AB085440B6C95045E68E4EF2FB4F4A2BDD0C479CC0CD43CB
:20660000217D827B9660437F4F460072F85BC176FD0B86684A16476C93300461242DC565EA
:20662000E94B9B115E565A1587701918306DD81C353D9F0282205E065B061D0BEC1BDC0F0A
:2066400051A69337E6BB52333F9D113E8880D03A8DD097243ACD5620E3EB152D54F6D4292A
:206660007926A9C5CE3B68C1171D2BCCA000EAC8A550ADD6124D6CD2CB6B2FDF7C76EEDB4A
:20668000C1CBA1E376D660E7AFF023EA18EDE2EE1DBDA5F0AAA064F4738627F9C49BE6FD6A
:2066A00009FDB889BEE0798D67C63A80D0DBFB84D58BBC9A62967D9EBBB03E930CADFF978A
:2066C000B110B0AF060D71ABDF2B32A66836F3A26D66B4BCDA7B75B8035D36B5B440F7B1AA
:2066E00039312921191109013B332B231B130B033D352D251D150D053F372F271F170F079A
:2067000038302820181008003A322A221A120A023C342C241C140C043E362E261E160E0699
:2067200027072F0F37173F1F26062E0E36163E1E25052D0D35153D1D24042C0C34143C1C29
:2067400023032B0B33133B1B22022A0A32123A1A2101290931113919200028083010381889
:206760002122232425262728292A2B2C2D2E2F303132333435363738393A3B3C3D3E3F4009
:206780000102030405060708090A0B0C0D0E0F101112131415161718191A1B1C1D1E1F20E9
:2067A000383028201810080039312921191109013A322A221A120A023B332B233E362E269D
:2067C0001E160E063D352D251D150D053C342C241C140C041B130B0300000D04100A1700EB
:2067E000000002091B0E051400001607120B031900000F01061A130C00002836331E242EA6
:2068000000001D2F27322C2000002B343026372100002D1F2931231C00001F04000102036C
:2068200000000308040506070000070C08090A0B00000B100C0D0E0F00000F141011121344
:2068400000001318141516170000171C18191A1B00001B001C1D1E1F1F0E272C3C1737245F
:20686000041E2E350C253E15050F2F1D3F360614261C3D0D2D1607340E040D01020F0B08D2
:20688000030A060C05090007000F07040E020D010A060C0B0905030804010E080D06020B11
:2068A0000F0C0907030A05000F0C080204090107050B030E0A00060D0F01080E060B0304E5
:2068C0000907020D0C00050A030D04070F02080E0C00010A06090B05000E070B0A040D01CA
:2068E00005080C060903020F0D080A01030F04020B06070C00050E090A00090E06030F05A6
:20690000010D0C070B0402080D0700090304060A0208050E0C0B0F010D060409080F03008B
:206920000B01020C050A0E07010A0D0006090807040F0E030B05020C070D0E030006090A63
:20694000010208050B0C040F0D080B05060F00030407020C010A0E090A0609000C0B070D41
:206960000F01030E05020804030F00060A010D080904050B0C07020E020C0401070A0B0636
:206980000805030F0D000E090E0B020C04070D0105000F0A030908060402010B0A0D070804
:2069A0000F090C050603000E0B080C07010E020D060F00090A0405030C010A0F09020608E0
:2069C000000D03040E07050B0A0F0402070C090506010D0E000B0308090E0F0502080C03C2
:2069E0000700040A010D0B060403020C09050F0A0B0E01070600080D040B020E0F00080DA8
:206A0000030C0907050A06010D000B070409010A0E03050C020F080601040B0D0C03070E88
:206A20000A0F060800050902060B0D0801040A070905000F0E02030C0D020804060F0B016B
:206A40000A09030E05000C07010F0D080A0307040C05060B000E0902070B0401090C0E0246
:206A600000060A0D0F03050802010E07040A080D0F0C09000305060B010102020202020254
:206A800001020202020202018040201008040201381000001A1002001910060018100A0014
:206AA00017100E001610160015101E00141022001310360012103A0011104600101056004A
:206AC0000F105E000E106E000D1082000C108E000B10A6000A10B2000910C2000810DA000A
:206AE0000710F2000610020105101E010410360103104E0102106E010110820100109E01CF
:206B0000FF0FBE01FE0FD601FD0FEE01FC0F0E02FB0F3202FA0F5602F90F7E02F80F9602E8
:206B2000F70FB202F60FE202F50F0203F40F2203F30F4E03F20F7E03F10FA203F00FDA032B
:206B4000EF0FFE03EE0F2E04ED0F5A04EC0F8E04EB0FB604EA0FEE04E90F2A05E80F5E0500
:206B6000E70FAE05E60FE205E50F2206E40F6E06E30FBE06E20F0A07E10F5E07E00FAA0760
:206B8000DF0FEE07DE0F5208DD0F9608DC0FDE08DB0F4E09DA0F9E09D90F020AD80F7A0A40
:206BA000D70FD20AD60F420BD50FA60BD40F2E0CD30FA20CD20FF60CD10F720DD00FE20D8F
:206BC000CF0F3A0ECE0FBE0ECD0F320FCC0F860FCB0FFE0FCA0F6E10C90FBA10C80F32115F
:206BE000C70F9611C60FD611C50F4212C40F9212C30FD612C20F2E13C10F7213C00FBE13FC
:206C0000BF0F0E14BE0F5214BD0F8614BC0FD214BB0F1A15BA0F4A15B90F9215B80FC2150C
:206C2000B70FFE15B60F3616B50F7216B40FA216B30FDE16B20F0E17B10F3617B00F6E17B6
:206C4000AF0FA617AE0FCA17AD0F0218AC0F3618AB0F5618AA0F9218A90FC218A80FE2186E
:206C6000A70F1A19A60F4A19A50F7219A40FA219A30FD219A20FF219A10F261AA00F561AFE
:206C80009F0F761A9E0FAE1A9D0FD21A9C0FFE1A9B0F261B9A0F4E1B990F721B980F9E1B54
:206CA000970FC21B960FE61B950F161C940F361C930F621C920F8A1C910FB61C900FD61C76
:206CC0008F0F021D8E0F261D8D0F461D8C0F781D8B0F961D8A0FBE1D890FF01D880F101EBD
:206CE000870F361E860F621E850F861E840FAA1E830FDA1E820FF61E810F1E1F800F4E1F0A
:206D00007F0F7A1F7E0F961F7D0FCA1F7C0FE61F7B0F06207A0F2820790F5620780F782067
:206D2000770F9620760FC820750FE620740F1421730F3621720F5A21710F8621700FA82124
:206D40006F0FD0216E0FF8216D0F20226C0F48226B0F66226A0F9822690FB622680FE82285
:206D6000670F0823660F3223650F5623640F8423630FB023620FC823610FFC23600F2824B6
:206D80005F0F48245E0F80245D0FA0245C0FBC245B0FF8245A0F1225590F3E25580F6425AC
:206DA000570F9025560FB425550FE825540F0626530F3426520F5826510F8426500FA826A8
:206DC0004F0FD8264E0F00274D0F2C274C0F64274B0F84274A0FB827490FD827480F082823
:206DE000470F2C28460F7028450F9028440FC028430FE828420F1829410F4C29400F7C2908
:206E00003F0FA4293E0FD4293D0FFC293C0F282A3B0F482A3A0F8C2A390FB02A380FDC2AD5
:206E2000370F082B360F3C2B350F702B340FA82B330FCC2B320FF82B310F382C300F642C28
:206E40002F0F882C2E0FCC2C2D0FF42C2C0F282D2B0F582D2A0F902D290FC42D280FF02DED
:206E6000270F242E260F582E250F882E240FBC2E230FF42E220F1C2F210F582F200F942F4F
:206E80001F0FBC2F1E0FEC2F1D0F2C301C0F54301B0F90301A0FC830190FF430180F283183
:206EA000170F6431160F8C31150FC831140FFC31130F2C32120F6C32110F9C32100FCC327E
:206EC0000F0F08330E0F3C330D0F6C330C0FAC330B0FCC330A0F1034090F4434080F803447
:206EE000070FA834060FE434050F2035040F4835030F8035020FB435010FE835000F1C362B
:206F0000FF0E5436FE0E8036FD0EB436FC0EF036FB0E1437FA0E4C37F90E7837F80EB4376D
:206F2000F70EE437F60E0C38F50E4438F40E7C38F30EAC38F20ED838F10E1439F00E3C3900
:206F4000EF0E7039EE0EA439ED0EDC39EC0E043AEB0E403AEA0E643AE90E9C3AE80ECC3A98
:206F6000E70E043BE60E243BE50E5C3BE40E883BE30EB03BE20EE03BE10E143CE00E383CC3
:206F8000DF0E6C3CDE0E9C3CDD0EC03CDC0EF43CDB0E243DDA0E483DD90E7C3DD80E9C3D81
:206FA000D70ECC3DD60E003ED50E303ED40E543ED30E883ED20EAC3ED10EDC3ED00E083F6D
:206FC000CF0E2C3FCE0E603FCD0E8C3FCC0EBC3FCB0EE03FCA0E0C40C90E3840C80E604092
:206FE000C70E8C40C60EAC40C50EDC40C40E1041C30E3841C20E5841C10E8441C00EB44114
:20700000BF0ED841BE0EFC41BD0E2C42BC0E4C42BB0E7442BA0EA042B90EC442B80EEC4206
:20702000B70E1043B60E3C43B50E6043B40E9043B30EB043B20ED843B10E0044B00E2C443A
:20704000AF0E5044AE0E7044AD0EA044AC0EC044AB0EF044AA0E1045A90E3045A80E604591
:20706000A70E8845A60EB045A50ED045A40E0046A30E2046A20E5446A10E7446A00E9446D3
:207080009F0EC4469E0EE8469D0E14479C0E44479B0E64479A0E8047990EB447980ED447FE
:2070A000970EF447960E2848950E4848940E7848930EA448920EC048910EE448900E184948
:2070C0008F0E3C498E0E68498D0E90498C0EB4498B0EE0498A0E0C4A890E304A880E504A45
:2070E000870E804A860EA84A850ED04A840EF44A830E204B820E404B810E744B800E9C4B54
:207100007F0EC84B7E0EFC4B7D0E204C7C0E504C7B0E704C7A0EA04C790EC04C780EF44CCD
:20712000770E244D760E444D750E7C4D740EA04D730ED04D720EF84D710E204E700E444E29
:207140006F0E744E6E0EA44E6D0EC44E6C0E004F6B0E284F6A0E504F690E804F680EA84F72
:20716000670ED44F660E1050650E3850640E6050630E9050620EC450610EDC50600E08514F
:207180005F0E40515E0E70515D0E9C515C0ED4515B0E08525A0E3052590E6052580E9452CB
:2071A000570EB852560EF052550E2053540E4853530E8053520EB053510EE053500E1454F8
:2071C0004F0E50544E0E70544D0EAC544C0ED8544B0E10554A0E4855490E8055480EAC5577
:2071E000470EE455460E1C56450E4456440E8856430EC056420EE456410E3057400E64574E
:207200003F0E94573E0ED0573D0E0C583C0E3C583B0E74583A0EB058390EE058380E205993
:20722000370E5059360E8C59350ECC59340E105A330E385A320E805A310EC45A300EF05A51
:207240002F0E405B2E0E705B2D0EB05B2C0EF45B2B0E305C2A0E685C290EB45C280EF05CF6
:20726000270E2C5D260E705D250EB45D240EF05D230E405E220E745E210EBC5E200E045FE1
:207280001F0E485F1E0E845F1D0ED05F1C0E0C601B0E4C601A0E9860190EE060180E1C611C
:2072A000170E7461160EBC61150EF461140E3C62130E8462120ED462110E2463100E706367
:2072C0000F0EAC630E0E04640D0E50640C0E84640B0EE0640A0E1865090E6465080EB4652C
:2072E000070E0466060E5066050E9866040EE866030E3867020E8867010ED867000E24683D
:20730000FF0D6868FE0DB868FD0D0869FC0D5869FB0DC069FA0DF869F90D5C6AF80DB46A99
:20732000F70DF06AF60D446BF50D946BF40DE46BF30D346CF20D886CF10DC86CF00D186DA5
:20734000EF0D686DEE0DB86DED0D086EEC0D6C6EEB0DA86EEA0DEC6EE90D606FE80DA06FD1
:20736000E70DF86FE60D4870E50D9870E40DE870E30D4C71E20D8871E10DD071E00D387269
:20738000DF0D7472DE0DCC72DD0D2473DC0D5C73DB0D9C73DA0D0074D90D4474D80D8874E8
:2073A000D70DF074D60D2875D50D6875D40DD075D30D0876D20D5876D10DA876D00DEC76DA
:2073C000CF0D3877CE0D8877CD0DD477CC0D2078CB0D7078CA0DA878C90DEC78C80D3C7937
:2073E000C70D8479C60DCC79C50D1C7AC40D4C7AC30D9C7AC20DDC7AC10D207BC00D5C7B8D
:20740000BF0D9C7BBE0DE47BBD0D1C7CBC0D6C7CBB0DA47CBA0DDC7CB90D2C7DB80D5C7D38
:20742000B70D9C7DB60DEC7DB50D147EB40D5C7EB30D8C7EB20DCC7EB10D147FB00D4C7FA8
:20744000AF0D847FAE0DBC7FAD0DFC7FAC0D3080AB0D7480AA0D9C80A90DE480A80D0C81FE
:20746000A70D4081A60D8481A50DAC81A40DE481A30D2082A20D6082A10D8482A00DBC8268
:207480009F0DEC829E0D20839D0D5C839C0D90839B0DB4839A0DEC83990D1C84980D488493
:2074A000970D8484960DAC84950DDC84940D1085930D4885920D6C85910DA085900DCC8567
:2074C0008F0DF8858E0D2C868D0D5C868C0D84868B0DB4868A0DE086890D1087880D4087CF
:2074E000870D6C87860D9087850DD087840DF087830D1888820D4C88810D7C88800D9C8894
:207500007F0DCC887E0DEC887D0D1C897C0D44897B0D6C897A0D9489790DC089780DE08929
:20752000770D0C8A760D388A750D608A740D808A730DA88A720DD08A710DF08A700D188B52
:207540006F0D388B6E0D608B6D0D848B6C0DB08B6B0DCC8B6A0DF08B690D148C680D308C41
:20756000670D548C660D708C650D948C640DBC8C630DE08C620DF88C610D1C8D600D388DE5
:207580005F0D588D5E0D808D5D0DA08D5C0DBC8D5B0DE08D5A0D048E590D1C8E580D408EC8
:2075A000570D608E560D788E550D9C8E540DB88E530DDC8E520DFC8E510D208F500D348FFD
:2075C0004F0D508F4E0D708F4D0D908F4C0DA88F4B0DD48F4A0DEC8F490D0C90480D2C907D
:2075E000470D4490460D6090450D8090440D9C90430DB490420DD490410DF490400D0C913E
:207600003F0D38913E0D50913D0D6C913C0D90913B0DAC913A0DC891390DE491380D0892B9
:20762000370D2892360D5092350D6892340D8092330DB492320DCC92310DF092300D1493D1
:207640002F0D3C932E0D60932D0D90932C0DB4932B0DE8932A0D1494290D3C94280D6C9447
:20766000270D9094260DC094250DF494240D3095230D5095220D8095210DB895200DDC9509
:207680001F0D0C961E0D40961D0D64961C0D90961B0DC8961A0DEC96190D1C97180D509794
:2076A000170D7097160DA097150DD497140DF497130D2498120D4C98110D7898100D9C98AE
:2076C0000F0DD0980E0DF0980D0D20990C0D44990B0D6C990A0D9099090DC099080DE89958
:2076E000070D089A060D449A050D5C9A040D809A030DB89A020DD49A010DF09A000D289B69
:20770000FF0C449BFE0C609BFD0C949BFC0CB49BFB0CD09BFA0C009CF90C209CF80C409C36
:20772000F70C709CF60C889CF50CA89CF40CC89CF30CEC9CF20C109DF10C2C9DF00C509D8A
:20774000EF0C689DEE0C849DED0CA49DEC0CC89DEB0CDC9DEA0CFC9DE90C149EE80C309E0F
:20776000E70C4C9EE60C649EE50C7C9EE40C949EE30CAC9EE20CC09EE10CD89EE00CE89EB1
:20778000DF0C049FDE0C189FDD0C289FDC0C3C9FDB0C549FDA0C609FD90C749FD80C849F89
:2077A000D70C989FD60CA49FD50CB89FD40CC49FD30CD49FD20CE49FD10CF49FD00C00A070
:2077C000CF0C10A0CE0C18A0CD0C28A0CC0C34A0CB0C40A0CA0C4CA0C90C58A0C80C64A021
:2077E000C70C70A0C60C7CA0C50C84A0C40C90A0C30C9CA0C20CA4A0C10CB0A0C00CB8A065
:20780000BF0CC0A0BE0CCCA0BD0CD4A0BC0CDCA0BB0CE8A0BA0CF0A0B90CF8A0B80C04A11B
:20782000B70C0CA1B60C14A1B50C1CA1B40C24A1B30C2CA1B20C34A1B10C3CA1B00C44A104
:20784000AF0C4CA1AE0C54A1AD0C5CA1AC0C64A1AB0C6CA1AA0C74A1A90C7CA1A80C84A124
:20786000A70C8CA1A60C90A1A50C98A1A40CA0A1A30CA8A1A20CB0A1A10CB4A1A00CBCA168
:207880009F0CC4A19E0CC8A19D0CD0A19C0CD8A19B0CE0A19A0CE4A1990CECA1980CF4A1CC
:2078A000970CFCA1960C04A2950C08A2940C10A2930C14A2920C1CA2910C24A2900C28A229
:2078C0008F0C30A28E0C34A28D0C3CA28C0C40A28B0C48A28A0C50A2890C54A2880C5CA2B4
